:0200000480007A
:10000000970500009385C506130540006B10B500E9
:10001000EF00C005130510006B0005001385811D5E
:10002000138681233306A64093050000EF30400C71
:100030001715000013054559EF00505FEF20C0551C
:10004000130540006B000500EF00D0206F00505FEB
:10005000B707000093870700638807003715008003
:100060001305455C6F00905C67800000130540003D
:100070006B000500978101009381C1A7F326100250
:100080009396A601732600029315A6001316260068
:1000900037F1FF6F3301B1403301D1403301C1006B
:1000A000F326100263860600130500006B000500AE
:1000B00067800000130101FD232681021304010360
:1000C000232EA4FC232CB4FC232AC4FC8327C4FDC8
:1000D00083A707002326F4FE930744FD2322F4FEA2
:1000E000832744FE03C707008327C4FE2380E7005D
:1000F0008327C4FE93871700032744FE0347170096
:100100002380E7008327C4FE93872700032744FE4C
:10011000034727002380E7008327C4FE9387370027
:10012000032744FE034737002380E7008327C4FEEC
:10013000938747002326F4FE232404FE832744FDEF
:10014000032784FE635CF702832784FE032784FD74
:10015000B307F70003C707008327C4FE2380E70027
:100160008327C4FE938717002326F4FE832784FE8B
:10017000938717002324F4FE6FF05FFC8327C4FEEF
:100180002320F4FE832704FE93F73700032704FEA1
:10019000B307F7002320F4FE832704FE2326F4FE92
:1001A0008327C4FD0327C4FE23A0E700130000003B
:1001B0000324C1021301010367800000130101FC45
:1001C000232E8102130401042326A4FC2324B4FC5F
:1001D0008327C4FC83A707002326F4FE9307C4FDEE
:1001E0002322F4FE8327C4FE03C70700832744FEAF
:1001F0002380E700832744FE938717000327C4FE6C
:10020000034717002380E700832744FE93872700D6
:100210000327C4FE034727002380E700832744FE0B
:10022000938737000327C4FE034737002380E70086
:100230008327C4FE938747002326F4FE232404FE6D
:100240008327C4FD032784FE635CF702832784FEB3
:10025000032784FCB307F7000327C4FE0347070006
:100260002380E7008327C4FE938717002326F4FE2C
:10027000832784FE938717002324F4FE6FF05FFC2E
:100280008327C4FE2320F4FE832704FE93F7370060
:10029000032704FEB307F7002320F4FE832704FEA0
:1002A0002326F4FE8327C4FC0327C4FE23A0E70013
:1002B000130000000324C103130101046780000040
:1002C000130101FF23268100130401011300000024
:1002D0000324C1001301010167800000130101FE26
:1002E000232E8100130401022326A4FE2324B4FE3E
:1002F000832784FE3727000023A2E700930700002E
:10030000138507000324C101130101026780000067
:10031000130101FE232E1100232C8100130401027E
:100320002326A4FEB757018013858717EF00C04F1F
:1003300093071000138507008320C1010324810166
:100340001301010267800000130101FD2326110241
:100350002324810213040103232EA4FC232CB4FCC8
:10036000232AC4FCB70700712326F4FEB7070072E6
:100370002324F4FE930730002322F4FE130744FEE7
:100380009307C4FE1306400093050700138507007A
:10039000EFF05FD21307C4FD9307C4FE13064000BD
:1003A0009305070013850700EFF0DFD0130784FDE6
:1003B0009307C4FE1306400093050700138507004A
:1003C000EFF05FCF130744FD9307C4FE1306400010
:1003D0009305070013850700EFF0DFCD83A7C11B4E
:1003E000E7800700130704FE930784FE93050700C8
:1003F00013850700EFF09FDC832704FE13850700B9
:100400008320C102032481021301010367800000DD
:10041000130101FD23261102232481021304010389
:10042000232EA4FC232CB4FC232AC4FCB7070071A0
:100430002324F4FEB70700722326F4FE930740003E
:100440002322F4FE130744FE930784FE13064000A4
:100450009305070013850700EFF0DFC51307C4FD00
:10046000930784FE130640009305070013850700D9
:10047000EFF05FC4130784FD930784FE130640006A
:100480009305070013850700EFF0DFC2130744FD53
:10049000930784FE130640009305070013850700A9
:1004A000EFF05FC183A7C11BE7800700832744FDEE
:1004B000138507008320C102032481021301010375
:1004C00067800000130101FD23261102232481020D
:1004D00013040103232EA4FC232CB4FC232AC4FC04
:1004E000B70700712326F4FE930750002324F4FE7F
:1004F000130784FE9307C4FE13064000930507000C
:1005000013850700EFF01FBB1307C4FD9307C4FE5C
:10051000130640009305070013850700EFF09FB90D
:100520009307C4FE032644FD832584FD138507003D
:10053000EFF05FB883A7C11BE7800700832744FD66
:10054000138507008320C1020324810213010103E4
:1005500067800000130101FD2326810213040103BB
:10056000232EA4FC8327C4FD63D807008327C4FD82
:10057000B307F040232EF4FC0327C4FDB737000077
:100580009387078063D8E700B73700009387078019
:10059000232EF4FC83A7011C2326F4FE03A7011CD1
:1005A0008327C4FD3307F70023A0E11C8327C4FE83
:1005B000138507000324C1021301010367800000B3
:1005C000130101FE232E1100232C810013040102CC
:1005D0002326A4FE13050000EF00001E13000000F8
:1005E0008320C101032481011301010267800000FF
:1005F000130101FD232611022324810213040103A8
:10060000232EA4FC232CB4FC232AC4FCB7070071BE
:100610002326F4FEB70700722324F4FE930770002C
:100620002322F4FE130744FE9307C4FE1306400082
:100630009305070013850700EFF0DFA71307C4FD3C
:100640009307C4FE130640009305070013850700B7
:10065000EFF05FA6130784FD9307C4FE1306400066
:100660009305070013850700EFF0DFA4130744FD8F
:100670009307C4FE13064000930507001385070087
:10068000EFF05FA383A7C11BE7800700130704FEF9
:10069000930784FE9305070013850700EFF01FB250
:1006A000832704FE138507008320C10203248102EF
:1006B0001301010367800000130101FF23261100CD
:1006C0002324810013040101B75701801385C71843
:1006D000EF008015130000008320C1000324810077
:1006E0001301010167800000130101FF232611009F
:1006F0002324810013040101EF00800E93070500FD
:10070000138507008320C100032481001301010128
:1007100067800000130101FF2326110023248100BC
:1007200013040101B75701801385071BEF00C00FA9
:10073000130000008320C100032481001301010184
:1007400067800000130101FF23261100232481008C
:1007500013040101B75701801385471DEF00C00C3A
:1007600083A7811E9386170023A4D11E138507003B
:100770008320C10003248100130101016780000070
:10078000130101FF2326110023248100130401011A
:10079000B757018013850720EF0000091300000000
:1007A0008320C10003248100130101016780000040
:1007B0006B10B500678000006B00050067800000CB
:1007C0006B40B500678000006B200500678000006B
:1007D0006B30000067800000732510026780000006
:1007E0007325000267800000130540006B000500C0
:1007F000F32610029396F600732600029315A600C6
:100800001316260037F1FF6F3301B1403301D14099
:100810003301C100F32610026386060013050000B1
:100820006B00050067800000130141FF23201100C9
:100830002322B1008345050063880500EF00C00155
:10084000130515006FF01FFF832001008325410071
:100850001301C10067800000B702010023A0B200AD
:1008600067800000130101FC232E810213040104A0
:10087000232EA4FC232CB4FC232AC4FC2328D4FC60
:100880002326E4FC2324F4FC03A7C11E93071000D5
:100890006316F7009307F0FF6F00000883A7C11EDF
:1008A0009386170023A6D11E13870700930707001E
:1008B00093971700B387E7009397370013870700D4
:1008C0009387011FB307F7002326F4FE8327C4FE96
:1008D0000327C4FD23A0E7008327C4FE032784FD6C
:1008E00023A2E7008327C4FE032744FD23A4E700D7
:1008F0008327C4FE032704FD23A6E7008327C4FE45
:100900000327C4FC23A8E7008327C4FE032784FC35
:1009100023AAE70093070000138507000324C103FF
:100920001301010467800000130101FC232E110252
:10093000232C810213040104232EA4FC232CB4FCD9
:10094000232AC4FC2328D4FC2326E4FC2324F4FC1F
:10095000232604FE83A7C11E0327C4FE6350F70E9F
:100960000327C4FE9307070093971700B387E70098
:1009700093973700138707009387011FB307F7008A
:100980002324F4FE832784FE83A707008325C4FD68
:1009900013850700EF20105193070500B337F000CF
:1009A00093F7F70F63920708832784FD638A070094
:1009B000832784FE03A74700832784FD23A0E70045
:1009C000832744FD638A0700832784FE03A78700EB
:1009D000832744FD23A0E700832704FD638A0700E3
:1009E000832784FE03A7C700832704FD23A0E70015
:1009F0008327C4FC638A0700832784FE03A70701BB
:100A00008327C4FC23A0E700832784FC638A0700B4
:100A1000832784FE03A74701832784FC23A0E700E4
:100A2000930700006F00C001130000008327C4FE7D
:100A3000938717002326F4FE6FF0DFF19307F0FF92
:100A4000138507008320C1030324810313010104DC
:100A500067800000130101FC232E1102232C810268
:100A6000130401042326A4FC2324B4FC1305100062
:100A7000EFF09FD4B757018013854726EF20100071
:100A8000B75701809385472AB75701801385872A76
:100A9000EF00904B930705002326F4FE1306200079
:100AA000930500000325C4FEEF1040360325C4FE65
:100AB000EF10D005930705002324F4FE1306000071
:100AC000930500000325C4FEEF104034832784FE05
:100AD0009387170013850700EF10D0549307050084
:100AE0002322F4FE832784FE8326C4FE1386070098
:100AF00093051000032544FEEF00506C0325C4FE4F
:100B0000EF000048832784FE032744FEB307F70065
:100B100023800700832544FEB75701801385C72D26
:100B2000EF20C07513050000EF008031130101FFB5
:100B30002326110023248100130401011385811D44
:100B4000EF004001032481008320C1001301010153
:100B500067800000130101FF232611002324810078
:100B600013040101232AA4FE375501801305F52D36
:100B7000B7150080938505CA1387811C9387812050
:100B80001306300093060000EFF0DFCD0324810050
:100B90008320C1001301010167800000130101FFE0
:100BA000232611002324810013040101EFF01FF814
:100BB000032481008320C10013010101678000002C
:100BC000130101FE232E1100232C8100232A910002
:100BD000232821012326310123244101232251010D
:100BE000130401021371C1FF138906009309060063
:100BF000138A0500930A050083A486011385040067
:100C00009305070097400100E780404C8325C90009
:100C10003385A50013152500B382AA003303AA006B
:100C2000B383A90003280902032EC9019308000019
:100C3000930E000013850200930503001386030042
:100C4000930700000327050083A60500B386E6008E
:100C50002320D60013054500938545001306460062
:100C600093871700E3E097FE938E1E00E3E4CEFD2A
:100C700093881800E3EE08FB130104FE832A410069
:100C8000032A81008329C100032901018324410132
:100C9000032481018320C101130101026780000048
:100CA000130101FF23261100232481002322910038
:100CB00023202101938405001309050003A4850165
:100CC000130504009305060097400100E7800040EB
:100CD00083A5C4003385A50013152500832589004D
:100CE00083A5050003264900032606008326090084
:100CF00083A60600B382A6003303A600B383A50033
:100D000003A8040203AEC40193080000930400008A
:100D10001385020093050300138603009307000068
:100D20008326050003A70500B306D7002320D600BD
:100D30001305450093854500130646009387170069
:100D4000E3E087FE93841400E3E4C4FD9388180075
:100D5000E3EE08FB03290100832441000324810002
:100D60008320C1001301010167800000130101FF0E
:100D70002326110023248100232291002320210116
:100D8000938405001309050003A4850113050400DD
:100D90009305060097400100E780403383A5C40017
:100DA0003385A500131525008325890003264900F6
:100DB00083260900B382A6003303A600B383A500EF
:100DC00003A8040203AEC4019308000093040000CA
:100DD00013850200930503001386030093070000A8
:100DE0008326050003A70500B306D7002320D600FD
:100DF00013054500938545001306460093871700A9
:100E0000E3E087FE93841400E3E4C4FD93881800B4
:100E1000E3EE08FB03290100832441000324810041
:100E20008320C100130101016780000093050500C4
:100E30009306000013060000130500006F500071B8
:100E4000130101FF930500002324810023261100D4
:100E500013040500EF50007903A5811B8327C50308
:100E600063840700E780070013050400EFF04FF5E7
:100E7000130101FF23261100232481002322910066
:100E800023202101638005021384050093040500DB
:100E90006306050083278503638C070A8317C40054
:100EA000639207028320C10003248100130900001C
:100EB00083244100130509000329010013010101E6
:100EC000678000009305040013850400EF00000C08
:100ED0008327C40213090500638A07008325C40120
:100EE00013850400E7800700634C05068357C400A0
:100EF00093F70708639E070683250403638C0500A8
:100F0000930704046386F50013850400EF00D03FC7
:100F10002328040283254404638805001385040004
:100F2000EF00903E23220404EF00C0662316040065
:100F3000EF0080668320C1000324810083244100E8
:100F40001305090003290100130101016780000056
:100F5000EF0040638317C400E38607F46FF09FF649
:100F60008357C4001309F0FF93F70708E38607F8D7
:100F70008325040113850400EF0010396FF0DFF7BB
:100F80009305050003A5C11C6FF09FEE8397C50074
:100F9000130101FE232C810023263101232E110091
:100FA000232A91002328210193F68700138405004A
:100FB00093090500639A061037170000130707808E
:100FC00083A64500B3E7E7002396F5006354D018E5
:100FD00003278402630A070C83A409009396070180
:100FE00023A00900139637018325C40193D6060177
:100FF00063480616930610001306000013850900C7
:10100000E70007009307F0FF630CF5188356C40050
:10101000032784028325C40193F64600638E0600ED
:1010200083264400832704033305D54063860700E5
:101030008327C4033305F54013060500930600001B
:1010400013850900E70007009307F0FF631EF51002
:1010500003A709008317C400630807169306D0018D
:101060006306D700930660016314D70C832604013E
:1010700037F7FFFF1307F77FB3F7E7002316F400F6
:10108000232204002320D4008325040323A09900F5
:10109000638C0500930704046386F500138509003B
:1010A000EF00902623280402130500008320C101CD
:1010B0000324810183244101032901018329C10003
:1010C000130101026780000003A90501E30E09FC7A
:1010D00083A40500139707011357070113773700FF
:1010E00023A02501B3842441930700006314070063
:1010F00083A745012324F400634890006FF0DFFAD2
:101100003309A900E35290FA832744028325C401DE
:10111000938604001306090013850900E780070081
:10112000B384A440E34EA0FC8357C4001305F0FF32
:1011300093E707048320C1012316F40003248101EF
:1011400083244101032901018329C1001301010204
:101150006780000003A7C503E34CE0E66FF0DFF40F
:10116000032504056FF05FEB8357C40037F7FFFFDB
:101170001307F77FB3F7E70083260401939707016E
:1011800093D707412316F400232204002320D40020
:1011900013973701E35A07EE2328A4046FF0DFEE1C
:1011A00083A70900E38407E61307D0016388E702F9
:1011B000130760016384E7028357C40093E70704C1
:1011C0002316F4006FF09FEE37F7FFFF1307F77F4A
:1011D00083260401B3F7E7006FF0DFFA23A099003C
:1011E000130500006FF09FEC130101FE232C81001A
:1011F000232E1100130405006306050083278503D1
:10120000638007028397C500639607028320C101AC
:10121000032481011305000013010102678000000F
:101220002326B100EF0000368325C1008397C50057
:10123000E38E07FC13050400032481018320C10110
:10124000130101026FF09FD49305050063060500AA
:1012500003A5C11C6FF05FF903A5811BB7150080C2
:101260009385851E6F10002813050000678000001D
:10127000B7150080938505E76F10C026130101FEA6
:10128000B7170080232E1100232C8100232A910000
:101290002328210123263101232441012322510146
:1012A000232061010324450093870727232EF5029D
:1012B0001307C52E930730002324E52E2322F52E95
:1012C0002320052E93074000130905002326F40070
:1012D0001306800093050000232204062320040047
:1012E000232204002324040023280400232A0400CA
:1012F000232C04001305C405EF10905F373B0080DA
:1013000083248900B73A0080373A0080B7390080DB
:10131000130B8B54938ACA5A130A4A639389C96977
:10132000B70701002320640323225403232444032A
:1013300023263403232E84009387970023A6F400EA
:10134000130680009305000023A2040623A00400D6
:1013500023A2040023A4040023A8040023AA040059
:1013600023AC04001385C405EF1090580324C90072
:10137000B707020023A0640323A2540323A4440359
:1013800023A6340323AE9400938727012326F40079
:101390002322040623200400232204002324040023
:1013A00023280400232A0400232C04001305C40569
:1013B0001306800093050000EF1090538320C101B5
:1013C00023206403232254032324440323263403C9
:1013D000232E84000324810193071000232CF9029B
:1013E00083244101032901018329C100032A8100CB
:1013F000832A4100032B01001301010267800000D2
:101400001305000067800000130101FF23229100F3
:10141000130680069384F5FFB384C40223202101C0
:101420001389050023248100232611009385440796
:10143000EF10C04013040500630005021305C5004A
:1014400023200400232224012324A40013868406DD
:1014500093050000EF10D0498320C100130504005C
:1014600003248100832441000329010013010101A9
:1014700067800000130101FE2328210103A9811BBD
:1014800023263101232E110083278903232C810079
:10149000232A9100930905006386070A1309092E80
:1014A0009304F0FF83274900032489009387F7FF03
:1014B00063D807006F00000813048406638C970646
:1014C0000317C4009387F7FFE31807FEB707FFFF72
:1014D00093871700232204062320040023220400FC
:1014E000232404002326F40023280400232A0400D4
:1014F000232C040013068000930500001305C40587
:10150000EF10103F23280402232A0402232204049C
:10151000232404048320C101130504000324810152
:1015200083244101032901018329C1001301010220
:101530006780000003240900630C04001309040001
:101540006FF05FF613050900EFF05FD36FF01FF542
:101550009305400013850900EFF01FEB2320A9003D
:1015600013040500E31C05FC9307C00023A0F90049
:101570006FF05FFA03A5811BB7150080938505E71F
:101580006F0050768327850363840700678000001F
:101590006FF0DFCE6780000067800000678000008A
:1015A0006780000003A5C11CB715008093858526C0
:1015B0006F00106903A5C11CB71500809385054015
:1015C0006F001068130101FF23248100B7770180A9
:1015D000377401801304C42E9387C72EB3878740C6
:1015E000232291002326110093D427406380040214
:1015F0009387C7FF33848700832704009384F4FF15
:101600001304C4FFE7800700E39804FE8320C100B1
:10161000032481008324410013010101678000003D
:10162000130101FD13070600232E31011306C1002B
:101630009389050093050700232021032326110227
:10164000232481022322910213090500EF50401147
:101650006300050A9304050013050900EFF09FE1FC
:1016600013040500630605080326C1009306601BEA
:101670009385090013050900EF10D0356344050672
:10168000B7370080938787542320F402B737008050
:101690009387C75A2322F402B737008093874763A2
:1016A0002324F402B73700809387C7692316940078
:1016B0002317A400232E84002326F40293F404109D
:1016C000639A04048320C1021305040003248102E9
:1016D00083244102032901028329C101130101036B
:1016E00067800000EFF01FEB23160400EFF0DFEA45
:1016F000130400008320C1021305040003248102A7
:1017000083244102032901028329C101130101033A
:10171000678000009305040013050900930620006C
:1017200013060000EF00406E8320C1021305040081
:101730000324810283244102032901028329C10178
:1017400013010103678000009307050003A5C11C76
:1017500013860500938507006FF09FEC130101FDD0
:1017600023286101338BC602232611022324810220
:101770002322910223202103232E3101232C410116
:10178000232A51012326710123248101232291015F
:1017900063080B12930A0600938B0600130A0500D8
:1017A00013890500130407006306050083278503DA
:1017B0006380071E8317C4001397070193962701C0
:1017C0001357070163CA060203274406B726000021
:1017D000B3E7D700B7E6FFFF939707019386F6FFBD
:1017E00093D707413377D7002322E40613970701E5
:1017F0002316F40013570701832444009386040042
:1018000063C00416937727008325040093090B0017
:10181000638E071063EC661913860900130509002F
:10182000EF10407B03270400832744008325040333
:1018300033073701B38737412320E4002322F40024
:10184000B3043B41638E05006386041693070404CA
:101850006386F50013050A00EF00002B232804021D
:10186000330939016F0080009304070093050400D9
:1018700013050A0063800414832C040183290400E7
:10188000032C44012328240123202401232A94002B
:10189000EF1050258327440023289401232A840134
:1018A00023203401232204003387F4403309F90054
:1018B000E30C05FA338B6701B3049B4033DB54031D
:1018C0008320C102032481028324410203290102EF
:1018D0008329C101032A8101832A4101832BC1008D
:1018E000032C8100832C410013050B00032B010105
:1018F0001301010367800000EF10C06D832704000F
:101900009305040013050A00B38797002320F40011
:10191000EF10501DB38799403309990063120506F3
:101920008325040083244400938907001386040060
:1019300013050900E3E234FD13860900EF10806906
:101940008327440083240400138B0B00B3873741A3
:10195000B38434012322F400232094006FF05FF657
:1019600023220400937727008325040093060000B8
:101970009304000093090B00E38A07FA6FF09FE9D4
:10198000B3846401B384344133DB54036FF05FF3F9
:10199000EFF05FBF8317C4001397070193962701E9
:1019A00013570701E3CA06E46FF01FE293890600AC
:1019B0006FF09FE6138B0B006FF09FF0930705000D
:1019C00003A5C11C138706009306060013860500B5
:1019D000938507006FF09FD8130101FE2326310184
:1019E000232C8100232A9100232821012324410153
:1019F000232E1100138A050013090500938981C263
:101A0000EF10C07C03A78900B71700001384F7FE0E
:101A1000832447003304444193F4C4FF3304940007
:101A20001354C4001304F4FF1314C400634EF400F1
:101A30009305000013050900EF10502B83A78900C0
:101A4000B38797006308F50213050900EF1040788B
:101A50008320C10103248101832441010329010161
:101A60008329C100032A810013050000130101022C
:101A700067800000B305804013050900EF101027B0
:101A80009307F0FF6308F5049387C12003A70700BD
:101A900083A68900B384844093E414003304874010
:101AA0001305090023A2960023A08700EF104072BF
:101AB0008320C10103248101832441010329010101
:101AC0008329C100032A81001305100013010102BC
:101AD000678000009305000013050900EF10102136
:101AE00003A789009306F000B307E540E3DEF6F4B0
:101AF00083A6011D93E717002322F7003305D54085
:101B000023A6A1206FF05FF463840512130101FF87
:101B100023248100232291001384050093040500EF
:101B200023261100EF10806A0328C4FF130784FFE7
:101B30009377E8FF3306F700938581C2832646003A
:101B400003A5850093F6C6FF6306C51A2322D600B7
:101B5000137818003305D600631E0808032384FF9A
:101B6000032845003307674083288700138501C396
:101B7000B387670013781800638EA8120323C70089
:101B800023A6680023241301630E081C93E61700A4
:101B90002322D7002320F6009306F01F63E6F60AFF
:101BA00093F687FF9386860003A54500B386D5008C
:101BB00003A6060013D8570093071000B397070138
:101BC000B3E7A700138586FF2326A7002324C700B9
:101BD00023A2F50023A0E6002326E60003248100CB
:101BE0008320C100138504008324410013010101F7
:101BF0006F10005E0325450013751500631C050278
:101C0000B387D700138501C38326860093E81700A6
:101C10003308F7006384A6160326C60023A6C60071
:101C20002324D600232217012320F8006FF0DFF6CB
:101C30006780000093E61700232ED4FE2320F600D1
:101C40009306F01FE3FEF6F493D6970013064000C8
:101C50006368D60E93D667001388960313868603AF
:101C6000131838003388050183260800130888FFFD
:101C70006304D81203A646001376C6FF63F6C700B6
:101C800083A68600E318D8FE03A8C6002326070112
:101C90002324D700032481008320C1002324E800EB
:101CA000138504008324410023A6E60013010101EB
:101CB0006F100052631208148325C60003268600A5
:101CC000B387F600032481002326B60023A4C500B1
:101CD00093E617008320C1002322D7001385040058
:101CE0003307F700832441002320F700130101018B
:101CF0006F10004E13781800B387D70063100802E6
:101D0000032584FF3307A7408326C70003268700E7
:101D1000B387A7002326D60023A4C60013E6170026
:101D200083A6411D2322C70023A4E500E3E8D7EAE8
:101D300083A5411E13850400EFF01FCA6FF01FEA50
:101D4000130640016374D602130640056364D60689
:101D500093D6C7001388F6061386E60613183800D4
:101D60006FF05FF0B387D7006FF01FEA1388C605E6
:101D70001386B605131838006FF0DFEE23AAE500CE
:101D800023A8E5002326A7002324A7002322170168
:101D90002320F8006FF09FE403A54500135626406A
:101DA000930710003396C7003366A60023A2C50030
:101DB0006FF0DFED13064015636CD60093D6F70085
:101DC0001388860713867607131838006FF09FE98B
:101DD00013064055636CD60093D627011388D607A7
:101DE0001386C607131838006FF0DFE71308803F2B
:101DF0001306E0076FF01FE793E617002322D700D2
:101E00002320F6006FF09FDD6F00C00193070500EF
:101E100003A5C11C930606001386050093850700E1
:101E20006F004000130101F7232481082322910849
:101E300023202109232C410723261108232E3107B3
:101E4000232A5107232861072326710793040500DD
:101E500013840500130A06001389060063060500B3
:101E600083278503638407068357C4001307801004
:101E700093F787106386E706832A840263800A400B
:101E800093071000630CF9129379D9FF6382090656
:101E90009307600123A0F4009309F0FF8320C10899
:101EA000032481088324410803290108032A8107A8
:101EB000832A4107032B0107832BC10613850900E1
:101EC0008329C1071301010967800000EFF08FEB40
:101ED0008357C4001307801093F78710E39EE7F839
:101EE0009305040013850400EFF00FB06FF0DFF8E6
:101EF00003270401930B0000630A07128316C40032
:101F0000B71700009387A78113970601135707019E
:101F1000B377F7006394070213770740631007163F
:101F2000B737008093874763638AFA10B7170000BA
:101F300093870780B3E6F6002316D40093050400C8
:101F400013850400EFF04FAA93090500E31605F48A
:101F50008325C4019306090013060A0013850400B3
:101F6000E7800A009307F0FFE308F5F283250403F6
:101F7000638C0500930704046386F5001385040051
:101F8000EFF09FB8232804028357C400832604017E
:101F900037F7FFFF1307F77DB3F7E7002320D400DF
:101FA000232204002316F40013068000930500008A
:101FB0001305C405EF10C0136FF05FEE9305040026
:101FC00013850400EFF04FA28357C4001397370125
:101FD0006344070E8325C401930610001306000016
:101FE00013850400E7800A009307F0FF93090500BA
:101FF000E304F5EA8357C4000327040193F647007E
:102000006384060C8327440083260403B389F940C4
:10201000638606008326C403B389D940930B090065
:10202000330A3A0113090000E31A07EC9305040090
:1020300013850400EF00006D6FF05FEC8315E40082
:10204000E3C605EE1306810013850400EF0080252A
:10205000631A051C8326C100B7F70000378700000C
:10206000B3F7D7008316C400E392E7EC93E606408B
:10207000930700402326F4042316D400130B0A0010
:102080006310091463900B068357C400139737013C
:10209000635A071603250405832744008325040398
:1020A00013870700B309F540638005148326C40332
:1020B000B389D9406F00000493F6470083290405D3
:1020C00003270401E39006F493F78700E38807F4FD
:1020D00083270400E38407F4B387E740B389F9005A
:1020E0006FF0DFF383250403638E050E832744001E
:1020F0008326C4030327840303260401B389F9005C
:10210000B307C740B389F940B387D70063463B01A3
:102110003387F900636CEB108329C4048325C40161
:1021200093060000B3093041B3F969011386090031
:1021300013850400E7800A009307F0FFE300F5E051
:102140008327040183250403232204002320F400B1
:10215000638C0500930704046386F500138504006F
:10216000EFF09F9A232804028357C400B30B3B412E
:1021700093F7F7FD2316F40063083B03930504006F
:1021800013850400EF100016E31A05DA83274400D4
:10219000E3E677DB03270400B38777412322F400CB
:1021A000B30B770123207401130680009305000010
:1021B0001305C405EF00D073930900006FF01FCE24
:1021C0008315E4001306810013850400EF00800DE1
:1021D000E31605D6032B8101330B6A01E3940BF060
:1021E0006FF09FEA032744008327040003260401BD
:1021F00093050000B387C740B389F940B307F700E0
:102200006FF0DFF08325C401930610001306000071
:1022100013850400E7800A009307F0FFE31EF5E64C
:102220006FF0DFD18316C4006FF05FD0B3093B417C
:1022300033063601B38937412320C40023223401F9
:10224000638C0500930704046386F500138504007E
:10225000EFF09F8B232804028357C40013068000ED
:102260009305000093F7F7FD2316F4001305C4054A
:10227000EF001068930900006FF05FC29307D00170
:1022800023A0F4009309F0FF6FF05FC193070500EE
:1022900003A5C11C9306060013860500938507005D
:1022A0006FF05FB8130101FF13870500232481003D
:1022B000232291001304050093050600130507006F
:1022C0002326110023AA0122EFE04F819307F0FF9C
:1022D000630CF5008320C1000324810083244100A6
:1022E000130101016780000083A74123E38407FEF7
:1022F0008320C1002320F4000324810083244100B3
:1023000013010101678000006F00000193050500C3
:1023100003A5C11C6F004000130101FF23248100AD
:102320002322910023261100930405001384050045
:102330006306050083278503638A070A032784024F
:10234000630E070C8357C4009306800013F6C70082
:102350006302D60A9396370163CC06048325C40131
:10236000930610001306000013850400E700070021
:102370009307F0FF630CF50A8357C40013F7470077
:10238000630E070203274400832704033305E54057
:10239000638607008327C4033305F5408320C1000B
:1023A00003248100832441001301010167800000A0
:1023B00013F7470003250405E31607FC93F787008E
:1023C000E38E07FC83270400E38A07FC032704014C
:1023D0008320C10003248100B387E74083244100A8
:1023E0003305F5001301010167800000EFF08F99BC
:1023F0006FF0DFF483260400E38E06F40326040165
:10240000B386C640E358D0F493F60710E38406F48D
:102410008325C401930620006FF0DFF49307D001F9
:1024200023A0F4001305F0FF6FF05FF71305F0FF32
:102430006FF0DFF69305050003A5C11C6FF0DFED1B
:10244000130101FE23282101232631012324410108
:102450002322510123206101232E1100232C81000E
:10246000232A9100138B0500930A052E130A0000FE
:10247000930910001309F0FF83A44A0003A48A0003
:102480009384F4FF63C604028357C4009384F4FF6B
:1024900063FCF9008317E400130504006386270139
:1024A000E7000B00336AAA0013048406E39E24FDB0
:1024B00083AA0A00E3920AFC8320C101032481015C
:1024C00083244101032901018329C100832A41009A
:1024D000032B010013050A00032A810013010102E6
:1024E00067800000130101FD23202103232E310109
:1024F000232C4101232A5101232861012326710144
:10250000232611022324810223229102930A05002B
:10251000938B0500130B052E130A0000930910007E
:102520001309F0FF83244B0003248B009384F4FFF2
:1025300063C804028357C4009384F4FF63FEF90068
:102540008317E4009305040013850A0063862701BE
:10255000E7800B00336AAA0013048406E39C24FD81
:10256000032B0B00E3100BFC8320C1020324810228
:1025700083244102032901028329C101832A4101E5
:10258000032B0101832BC10013050A00032A8101DB
:102590001301010367800000130101FF2324810060
:1025A0002320210137740180377901809307442E5D
:1025B0001309492E3309F9402326110023229100E3
:1025C00013592940630009021304442E93040000A8
:1025D000832704009384140013044400E780070059
:1025E000E31899FE37740180377901809307442EF0
:1025F0001309C92E3309F940135929406300090210
:102600001304442E930400008327040093841400D1
:1026100013044400E7800700E31899FE8320C100FB
:1026200003248100832441000329010013010101D7
:1026300067800000130101F923248106138405003B
:102640008395E500232291062320210723261106E6
:10265000930406001389060063CA0504130681006B
:10266000EFF05FC4634405040327C100B7F700001F
:102670008320C106B3F7E70037E7FFFFB387E70022
:102680000324810693B717002320F9009307004025
:1026900023A0F40037150000832441060329010616
:1026A0001305058013010107678000008357C400EC
:1026B0002320090093F70708638407028320C106DB
:1026C000032481069307000423A0F40003290106D4
:1026D00083244106130500001301010767800000F1
:1026E0008320C106032481069307004023A0F40041
:1026F0000329010683244106130500001301010785
:102700006780000083D7C500130101FE232C8100E0
:10271000232E1100232A91002328210193F727005B
:1027200013840500638807029387350423A0F5000E
:1027300023A8F5009307100023AAF5008320C10108
:1027400003248101832441010329010113010102B2
:10275000678000009306C100130681009304050002
:10276000EFF05FED83258100130905001385040058
:10277000EF00C00C8317C4006308050437170080FE
:102780001307072723AEE402032781008326C10035
:1027900093E707082316F4002320A4002328A400AD
:1027A000232AE40063980604B3E727018320C101CC
:1027B0002316F4000324810183244101032901012C
:1027C000130101026780000013F70720E31807F6E2
:1027D00093F7C7FF93E72700130734042316F40089
:1027E000930710002320E4002328E400232AF400A8
:1027F0006FF0DFF48315E40013850400EF4000015F
:10280000631605008317C4006FF01FFA0357C40056
:102810001377C7FF136717009317070193D7074173
:102820006FF09FF89305050003A5C11C6F00000120
:102830009305050003A5C11C6FF00FAD130101FD49
:10284000232E310123261102232481022322910207
:1028500023202103232C4101232A51012328610134
:102860002326710123248101232291019387B5003E
:1028700013076001930905006364F70693070001DD
:1028800063E2B71EEF0090149304000113062000CA
:1028900093078001138981C2B307F90003A447009D
:1028A000138787FF6308E420832744008326C4003E
:1028B0000326840093F7C7FFB307F40003A747007C
:1028C0002326D60023A4C60013671700138509002A
:1028D00023A2E700EF00D00F130584006F0040191A
:1028E00093F487FF63C0071863EEB416EF00100E71
:1028F0009307701F63FA974493D794006384071A71
:10290000130740006360F73C93D764001386970376
:102910001385870393163600138981C2B306D90045
:1029200003A44600938686FF638686029305F00023
:102930006F000001635207320324C400638C8600D9
:102940008327440093F7C7FF33879740E3D4E5FE1E
:10295000130605000324090193088900630814176E
:10296000032544009306F0001375C5FFB307954097
:1029700063C2F640232A19012328190163DC073CAE
:102980009307F01F63E0A72E937785FF9387870057
:1029900083254900B307F90083A6070013555500A6
:1029A000130710003317A7003367B700938587FF1D
:1029B0002326B4002324D4002322E90023A0870087
:1029C00023A686009357264093051000B395F50083
:1029D0006368B710B3F7E500639407029395150099
:1029E0001376C6FFB3F7E50013064600639A0700A7
:1029F00093951500B3F7E50013064600E38A07FE3A
:102A00001308F000131336003303690013050300A5
:102A10008327C500130E06006308F52C03A74700A3
:102A20001384070083A7C7001377C7FFB306974037
:102A30006348D82CE3C206FE3307E4008326470030
:102A4000032684001385090093E616002322D7008D
:102A50002326F60023A4C700EF0080771305840027
:102A60006F0000019307C00023A0F90013050000C8
:102A70008320C1020324810283244102032901022D
:102A80008329C101032A8101832A4101032B01010A
:102A9000832BC100032C8100832C4100130101030F
:102AA0006780000093060020130600041305F0035E
:102AB0006FF09FE603A4C70013062600E39687DEA7
:102AC0000324090193088900E31C14E90327490042
:102AD0009357264093051000B395F500E37CB7EEBD
:102AE00003248900832A440013FBCAFF63689B0008
:102AF000B3079B401307F000634CF71283AA411EF3
:102B000003A7011D9307F0FF330A6401B38A540140
:102B10006304F734B71700009387F700B38AFA000D
:102B2000B7F7FFFFB3FAFA0093850A00138509008F
:102B3000EF00D01B9307F0FF930B05006306F52809
:102B400063624529138CC12083250C00B385BA002C
:102B50002320BC0093870500630EAA3883A6011DBD
:102B60001307F0FF6386E63A338A4B41B307FA0056
:102B70002320FC0093FC7B0063820C30B71700001D
:102B8000B38B9B4193858700938B8B00B3859541D5
:102B9000B38A5B019387F7FFB385554133FAF5009C
:102BA00093050A0013850900EF0050149307F0FF06
:102BB000630AF53A33057541B30A450183250C00D4
:102BC0002324790193EA1A00B305BA002320BC003C
:102BD00023A25B01630224359306F00063F266359D
:102BE0000327440093074BFF93F787FF13771700E2
:102BF0003367F7002322E400130650003307F40084
:102C00002322C7002324C70063E8F63683AA4B00BB
:102C100013840B0003A7011E6374B70023A0B11E29
:102C200003A7C11D6376B71A23AEB11C6F00401A0B
:102C300013E714002322E400B30494002324990032
:102C400093E717001385090023A2F400EF00405812
:102C5000130584006FF0DFE18326C400032684009F
:102C60006FF09FC593579500130740006372F714E8
:102C700013074001636AF7229386C7059385B7055A
:102C800093963600B306D90083A70600938686FF85
:102C90006388F61C03A747001377C7FF6376E50038
:102CA00083A78700E398F6FE83A6C70003274900A1
:102CB0002326D4002324F40023A4860023A687001F
:102CC0006FF05FD0130740016376F71213074005DA
:102CD000636AF71E93D7C4001386F7061385E706C9
:102CE000931636006FF05FC3130E1E0093773E00FD
:102CF00013058500638E07108327C5006FF0DFD1B1
:102D00000326840093E514002322B4002326F60052
:102D100023A4C700B3049400232A99002328990010
:102D200093E7160023A6140123A4140123A2F400A0
:102D30003307E400138509002320D700EF00404942
:102D4000130584006FF0DFD213D63400938784001C
:102D50006FF05FB43307A400832747001385090091
:102D600093E717002322F700EF0080461305840045
:102D70006FF01FD013E714002322E400B304940083
:102D8000232A99002328990013E7170023A614018A
:102D900023A4140123A2E4003305A4002320F5009A
:102DA00013850900EF00C042130584006FF05FCC6B
:102DB0009357650093869703938587039396360010
:102DC0006FF05FEC630E241103248900832A440012
:102DD00093FACAFFB3879A4063E69A001307F0009C
:102DE000E348F7E413850900EF00803E1305000077
:102DF0006FF01FC81386C7051385B70593163600F5
:102E00006FF09FB1832783001306F6FF6390671C62
:102E100093773600130383FFE39607FE03274900E9
:102E200093C7F5FFB3F7E7002322F9009395150048
:102E3000E3E8B7CAE38605CA33F7F500631A07006B
:102E40009395150033F7F500130E4E00E30A07FEC5
:102E500013060E006FF01FBB938A0A016FF0DFCCE0
:102E60000325490093D52540130710003317B700F9
:102E70003367A7002322E9006FF09FE3B3855B016E
:102E8000B305B0409395450113DA450193050A0057
:102E900013850900EF0080659307F0FFE31CF5D070
:102EA000130A00006FF09FD1130740056360F70815
:102EB0009357C5009386F7069385E70693963600E9
:102EC0006FF05FDC130740156360F70893D7F400D9
:102ED0001386870713857707931636006FF0DFA3F5
:102EE000138CC12083270C00B387FA002320FC0039
:102EF0006FF0DFC613174A01E31207C603248900E7
:102F0000B30A5B0193EA1A00232254016FF09FD0A9
:102F100023A8711D6FF01FC613840B006FF09FCFA5
:102F20009307100023A2FB006FF0DFEB130740159F
:102F30006362F7069357F5009386870793857707B3
:102F4000939636006FF01FD4130740556362F7065F
:102F500093D724011386D7071385C7079316360026
:102F60006FF09F9B938C8CFFB38A9A01B38A7A414E
:102F7000130A00006FF09FC49305840013850900B5
:102F8000EFE09FB80324890083250C00832A4400C6
:102F90006FF05FC8130740556364F702935725012C
:102FA0009386D7079385C707939636006FF09FCD1A
:102FB0009306803F1306F0071305E0076FF0DF95D7
:102FC0009306803F9305E0076FF0DFCB832749002E
:102FD0006FF0DFE5B3C7A50093F73700B308C5006E
:102FE000639207069307300063FEC70493773500AA
:102FF000130705006398070613F6C8FF930706FE3C
:10300000636CF708637CC70293860500930707008B
:1030100003A80600938747009386460023AE07FF68
:10302000E3E8C7FE9307F6FFB387E74093F7C7FFD0
:10303000938747003307F700B385F50063681701EE
:103040006780000013070500E37C15FF83C70500B8
:103050001307170093851500A30FF7FEE36817FF0A
:103060006780000083C605001307170093773700B9
:10307000A30FD7FE93851500E38007F883C60500EC
:103080001307170093773700A30FD7FE938515001A
:10309000E39A07FC6FF05FF683A6450083A2050064
:1030A00083AF850003AFC50083AE050103AE4501C4
:1030B00003A3850103A8C5012322D70083A6050227
:1030C000232057002324F7012326E7012328D701D3
:1030D000232AC701232C6700232E07012320D702B0
:1030E0001307470293854502E368F7FA6FF09FF1F3
:1030F0001303F00013070500637EC3029377F70004
:103100006390070A63920508937606FF1376F6002C
:10311000B386E6002320B7002322B7002324B7009C
:103120002326B70013070701E366D7FE63140600E2
:1031300067800000B306C340939626009702000004
:10314000B38656006780C6002307B700A306B70002
:103150002306B700A305B7002305B700A304B700F3
:103160002304B700A303B7002303B700A302B700EB
:103170002302B700A301B7002301B700A300B700E3
:103180002300B7006780000093F5F50F9396850044
:10319000B3E5D50093960501B3E5D5006FF0DFF6F2
:1031A0009396270097020000B38656009382000092
:1031B000E78006FA93800200938707FF3307F74002
:1031C0003306F600E378C3F66FF0DFF367800000A4
:1031D00067800000130101FF13870500232481008D
:1031E00023229100930506001304050013860600B0
:1031F000130507002326110023AA0122EFD04FBF99
:103200009307F0FF630CF5008320C10003248100C5
:1032100083244100130101016780000083A741233B
:10322000E38407FE8320C1002320F40003248100EF
:10323000832441001301010167800000130101FC98
:103240002324C1022326D1022328E102232AF102EA
:10325000232C0103232E11031386050083258500EB
:1032600093068102232E11002326D100EF00405B3C
:103270008320C101130101046780000003A3C11C66
:10328000130101FC2324C1022326D1022322B1020F
:103290002328E102232AF102232C0103232E110308
:1032A00083258300930641021306050013050300DE
:1032B000232E11002326D100EF0080568320C10168
:1032C00013010104678000008357C50013079000B5
:1032D00093F797006386E7001305000067800000FE
:1032E0006FD09FF6130101FE232C8100232A910049
:1032F000232E1100232821012326310193040500E8
:103300001384050063060500832785036384071281
:103310008317C400139707019396270113570701DA
:1033200063CA060203274406B7260000B3E7D700A6
:10333000B7E6FFFF939707019386F6FF93D7074100
:103340003377D7002322E406139707012316F400EE
:10335000135707012322040093760702639C061487
:1033600093764700639006089376070163840616F8
:10337000137787006310071093E747002316F400C4
:1033800083270401638A07100319C40093190901F4
:103390009377390093D909016392070A0326040140
:1033A00083270402832644018325C4012320C4000B
:1033B00013850400E7800700930705002322A4007B
:1033C00013050000635CF00E8320C101032481011A
:1033D00083244101032901018329C1001301010252
:1033E0006780000083250403E38C05F89307040439
:1033F0006386F50013850400EFE00FF18327C40313
:10340000232804022322F400E38C07F68327840395
:103410008320C101832441012320F400032481017E
:10342000032901018329C1001305000013010102D2
:1034300067800000EFE00F956FF09FED03A5811B03
:10344000B7350080930710002316F4009385852C70
:10345000EFE01FFF93F999002316240193079000D2
:10346000E39EF9F29305040013850400EFD01FB228
:103470006FF0DFF29305040013850400EFD0DFD670
:10348000631A05028317C40023240400232C0400BC
:1034900093F777FF6FF05FEE930504001385040048
:1034A000EFF04FA66FF05FEE1367070423220400CE
:1034B0002316E4001305F0FF6FF01FF10317C4009B
:1034C000E39407FE136707022316E4001305F0FFD9
:1034D0006FF09FEF1307900023A0E40093E7070429
:1034E0002316F4001305F0FF6FF01FEE130101FF28
:1034F0002324810023229100130405001385050075
:103500002326110023AA0122EFD0CF849307F0FFD6
:10351000630CF5008320C100032481008324410053
:10352000130101016780000083A74123E38407FEA4
:103530008320C1002320F400032481008324410060
:103540001301010167800000130101FF23248100A2
:10355000138405008395E50023261100EF70001504
:1035600063400502832704058320C100B387A700B9
:103570002328F40403248100130101016780000063
:103580008357C40037F7FFFF1307F7FFB3F7E700D0
:103590008320C1002316F4000324810013010101DC
:1035A0006780000013050000678000008397C50056
:1035B000130101FE232C8100232A910023282101DD
:1035C00023263101232E110013F707101384050061
:1035D000930405008395E50013090600938906000E
:1035E000631E070237F7FFFF1307F7FFB3F7E70084
:1035F0002316F400032481018320C101938609006E
:10360000130609008329C100032901011385040061
:1036100083244101130101026F20105793062000FB
:1036200013060000EF5090668317C4008315E40072
:103630006FF05FFB130101FF232481001384050059
:103640008395E50023261100EF5050649307F0FFA7
:103650006304F5028357C400371700008320C100BC
:10366000B3E7E7002328A4042316F4000324810011
:1036700013010101678000008357C40037F7FFFF83
:103680001307F7FFB3F7E7008320C1002316F40008
:103690000324810013010101678000008395E50088
:1036A0006F3040063367B5009303F0FF13773700A0
:1036B00063100710B7877F7F9387F7F7032605000E
:1036C00083A60500B372F6003363F600B382F200FE
:1036D000B3E26200639272106316D60803264500B7
:1036E00083A64500B372F6003363F600B382F2009E
:1036F000B3E26200639E720C6316D6060326850051
:1037000083A68500B372F6003363F600B382F2003D
:10371000B3E262006398720C6316D6040326C500F8
:1037200083A6C500B372F6003363F600B382F200DD
:10373000B3E262006392720C6316D602032605019F
:1037400083A60501B372F6003363F600B382F2007C
:10375000B3E26200639C720A13054501938545013B
:10376000E30ED6F41317060193970601631EF700C4
:103770001357060193D706013305F7409375F50FEC
:1037800063900502678000001357070193D7070174
:103790003305F7409375F50F6394050067800000CB
:1037A0001377F70F93F7F70F3305F74067800000A3
:1037B0000346050083C60500130515009385150013
:1037C0006314D600E31606FE3305D640678000007A
:1037D0001305450093854500E31CD6FC1305000046
:1037E000678000001305850093858500E312D6FCF1
:1037F00013050000678000001305C5009385C50010
:10380000E318D6FA130500006780000013050501D0
:1038100093850501E31ED6F81305000067800000BC
:10382000130101E12326111E2320211F2324811DC2
:103830002320A11D138C050013090600232AD100A3
:103840002324811E2322911E232E311D232C411D52
:10385000232A511D2328611D2326711D2322911D1A
:10386000232EB11B130D0500EF50D0378327050021
:10387000138507002328F102EF70800D2326A10293
:103880002328010E232A010E232C010E232E010EC4
:1038900063060D0003278D03E308070A8316CC0097
:1038A00013970601939726011357070163CA07026E
:1038B0003727000003264C0633E7E60013170701FD
:1038C000B7E6FFFF135707419386F6FFB376D6009E
:1038D0002316EC00131707012322DC0613570701F8
:1038E000937687006388062E83260C016384062E58
:1038F0001377A7019306A0006300D7309307C11088
:10390000375701802322F10E938807009307C732AF
:1039100037570180232CF100130B09009307874AC6
:103920002324F10083470B002326010E2324010EDC
:1039300023200102232A0102232C0102232E01024B
:103940002324010423260104232601006386072281
:1039500013040B0093065002638AD7308347140088
:1039600013041400E39A07FEB30464416306642160
:103970008326C10E8327810E23A06801B38696009B
:103980009387170023A298002326D10E2324F10E3B
:10399000930670009388880063C2F62E0327C10047
:1039A00083470400330797002326E1006386071C42
:1039B00083441400A303010C13041400930DF0FFBF
:1039C00093090000130A00001309A005930A900050
:1039D000930BA002938C080013041400938704FE39
:1039E0006364F9040327810193972700B387E700F5
:1039F00083A707006780070093090000938604FDF2
:103A00008344040093972900B387370193971700E5
:103A1000B389F600938604FD13041400E3F2DAFE82
:103A2000938704FEE370F9FC93880C00638604140A
:103A300023069114A303010C930A1000930C1000A9
:103A4000130BC11423280100930D0000232401024D
:103A500023220102232E0100937B2A0063840B00A2
:103A6000938A2A0013794A088327C10E6316090036
:103A700033885941E34600718346710C638A06021C
:103A80008326810E1306710C23A0C80093871700AC
:103A9000130610009386160023A2C8002326F10EF9
:103AA0002324D10E13067000938888006342D652F7
:103AB000638C0B028326810E1306810C23A0C800A1
:103AC00093872700130620009386160023A2C800C0
:103AD0002326F10E2324D10E13067000938888004C
:103AE0006354D6006F00D07893060008E30ED93CEB
:103AF000B38D9D41E34AB04993760A10E3980628B6
:103B00000327810EB387970123A0680113071700CD
:103B100023A298012326F10E2324E10E93067000C0
:103B200063C8E65493888800137A4A0063060A0043
:103B3000B3845941634E905463D4590193890A0068
:103B40000327C100330737012326E100E398074E1E
:103B5000832701012324010E6388070083250101C7
:103B600013050D00EFD05FFA9308C110130B04008A
:103B700083470B00E39E07DC8327C10E63840700A5
:103B80006F1050328357CC0093F70704638407000B
:103B90006F2000238320C11E0324811E0325C10042
:103BA0008324411E0329011E8329C11D032A811D6F
:103BB000832A411D032B011D832BC11C032C811C57
:103BC000832C411C032D011C832DC11B1301011FDC
:103BD0006780000093050C0013050D00EF205001D5
:103BE000630405006F20C01D0357CC009306A0009E
:103BF0001377A701E314D7D00317EC00E34007D0F5
:103C0000832641011306090093050C0013050D00DE
:103C1000EF20806B2326A1006FF0DFF713050D0066
:103C2000EF50407C83274500138507002326F104CD
:103C3000EF6010529307050013050D0093840700F1
:103C40002324F104EF50007A83278500232EF1020C
:103C5000638404006F10C012834404006FF0DFD748
:103C600083440400136A0A026FF01FD7B30464414F
:103C7000E31064D1834704006FF05FD31306410E55
:103C800093050C0013050D00EF901010E31C05EEDA
:103C90009308C1106FF09FD093778A0093880C002F
:103CA000638407006F10C012832741011305010BC5
:103CB000232891019387770093F787FF83A5070057
:103CC00003A6470093878700232AF100EF00D16BFA
:103CD0008327010B832801012328F10E8327410B41
:103CE000232AF10E8327810B232CF10E8327C10B8E
:103CF000232EF10E1305010F23281101EF50C06789
:103D00002326A10C93072000832801016314F500EA
:103D10006F10C04F930710006314F5006F104064DC
:103D2000930710066394F4006F20401C930710045F
:103D30006394F4006F10101993FBF4FD9307F0FFE8
:103D4000232271056394FD006F20002893077004FF
:103D50006394FB006F20001E0323C10F2324410343
:103D6000032E010F832E410F032F810F93670A103B
:103D7000635403006F20003E232C0104138A0700C4
:103D800023280100930760046394FB006F1090697F
:103D900093075004232811056384FB006F10906083
:103DA00013891D00930A010B930609001308C10D26
:103DB0009307010D1307C10C1306200093850A0019
:103DC00013050D002328C10B2320C105232AD10B85
:103DD0002322D103232CE10B2320E103232E610AAC
:103DE000232E6100EF40C02F0323C101032F0102E6
:103DF000832E4102032E010483280105130B0500C5
:103E000033092501930C010A93850C0013850A00E0
:103E1000232E11012328C10B232AD10B232CE10BC4
:103E2000232E610A2320010A2322010A2324010AE6
:103E30002326010AEFE080278328C1011307090028
:103E4000630205020327C10D637E27019306000369
:103E500093071700232EF10C2300D7000327C10D71
:103E6000E36827FFB30767412320F1020327C10C52
:103E700093077004232EE100032741046314F70025
:103E80006F10D04303274104930760046314F700C5
:103E90006F10D0678327C1010327410493051004E5
:103EA0009387F7FF2326F10C93F6F40F1306000017
:103EB0006318B7009386F60093F6F60F130610000A
:103EC000230AD10C9306B00263DA07000327C1016D
:103ED000930710009306D002B387E740A30AD10CE2
:103EE0009306900063C4F6006F20C0281308310EBB
:103EF000130508001306A000130E300633E7C702AF
:103F000093050500938607001305F5FF13070703C4
:103F1000A38FE5FEB3C7C702E342DEFE9387070324
:103F200013F6F70FA30FC5FE9387E5FF63E40701C0
:103F30006F2040379306610D6F00800003C60700B5
:103F40002380C6009387170093861600E39807FF27
:103F50009307510EB387B7401307610DB307F700FE
:103F60009306410DB387D740232CF10203270102AA
:103F70008326810393071000B30CD70063C4E700C6
:103F80006F2040298327C102B38CFC008327810264
:103F900093CAFCFF93DAFA4113FAF7BF136A0A10C7
:103FA000B3FA5C012324010223220102232E010023
:103FB00083278105639407006F1090379307D00221
:103FC000A303F10C930D0000938A1A006FF0DFA891
:103FD0001306410E93050C0013050D00EF90C05A17
:103FE000E31805068327C10E9308C1106FF05FAC7C
:103FF000832601030327C1021306700023A0D80003
:104000008326810EB307F70023A2E80093861600EB
:104010002326F10E2324D10E938888006354D60200
:104020001306410E93050C0013050D00EF90C055CB
:10403000E31005028325C10C8327C10E8326810E60
:104040009308C11063D405006F1050580327010274
:104050009386160023A06801B307F70023A2E800A7
:104060002326F10E2324D10E13077000E35CD7AA98
:104070001306410E93050C0013050D00EF90C05080
:104080006318057C8327C10E9308C1106FF0DFA968
:10409000930600010327810E63C496006F109051B0
:1040A000B7560180938E864913090001130A7000E8
:1040B000138B0E006F00C000938404FF63569904B5
:1040C000938707011307170023A0680123A2280183
:1040D0002326F10E2324E10E93888800E35EEAFC98
:1040E0001306410E93050C0013050D00EF90C04917
:1040F00063100576938404FF8327C10E0327810E86
:104100009308C110E34E99FA930E0B00B387970002
:104110001307170023A0D80123A298002326F10E2D
:104120002324E10E93067000E3D8E6A01306410EA7
:1041300093050C0013050D00EF900045631A057000
:104140008327C10E6FF05F9F13050D00EFD08FC363
:104150006FF0CFF40327410193880C00A303010CF7
:104160008327070013074700232AE1002306F114E1
:10417000930A1000930C1000130BC1146FF09F8C66
:1041800083274101A303010C93880C0003AB0700B4
:1041900013894700E30E0B5A9307F0FF6394FD0069
:1041A0006F10001013860D009305000013050B001F
:1041B000232A9101EF50003B2328A10083284101CD
:1041C000631405006F10D03183270101232A2101D8
:1041D00023280100B38C67418347710C93CAFCFF0D
:1041E00093DAFA412324010223220102232E010043
:1041F000B3FA5C01930D0000E3800786938A1A00EE
:104200006FF09F8583440400136A4A006FF0CFFC6F
:104210008326410193770A0293880C0003A70600C6
:1042200093864600232AD100E39E073693770A013E
:10423000638407006F10C00593770A046384070046
:104240006F10C03F137A0A2063140A006F104004F5
:104250008327C100130B04002300F7006FF05F9168
:10426000834404009307C006E384F44C136A0A01F4
:104270006FF08FF603274101B787FFFF93C70783CE
:104280002314F10C93074700232AF10003290700A8
:10429000B75701809387872F93880C00232AF10258
:1042A000930C0000936B2A0093072000930480076F
:1042B000A303010C1307F0FF6386ED203367990118
:1042C00013FAFBF7631E071E63940D266390071C09
:1042D00093FC1B00130B011BE39C0C28938A0C001E
:1042E00063D4BC01938A0D008347710C232801001D
:1042F0002324010223220102232E0100E39007F070
:104300006FF08FF58344040093078006E38AF4423C
:10431000136A0A046FF04FEC9307B0028344040061
:10432000A303F10C6FF04FEB83440400136A0A08F7
:104330006FF08FEA83440400130714006394740140
:104340006F105072938604FD13040700930D000054
:1043500063E6DAE88344040093972D00B387B7013E
:1043600093971700B38DD700938604FD13041400B0
:10437000E3F2DAFE6FF08FE6832741018344040005
:1043800083A9070093874700232AF10063D609E435
:10439000B3093041136A4A006FF00FE4834404000C
:1043A000136A1A006FF04FE38347710C83440400D3
:1043B000639407E293070002A303F10C6FF0CFE1CF
:1043C00093880C00136A0A0193770A02E38E070CA4
:1043D00083274101138B7700137B8BFF03290B008D
:1043E000832C4B0093078B00232AF100937BFABFA9
:1043F000930700006FF0DFEB93880C00936B0A01CA
:1044000093F70B02E388070C83274101138B770096
:10441000137B8BFF93078B00232AF10003290B00EA
:10442000832C4B00930710006FF09FE88344040037
:10443000136A8A006FF04FDA93880C00136A0A013E
:1044400093770A02E380070C83274101138B7700DF
:10445000137B8BFF83274B0003290B0013078B0073
:10446000232AE100938C0700E3C6070C9307F0FFB3
:10447000930B0A006384FD02B3679901937BFAF7FB
:10448000639E070063920D02138A0B00930D0000D8
:10449000930C0000130B011B6FF05FE4E3920C3AE6
:1044A00093079000E3EE273913090903A307211BA3
:1044B000138A0B00930C1000130BF11A6FF01FE21C
:1044C000930B0A0013071000E38AE7FC1307200090
:1044D000638CE706130B011B1397DC0193777900BC
:1044E00013593900938707033369270193DC3C0094
:1044F000A30FFBFE3367990113060B00130BFBFFA1
:10450000E31C07FC93F61B00638A06069306000370
:104510006386D7061306E6FF9307011BA30FDBFE96
:10452000B38CC740138A0B00130B06006FF01FDB20
:10453000130710006394E7006F10D01413072000D6
:10454000930B0A00E398E7F883264103130B011B42
:104550009377F900B387F60003C7070013594900A2
:104560009397CC0133E9270193DC4C00A30FEBFEBA
:10457000B3679901130BFBFFE39C07FC9307011B37
:10458000B38C6741138A0B006FF05FD5930650061A
:1045900063DC962C8326010F9305010A1305010B9A
:1045A0002328D10A8326410F232211052320F10459
:1045B000232AD10A8326810F2320010A2322010AFC
:1045C000232CD10A8326C10F2324010A2326010AA2
:1045D000232ED10AEFD0902D832701048328410494
:1045E0006318054A0327810EB756018093868632E9
:1045F00023A0D80093871700930610001307170015
:1046000023A2D8002326F10E2324E10E9306700086
:1046100093888800E3C6E63A0327C10C832601028B
:10462000635CD772032701038326C1029388880045
:1046300023ACE8FE0327810EB387D70023AED8FE54
:10464000130717002326F10E2324E10E93067000B2
:10465000E3C0E60C032701029304F7FF635690CCF6
:10466000930600010327810EE3DC9636130900014F
:10467000930C70006F00C000938404FFE3529936DE
:1046800083268100938707011307170023A0D80012
:1046900023A228012326F10E2324E10E938888000B
:1046A000E3DCECFC1306410E93050C0013050D0032
:1046B000EF80906D631E05188327C10E0327810EBE
:1046C0009308C1106FF05FFB33895941635220C3D7
:1046D000130600018326810E63542607130E000182
:1046E000930B70006F00C000130909FF635A2E0579
:1046F00003278100938707019386160023A0E80013
:1047000023A2C8012326F10E2324D10E938888000A
:10471000E3DCDBFC1306410E93050C0013050D00D2
:10472000EF80906663160512130E0001130909FF4E
:104730008327C10E8326810E9308C110E34A2EFB06
:1047400003278100B38727019386160023A0E80082
:1047500023A228012326F10E2324D10E1306700074
:10476000938888006356D6B81306410E93050C0053
:1047700013050D00EF805061631C050C8327C10EEB
:104780009308C1106FF0CFB6130600018326810E87
:104790006352B607930B0001130970006F00C0004D
:1047A000938D0DFF63D8BB05032781009387070115
:1047B0009386160023A0E80023A278012326F10E99
:1047C0002324D10E93888800E35CD9FC1306410EA4
:1047D00093050C0013050D00EF80105B631A0506AE
:1047E000938D0DFF8327C10E8326810E9308C11080
:1047F000E3CCBBFB03278100B387B7019386160088
:1048000023A0E80023A2B8012326F10E2324D10E11
:1048100013067000938888006350D6AE1306410ECD
:1048200093050C0013050D00EF801056631205026E
:104830008327C10E9308C1106FF00FAC1306410E11
:1048400093050C0013050D00EF801054630205B0B2
:10485000832B010163880BB293850B0013050D00B8
:10486000EFD08FAA6FF00FB28326810E938C1700C2
:10487000832701021306100023A068019384160009
:10488000138988006356F6389307100023A2F800B6
:104890002326910F2324910E9307700063CE977403
:1048A0008327C1020327010393841400B38CFC0007
:1048B0002322F9002320E9002326910F2324910EBF
:1048C000930770001309890063CA97748327010F47
:1048D000138614009305010A2328F10A8327410F48
:1048E0001305010B232EC100232AF10A8327810F10
:1048F0002320010A2322010A232CF10A8327C10F56
:104900002324010A2326010A232EF10AEFD0007A7C
:104910000326C1018327010293088900930606003C
:10492000938DF7FF630A053013071B00B38CBC019E
:104930002320E9002322B9012326910F2324C10E4D
:104940009307700063CCC750930709019386240036
:104950001389080093880700032681031307410D7C
:104960002320E900B30796012322C9002326F10E74
:104970002324D10E130770006358D79A6FF04FEFBE
:1049800037570180130600018326810E930E874955
:10499000635C0609232081042322910413040D0083
:1049A00093040C00130E000193027000130C080016
:1049B000138D0E006F00C000130C0CFF635A8E05A0
:1049C000938707019386160023A0A80123A2C8019C
:1049D0002326F10E2324D10E93888800E3DED2FC37
:1049E0001306410E9385040013050400EF80D039AF
:1049F0006312057A130E0001130C0CFF8327C10EFE
:104A00008326810E9308C11093027000E34A8EFB47
:104A100013080C00930E0D00138C0400130D0400FA
:104A20008324410403240104B387070193861600FD
:104A300023A0D80123A208012326F10E2324D10E9E
:104A400013067000938888006344D6006FF0CF820D
:104A50001306410E93050C0013050D00EF80D032B4
:104A6000E31805DE8327C10E9308C1106FF0CF80D5
:104A70001306410E93050C0013050D00EF80D03096
:104A8000E31805DC8327C10E9308C1106FF0CF85B2
:104A90008325C10C635CB0660327C1018326010234
:104AA0009304070063C2E638635690028326810EA2
:104AB000B387970023A068019386160023A298006D
:104AC0002326F10E2324D10E13067000938888004C
:104AD000E342D63293C6F4FF0327C10193D6F641D1
:104AE000B3F4D400B3049740634490480327C10152
:104AF00093760A40B30DEB00E398060C8324C10CB7
:104B00000327010263C6E40093761A00E3880630A7
:104B1000832601030327C1021306700023A0D800D7
:104B20008326810EB387E70023A2E8009386160050
:104B30002326F10E2324D10E938888006354D600D7
:104B40006F108017832601023307DB00B384964081
:104B50003307B74113890400635497001309070012
:104B6000635820030327810EB387270123A0B801D0
:104B70001307170023A228012326F10E2324E10E98
:104B8000930670009388880063D4E6006F10801C41
:104B90001347F9FF1357F7413377E900B384E44033
:104BA000634490006FE05FF8930600010327810ED5
:104BB00063D8966213090001930C70006F00C00067
:104BC000938404FF635E99608326810093870701C5
:104BD0001307170023A0D80023A228012326F10ED3
:104BE0002324E10E93888800E3DCECFC1306410EDD
:104BF00093050C0013050D00EF801019E31A05C48E
:104C00008327C10E0327810E9308C1106FF05FFB4D
:104C100093771A00E39A07C623A2C8002326910FB0
:104C20002324910E9307700063CA9722938626006F
:104C3000938808016FF05FD2E350B0D313070001EF
:104C40006344B7016F108061130B7000930406007A
:104C50006F000001938D0DFF635EB71D93841400F8
:104C600083278100938C0C012322E9002320F90083
:104C70002326910F2324910E13098900E35C9BFCEA
:104C80001306410E93050C0013050D00EF80D00FA5
:104C9000E31005BC832CC10E8324810E1309C110BF
:104CA000130700016FF01FFB8326410193770A0170
:104CB000138746006392071693770A046384076894
:104CC00083274101930C0000232AE10003D9070048
:104CD0006FF0CFF18326410193F70B011387460054
:104CE000639E070C93F70B04638E076083274101D3
:104CF000930C0000232AE10003D90700930710005A
:104D00006FF00FDB8326410193770A01138746007A
:104D1000639A070E93770A0463860760832741012D
:104D2000232AE10003990700935CF94193870C0063
:104D300063DE07F2B3372001B30C9041B38CFC4023
:104D40009307D002A303F10C33092041930B0A000F
:104D5000930710006FF00FD613771A006314070043
:104D60006FE09FDC6FF01F8C93880C006FF04FEDAD
:104D700093070003A307F11A130BF11A6FF00FD674
:104D80008327C10383440400639407006FE0DFC4FA
:104D900083C70700639407006FE01FC4136A0A40CB
:104DA0006FE09FC38326C100130B040093D7F64125
:104DB0002320D7002322F7006FE09FDB03A9060022
:104DC000930C0000232AE100930710006FF04FCEF0
:104DD000032741018327070013074700232AE10027
:104DE00083A5070003A6470083A6870083A7C70003
:104DF0002328B10E232AC10E232CD10E232EF10E0F
:104E00006FE05FEF03A90600232AE100935CF941FC
:104E100093870C006FF04FE503A90600930C000088
:104E2000232AE1006FF08FDC93840600E34090C8F2
:104E30006FF05FCA938614001307890083278100EF
:104E4000B38CBC012322B9012320F9002326910F42
:104E50002324D10E9307700063DED7741306410E2E
:104E600093050C0013050D00EF800072E312059E00
:104E70008326810E832CC10E930841119386160060
:104E80001309C1106FF05FAD93880C00930B0A00FB
:104E90006FF00FD7B75701809387872F93880C0047
:104EA000232AF10293770A026388071283274101BC
:104EB000138B7700137B8BFF03290B00832C4B0094
:104EC00093078B00232AF10093771A00638E070063
:104ED000B3679901638A0700930700032304F10C69
:104EE000A304910C136A2A00937BFABF9307200056
:104EF0006FF00FBCB75701809387C73093880C00C1
:104F0000232AF1026FF01FFA93880C006FF0CFCBC9
:104F10001306410E93050C0013050D00EF80C066CB
:104F2000E31805928327C10E9308C1106FF08FF22A
:104F300083441400136A0A02130414006FE0DFA90B
:104F400083441400136A0A20130414006FE0DFA8DE
:104F500093076000938C0D0063EEB76B37570180A9
:104F6000938A0C00232A2101130B07326FE09FADB7
:104F7000130600018326810E63549640930C0001B2
:104F8000930D70006F00C000938404FF63DA9C3EB1
:104F900003278100938707019386160023A0E8006A
:104FA00023A298012326F10E2324D10E9388880092
:104FB000E3DCDDFC1306410E93050C0013050D0028
:104FC000EF80805CE31605888327C10E8326810E5F
:104FD0009308C1106FF05FFB8326410193770A01AC
:104FE000138746006380071C03A90600930C00008A
:104FF000232AE1006FF05FED1306410E93050C00CC
:1050000013050D00EF804058E3140584832CC10E76
:105010008324810E1309C1106FF09F881306410E7F
:1050200093050C0013050D00EF800056E312058276
:10503000832CC10E8324810E1309C1106FF01F89C8
:10504000130B011B9307000023288100232E9100DE
:1050500013040B0023223103130B0C0093040900EB
:1050600093890C0013FA0B40832CC103930AF00FB1
:10507000138C0800138907006F0040021306A0007C
:10508000930600001385040093850900EFB0903368
:10509000E38A092A93040500938905001306A000FA
:1050A000930600001385040093850900EFB0D074C7
:1050B00013050503A30FA4FE130919001304F4FF3D
:1050C000E30E0AFA83C60C00E31AD9FAE30859FB87
:1050D0006392094A9307900063EE974893080C0087
:1050E0009307011B130C0B00130B0400232E9103D9
:1050F0008324C101832941020324010123202103C8
:10510000B38C6741138A0B006FF04F9D8326810E8D
:10511000375601801306863223A0C80093871700F4
:10512000130610009386160023A2C8002326F10E52
:105130002324D10E13067000938888006344D64858
:10514000638405006FE0DFEA0327010293761A000B
:10515000B3E6E600639406006FE01F9D832601031B
:105160000327C1021306700023A0D8008326810EF6
:10517000B307F70023A2E800938616002326F10E5A
:105180002324D10E6354D6006FE09FE993888800F2
:105190006FE0DFEB832B0101130D0400138C04007F
:1051A0006FF04FEB93770A04638007148327410164
:1051B000930C0000232AE10003D907006FF0DFD031
:1051C0001306410E93050C0013050D00EF80C03B44
:1051D000631005E88327C10E9308C1106FF0CFC399
:1051E00083268100B387970023A2980023A0D800CC
:1051F000130717002326F10E2324E10E93067000F7
:1052000063C4E6006FE01F926FE09FE68327010F03
:105210009305010A1305010B2328F10A8327410F87
:105220002320010A2322010A232AF10A8327810F5E
:105230002324010A2326010A232CF10A8327C10F04
:10524000232EF10AEFD0800783280101E3400526D1
:105250008347710C130770046358973837570180E0
:10526000130BC72E2328010023240102232201024D
:10527000232E0100137AFAF7930A3000930C3000C2
:10528000930D0000638407006FE05FF76FE0CFFCD1
:105290008327C100130B04002320F7006FE05F8D0C
:1052A00013050B0023209105EF50806A8347710C92
:1052B000934AF5FF93DAFA41232A210123280100BA
:1052C0002324010223220102232E0100832801044A
:1052D000930C0500B37A5501930D00006384070019
:1052E0006FE0DFF16FE04FF793770A206382073AB0
:1052F00083274101930C0000232AE10003C9070022
:105300006FF09FBC93F70B2063880736832741011A
:10531000930C0000232AE10003C907009307100043
:105320006FE01FF993770A20638C073283274101CE
:10533000232AE10003890700935CF94193870C005D
:105340006FF08F9293770A206382073083274101A1
:10535000930C0000232AE10003C907006FF00F89B6
:105360008327C10F63CA07348347710C1307700486
:10537000E35C971C37570180130B472F6FF09FEEAC
:1053800003278100B38797009386160023A0E800C7
:1053900023A298002326F10E2324D10E13067000B9
:1053A000938888006354D6F41306410E93050C00CD
:1053B00013050D00EF80401D631C05C88327C10E37
:1053C0009308C1106FF08FF203270102832C410272
:1053D000232E41012320810423223105232251035E
:1053E0008329810223246103B30BEB000324C1034F
:1053F000032A8104832AC104930470001309000165
:10540000130B0C0063880C08639809081304F4FF5D
:10541000938CFCFF0327810EB387470123A058011B
:105420001307170023A248012326F10E2324E10EBF
:105430009388880063CEE40E834604003386BB4124
:10544000138C06006354D600130C060063568003C9
:105450008326810EB387870123A0B80193861600A7
:1054600023A288012326F10E2324D10E63C2D40E79
:1054700083460400938888001346FCFF1356F641C8
:105480003377CC00338CE640634C8001B38DDD0074
:10549000E39C0CF6638A095E9389F9FF6FF09FF72E
:1054A0008326810E634889016F008005130C0CFF71
:1054B00063588905032781009387070193861600A7
:1054C00023A0E80023A228012326F10E2324D10ED5
:1054D00093888800E3DCD4FC1306410E93050B008F
:1054E00013050D00EF80400A63140566130C0CFFD2
:1054F0008327C10E8326810E9308C110E34C89FBDC
:1055000003278100B38787019386160023A0E80054
:1055100023A288012326F10E2324D10E63C0D46672
:105520008346040093888800B38DDD006FF05FF63A
:105530001306410E93050B0013050D00EF80C00408
:10554000631805608327C10E9308C1106FF0DFEE6A
:105550001306410E93050B0013050D00EF80C002EA
:105560006318055E834604008327C10E9308C110AB
:105570006FF09FF0832781048325C1041309000085
:105580003304F4401386070013050400EF50004570
:1055900083C51C001306A000930600003338B0003A
:1055A0001385040093850900B38C0C01EFB0806172
:1055B0006FF05FAE9386160093088700130907000B
:1055C0006FF08FB91306410E93050C0013050D0003
:1055D000EF70907B631E05A68325C10C8327C10E47
:1055E0009308C1106FF0DFB537570180130B872E7A
:1055F0006FF05FC71306410E93050C0013050D00F5
:10560000EF709078631605A48327C10E9308C1102C
:105610006FF04FCC930C60006FF05F948326010213
:105620003307DB00B38496403308B7411389040085
:10563000635098D6130908006FF08FD58327C100F7
:10564000130B04002310F7006FE08FD28327410172
:10565000930C0000232AE10003A907006FE01FD983
:1056600083274101232AE10003A90700935CF94144
:1056700093870C006FE05FDF83274101930C0000EC
:10568000232AE10003A90700930710006FE05FC21F
:1056900083274101930C0000232AE10003A907009E
:1056A0006FF09F821306410E93050C0013050D0049
:1056B000EF70906D6FE00FCD9307D002A303F10C54
:1056C0006FF0DFCA930700032304F10C93078005F2
:1056D00013672A00A304F10C2324E1029307300688
:1056E00023280100130BC114E3C4B7030323C10F24
:1056F00093FBF4FD23227105232C0104032E010FDB
:10570000832E410F032F810F136A2A10634E034427
:1057100093071006E38EF40A930710046384F400E1
:105720006FE04FE6930A010B13850A00232A110547
:105730002328C10B232AD10B232CE10B232E610A32
:10574000EFF0C0631306C10CEF40D07C1386050058
:105750009305050013850A00EFF000438327010B32
:10576000930C010A130901092328F1088327410B2F
:105770001306010893050900232AF1088327810BEA
:1057800013850C002320C104232CF1088327C10BAF
:105790002320010823220108232EF108B707FC3F2C
:1057A0002326F10823240108EFC090450328010AAD
:1057B000032E410A832E810A032FC10A93850C0010
:1057C00013850A002328010B23280105232AC10B76
:1057D0002322C103232CD10B2320D103232EE10B41
:1057E000232EE1012320010A2322010A2324010A96
:1057F0002326010AEFC0900B032FC101832E010263
:10580000032E410203280105832841056316050084
:10581000930710002326F10CB75701809387C730F8
:105820002322F1029386FDFF232E410523229106B8
:105830002326B107232AA107232C810723208106D1
:105840002324310723281107130C0B00938B060028
:10585000232E6107130D0800930D0E0093840E0094
:10586000130A0F006F00800493850C0013850A0053
:105870002320C102232EF101232CF10B232EC10A78
:105880002328610B232A310B2320010A2322010A3A
:105890002324010A2326010AEFC05001832FC101EE
:1058A00003260102938BFBFF6302050EB70703403B
:1058B0001306090093850C0013850A00232EF108B6
:1058C0002320A10B2322B10B2324910A2326410B71
:1058D00023280108232A0108232C0108EFC0503295
:1058E00013850A00EFF0000493050500130405007A
:1058F00013850A008329010B8324410B032B810BA1
:10590000032AC10BEFF040130327010B0326010408
:10591000930509002320E1080327410B13850C00A0
:10592000232831092322E1080327810B232A910828
:10593000232C61092324E1080327C10B232E4109ED
:105940002326E108EFD0102C83274102032B010A04
:105950008329410A3387870003470700832F810A81
:105960000326C10A232A81052300EC0023287105A0
:105970009307F0FF130C1C00130D0B00938D09000F
:1059800093840F00130A0600E390FBEE83280107BF
:1059900093030B00938209003709FE3F93850C00A7
:1059A00013850A0023201103232E8100032AC10539
:1059B00083244106032401062328710A2322710649
:1059C000232A510A23205106232CF10B232EF10503
:1059D000232EC10A2320C1042320010A2322010A05
:1059E0002324010A2326210BEFC00079930B0C001E
:1059F000832DC106032D4107032C8107032BC1070B
:105A000083298106832801026342A048832341063B
:105A100083220106832FC1050326010493850C0010
:105A200013850A002328710A232A510A232CF10B1B
:105A3000232EC10A2320010A2322010A2324010A5A
:105A40002326210BEFC0806683280102631805001E
:105A50008327C10193FC1700639A0C428327010539
:105A60001306000393861700B386DB0063C80700A4
:105A7000938B1B00A38FCBFEE39C76FFB3876B4118
:105A80002320F1026FE08FBE03270102130C0B00ED
:105A9000032B8102232E8102032AC101B306EB00EE
:105AA0000324010483294104832A410263E4B601EB
:105AB0006FF0CF84938D06006FF04F840327C101F0
:105AC0009307D0FF6344F70063DAED009384E4FFAB
:105AD00093F7F4FD2322F1046FE0CFBB832701028B
:105AE0000327C1016340F72A83278102930C070033
:105AF00093F71700638607008327C102B30CF700F2
:105B00008327810293F70740638607008327C1013B
:105B10006342F05C93CAFCFF93DAFA41B3FA5C018A
:105B20009304700623240102232201026FE04FC870
:105B30008347710C930D0000638407006FE00FEC46
:105B40006FD09FF19307900063E697D46FF00FD961
:105B5000832B0101130C0B006FE0DFCF23244103E3
:105B600023280100130A0900B707008033C3670028
:105B70009307D002232CF1046FF09FB91306410E56
:105B800093050B0013050D00EF701020E31205FCC8
:105B9000834604008327C10E9308C110B38DDD0036
:105BA0006FF01F8F930A010B9307010D1308C10DAE
:105BB0001307C10C93860D001306200093850A007D
:105BC00013050D002328C10B2320C105232AD10B67
:105BD0002322D103232CE10B2320E103232E610A8E
:105BE000232E6100EF20C04F930770040323C101EF
:105BF000032F0102832E4102032E01048328010595
:105C0000130B05006390FB088327810293F71700AD
:105C10006396072E930770040327C10D2322F10416
:105C20006FE04FA4930A010B1308C10D9307010DF8
:105C30001307C10C93860D001306300093850A00EC
:105C400013050D00232811052328C10B2320C105AE
:105C5000232AD10B2322D103232CE10B2320E103A0
:105C6000232E610A232E6100EF2080470323C10108
:105C7000032F0102832E4102032E01048328010514
:105C8000130B0500930760043309BB01639EFB26D9
:105C900083460B00930700036386F650930C010ABA
:105CA0008327C10C3309F9006FE00F969307D002E8
:105CB000A303F10C6FF00FDA1306410E93050C00ED
:105CC00013050D00EF70500C630405006FE05FB822
:105CD0008324C10C8327C10E9308C1106FE09FE697
:105CE0008347710C232A210123240102232201026C
:105CF000232E0100938A0D00938C0D00930D00005C
:105D0000638407006FE08FCF6FD01FD58327810298
:105D10000327C10193F71700B3E7B7016356E050BB
:105D200063900744832CC10193046006832781029A
:105D300093F707406392073A93CAFCFF93DAFA415C
:105D4000B3FA5C016FF01FDE37570180130B072F8A
:105D50006FF04FD11306410E93050C0013050D0093
:105D6000EF709002630405006FE09FAE8324C10CC6
:105D7000032701028327C10E9308C110B304974083
:105D80006FE01FE1832701020327C102930470061D
:105D9000B38CE7008327C101E34AF0F8B38CFC40E1
:105DA000938C1C0093CAFCFF93DAFA41B3FA5C01AE
:105DB0006FF05FD7B7560180938E86496FE00FB5BD
:105DC0009307F0FF2326F1006FD0DFDC130600FFFE
:105DD000B304B04063D2C50613090001930C7000F0
:105DE0006F00C000938404FF635899040327810067
:105DF000938707019386160023A0E80023A22801B9
:105E00002326F10E2324D10E93888800E3DCDCFCEA
:105E10001306410E93050C0013050D00EF70C076BC
:105E2000630405006FE0DFA28327C10E8326810E85
:105E30009308C1106FF01FFB03278100B387970001
:105E40009386160023A0E80023A298002326F10ED3
:105E50002324D10E13067000635AD6B21306410EE6
:105E600093050C0013050D00EF700072630405002C
:105E70006FE01F9E8327C10E8326810E9308C110F9
:105E80006FE0CF9C930B0A006FE00FE28327410580
:105E900093860B00232EF10C8327410203C6FBFFE0
:105EA00083C5F7006310B60213050003A38FA6FE97
:105EB0008326C10D9387F6FF232EF10C03C6F6FF50
:105EC000E386C5FE930516001305900393F5F50FC1
:105ED0006306A600A38FB6FE6FF05FBA8327410268
:105EE00083C5A700A38FB6FE6FF05FB993070003C9
:105EF0002304F10C930780076FF08FFD9307700464
:105F00003309BB012322F104930C010A6FD0DFEFA8
:105F100093851D0013050D0023281101EFC01F926A
:105F200083280101130B0500630005362328A10017
:105F30006FF0CFFB63940D00930D10000323C10F8E
:105F4000032E010F832E410F032F810F13690A10B7
:105F5000E34603C0930A010B1308C10D9307010D1B
:105F60001307C10C93860D001306200093850A00C9
:105F700013050D00232211052328C10B2320C10581
:105F8000232AD10B2322D103232CE10B2320E1036D
:105F9000232E610A232E6100EF2080140323C10108
:105FA00023244103032F0102832E4102032E010407
:105FB00083284104130B0500130A0900232C010454
:105FC000232801006FF05FC4930D60006FD0DFD80D
:105FD000930A010B13850A00232A11052328C10BFC
:105FE000232AD10B232CE10B232E610AEFE0105959
:105FF0001306C10CEF4000721386050093050500DF
:1060000013850A00EFE050388327010B930C010A37
:10601000130901092328F1088327410B13060108FE
:1060200093050900232AF1088327810B13850C00AF
:106030002320C104232CF1088327C10B232001084E
:1060400023220108232EF108B707FC3F2326F1087D
:1060500023240108EFC0C03A0328010A032E410A95
:10606000832E810A032FC10A93850C0013850A0031
:106070002328010B23280105232AC10B2322C10356
:10608000232CD10B2320D103232EE10B232EE1015E
:106090002320010A2322010A2324010A2326010ABC
:1060A000EFC0C000032FC101832E0102032E410265
:1060B0000328010583284105631605009307100096
:1060C0002326F10CB75701809387872F2322F102F3
:1060D0006FF04FF5930470060326C1039306F00F8B
:1060E00083470600638AD71A0327C10113050000FE
:1060F0009305000063DEE7003307F740834716008F
:10610000638407049385150013061600E394D7FEF5
:10611000232EC102232EE1002322B1022324A10257
:106120000327810283274102B387E7000327810405
:10613000B387E702B38C970193CAFCFF93DAFA4165
:10614000B3FA5C016FD0DFE6834706001305150044
:106150006FF0DFFB23280100138A07006FF0DFA038
:106160008327C10293046006B30CF700B38CBC0113
:106170006FF0DFBB9306610D631806009306000302
:10618000230BD10C9306710D1307011B9387070393
:106190003386E6402380F6009307D60D232CF102C8
:1061A0006FD0DFDC930C010A93850C0013850A0085
:1061B000232811052328C10B2320C105232AD10B35
:1061C0002322D103232CE10B2320E103232E610A98
:1061D000232E61002320010A2322010A2324010A1D
:1061E0002326010AEFB0906C0323C101032F0102A3
:1061F000832E4102032E010483280105E30205AA30
:1062000093071000B387B7412326F10C3309F90037
:106210006FD09FBF8327810293F717006394070015
:106220006FD0DFD66FD01FD6639A0700930A100095
:1062300093046006930C10006FF0DF8E8327C10279
:1062400093046006938C1700B38CBC0193CAFCFFC7
:1062500093DAFA41B3FA5C016FF0DF8C1387080020
:106260006FE0DFBD8327410183AD070093874700BF
:1062700063D40D00930DF0FF83441400232AF10032
:10628000130407006FD04FF58357CC0093E7070442
:106290002316FC006FD01F8F23240102232201024A
:1062A0006FF01FE893072000232CF1026FD01FCC62
:1062B0009307050003A5C11C93060600138605007D
:1062C000938507006FD0CFD583D7C50003AE4506B1
:1062D00003D3E50083A8C50103A84502130101B853
:1062E00093F7D7FF13070040232C8146231AF100B0
:1062F000138405009307010793058100232A914623
:1063000023282147232E1146130905002326C10700
:10631000231B610023221103232601032324F10000
:10632000232CF1002328E100232EE1002320010289
:10633000EFD00FCF93040500635C05028357410142
:1063400093F70704638807008357C40093E70704A3
:106350002316F4008320C147032481470329014702
:10636000138504008324414713010148678000001E
:106370009305810013050900EFA01FE7E30005FC6A
:106380009304F0FF6FF09FFB130101FF13870500DB
:1063900023248100232291009305060013040500A5
:1063A00013860600130507002326110023AA0122E5
:1063B000EFA04F919307F0FF630CF5008320C1001D
:1063C0000324810083244100130101016780000040
:1063D00083A74123E38407FE8320C1002320F40028
:1063E0000324810083244100130101016780000020
:1063F00083A7C11C130101FF2324810023229100E4
:10640000232611009304050013840500638607000A
:1064100003A787036300070E0317C4009317070140
:106420009376870093D707016380060483260401CF
:106430006380060613F6170063040608032644016A
:1064400023240400130500003306C040232CC4009D
:10645000638606088320C100032481008324410051
:10646000130101016780000093F607016384060CA5
:1064700093F7470063960708832604011367870094
:10648000931707012316E40093D70701E39406FA54
:1064900013F6072893050020E30EB6F893050400D1
:1064A00013850400EFC00FA60317C4008326040160
:1064B0009317070193D7070113F61700E31006F8A7
:1064C00013F627009305000063140600832544019A
:1064D0002324B40013050000E39E06F693F7070893
:1064E000E38A07F6136707042316E4001305F0FF99
:1064F0006FF05FF613850700EFB0CF886FF0DFF124
:1065000083250403638E0500930704046388F50064
:1065100013850400EFB04FDF0317C40023280402E3
:10652000832604011377B7FD232204002320D4001F
:106530006FF0DFF49307900023A0F40013670704C3
:106540002316E4001305F0FF6FF0DFF003A7811BB3
:1065500083278714638C070403A747001308F001FF
:10656000634EE8061318270063060502338307010C
:106570002324C30883A88718130610003316E600E7
:10658000B3E8C80023A417192324D31093062000CE
:106590006304D5021307170023A2E700B38707019E
:1065A00023A4B70013050000678000009307C714F9
:1065B0002324F7146FF05FFA83A6C7181307170098
:1065C00023A2E70033E6C60023A6C718B387070156
:1065D00023A4B70013050000678000001305F0FF37
:1065E00067800000130101FD232C410103AA811BD8
:1065F000232021032326110203298A142324810244
:1066000023229102232E3101232A510123286101E3
:10661000232671012324810163000904130B050063
:10662000938B0500930A10009309F0FF832449001F
:106630001384F4FF6342040293942400B30499008A
:1066400063840B0483A74410638077051304F4FF6D
:106650009384C4FFE31634FF8320C1020324810224
:1066600083244102032901028329C101032A8101F4
:10667000832A4101032B0101832BC100032C8100DC
:1066800013010103678000008327490083A64400AB
:106690009387F7FF638E870423A20400E38806FA3A
:1066A0008327891833978A00032C4900B377F700B2
:1066B00063920702E78006000327490083278A14B4
:1066C00063148701E304F9F8E38807F813890700E6
:1066D0006FF0DFF58327C91883A544083377F700E7
:1066E000631C070013050B00E78006006FF0DFFC5A
:1066F000232289006FF09FFA13850500E7800600CA
:106700006FF09FFB130101FF2324810023229100DE
:1067100013040500138505002326110023AA012276
:10672000EF901FBA9307F0FF630CF5008320C100C0
:1067300003248100832441001301010167800000CC
:1067400083A74123E38407FE8320C1002320F400B4
:1067500003248100832441001301010167800000AC
:1067600083C7050013072007638AE708130770072C
:10677000638EE70013071006638AE706930760013C
:106780002320F5001305000067800000130300605C
:10679000130710001305800083C7150093851500AB
:1067A00063860702B71800001308B002930680073B
:1067B00093880880638207036394D70033671701C7
:1067C00083C7150093851500E39607FE3367E30042
:1067D0002320E60067800000137535FE1377C7FF9E
:1067E00013650501136727006FF09FFD13038020D9
:1067F00013071000130580106FF01FFA1303000039
:1068000013070000130540006FF01FF9130101FF8B
:106810002324810023229100130405001385050021
:106820002326110023AA0122EF909FAE9307F0FFC9
:10683000630CF5008320C100032481008324410000
:10684000130101016780000083A74123E38407FE51
:106850008320C1002320F40003248100832441000D
:1068600013010101678000009306450093070000B3
:106870001305A5013788FFFF6F00C001939717002C
:106880002390E600939707019386260093D707018C
:10689000630ED50203D706001376170063040600C3
:1068A00093E717001357170013F62700B365070186
:1068B000E30606FC939717002390B6009397070111
:1068C0009386260093D70701E316D5FC6780000066
:1068D0009306850113070000130525006F00C00112
:1068E000131717002390F600131707019386E6FF8E
:1068F000135707016304D50483D7060013960701D5
:106900001356064193971700635406001367170048
:106910009397070193D707011376270093E5170094
:10692000E30006FC131717002390B60013170701A6
:106930009386E6FF13570701E310D5FC678000003C
:10694000130101FE370E0100231D0100231E01006B
:10695000938585019307C10113088100130EFEFF83
:1069600003D705009387E7FF9385E5FF63180702C8
:10697000239F07FEE39607FF130646009306E101F7
:1069800003D707009387270013062600231FE6FE80
:10699000E398D7FE13010102678000003307A702C6
:1069A00083D8270003D30700B376C701B386160147
:1069B0001357070193D80601330767003307170100
:1069C000935807012391D7002390E700239F17FFD7
:1069D000E39807F96FF05FFA130725018357050065
:1069E0001305250063980700E31AE5FE1305000070
:1069F000678000001305100067800000130101FF8D
:106A00002322910083542501232481002326110091
:106A100093C7F4FF139717011304050063160700CB
:106A2000EFF09FFB63180500B787FFFFB3C4F400C6
:106A3000231994008320C100032481008324410092
:106A40001301010167800000130101FF232481006D
:106A500003542501232611009347F4FF13971701D0
:106A6000631A0700EFF05FF79307050013050000B6
:106A7000639407001355F4008320C10003248100B0
:106A8000130101016780000083572501130101FDF7
:106A90002324810293D7F700232291022326110297
:106AA00023202103232E3101B307F0402390F5006A
:106AB00083572501378700001307F7FFB377F700E7
:106AC0002391F50093040500130405016382E70494
:106AD00093876500239205001305E5FF0357040023
:106AE0001304E4FF93872700239FE7FEE31885FE46
:106AF000239C05008320C1020324810283244102D8
:106B0000032901028329C1011301010367800000E9
:106B1000035725011389450033F7E700631CF7028B
:106B20002326B100EFF05FEB8325C100630405026B
:106B300093876500239205001385C4FF0357040063
:106B40001304E4FF93872700239FE7FEE31885FEE5
:106B50006FF05FFA9389A50113092900231F09FE2D
:106B6000E39C29FF8320C102032481028324410284
:106B7000032901028329C101130101036780000079
:106B800083572501130101FB2324810493C7F7FFD9
:106B9000232291042326110413971701930405005F
:106BA0001384050063160700EFF01FE36312050866
:106BB0008357240193C7F7FF139717016304070650
:106BC0009305810013850400EFF01FEC930541024B
:106BD00013050400EFF05FEB83558100035541027C
:106BE000630CB5049307A1001307610213060102A9
:106BF00083D6070093872700639A06088356070009
:106C00001307270063940608E394C7FE13050000EA
:106C10008320C1040324810483244104130101055A
:106C20006780000013050400EFF01FDBE30A05F89E
:106C30001305E0FF6FF0DFFD133515000356A100CB
:106C4000835661023305A0401307A1009307610238
:106C5000137525001305F5FF9305C10393872700DE
:106C600013072700631ED600E382B7FA0356070016
:106C700083D607001307270093872700E306D6FE75
:106C8000E3E8C6F83305A0406FF09FF81305100045
:106C9000E38005F81305F0FF6FF09FF7130101FF84
:106CA00023261100EFF05FD38320C10013351500B8
:106CB0001301010167800000130101FE232C8100F4
:106CC000232A9100232E110023282101232631019C
:106CD000938405001304050063C4050A9307F000BC
:106CE0001386050013054500930684019305F00003
:106CF00063D497029307050003D7270093872700E3
:106D0000239FE7FEE39AD7FE231C0400130606FF29
:106D1000E3C2C5FE93F4F4009307700063D89702B2
:106D2000130784019305240093070000835607008E
:106D30001307E7FF13968600B3E7C7002311F70098
:106D400093D78600E314B7FE938484FF638A04001C
:106D50009384F4FF13050400EFF09FB7E39A04FE59
:106D6000130500008320C101032481018324410114
:106D7000032901018329C10013010102678000007A
:106D8000930710FF3309B04063DCF51293058501CA
:106D900093090000930645001306F0000357840191
:106DA00093870500B3E9E90003D7E7FF9387E7FF7F
:106DB0002391E700E39AD7FE23120400130909FF89
:106DC000E34E26FD930700FF130710FFB38797409C
:106DD0001309000063C4E40A3309F9009307700043
:106DE00063D627059399090193D909418347840103
:106DF0009305A401B3E9F9009399090193D9090115
:106E00009307000003D606009386260013578600DA
:106E100033E7E7009317860093970701239FE6FE69
:106E200093D70701E390B6FE130989FF630C0906A7
:106E3000835784011309F9FF1305040093F7170022
:106E4000B3E93701EFF05FA2E31409FE939709015C
:106E500093D7074163900704139509011355050162
:106E60008320C101032481018324410103290101FD
:106E70008329C100130101026780000013F907FF95
:106E8000330920413309F90093077000E3D027FB51
:106E90006FF05FF593091000139509011355050173
:106EA0006FF01FFC13850900639809001315050195
:106EB000135505016FF01FEB130510006FF01FFF56
:106EC000930790FF93090000E3D4F5F6930644007E
:106ED0006FF0DFF183574500130101FF232291007A
:106EE000232611002324810023202101930405007F
:106EF000639C070C035765001304000093170701F8
:106F000093D7074163C4070A9306A5011306000A35
:106F100063180702938764006F00800003D707009F
:106F200093872700239EE7FEE39AF6FE239C040046
:106F300013040401630CC40603D76400E30C07FCCC
:106F4000937707F0639007041385840193852400E9
:106F50009307000013070500835607001307E7FF98
:106F600013968600B3E7C7002311F70093D7860076
:106F7000E394E5FE03D7640013048400937707F0DD
:106F8000E38807FC1309000A6F0040011304140092
:106F9000EFF01F94634C890003D7640013170701B7
:106FA0001357074113850400E35207FE8320C100F5
:106FB00013050400032481008324410003290100F8
:106FC000130101016780000013F707F013040000AC
:106FD000631007041309F0F66F0040011304F4FF77
:106FE000EFF09F88E30424FD83D744001385040059
:106FF000E39607FE8320C1001305040003248100EB
:10700000832441000329010013010101678000006E
:10701000930645009305A501130700006F0080004B
:1070200083D7060013D687003367C700939787007E
:107030002390E60013970701938626001357070154
:10704000E390B6FE83D74400130480FF6FF09FF8EF
:10705000130101FE232C8100232A91002328210102
:1070600023263101232441012322510113890600E3
:1070700093840700232E1100130405009389050053
:10708000130A0600930A0700EFF0DFE493070009F4
:107090003309A94063DCA716B78700009387E7FF91
:1070A00063DA271F63840A1C03A5440083A7040036
:1070B000630AF5061387A401938744031307270087
:1070C000231F07FEE31CF7FE93078003630CF532D2
:1070D00063D0A71693070004630CF52E93071007DF
:1070E0006318F534B78700409387F7FF1307A000B4
:1070F00023AAF400B787FFFF23A4E400239CF40035
:1071000023A6E4009307A000378700009387870039
:1071100093971700B387F4002395E70023A0A400FA
:107120006358201B83A5840083D744011308F0080B
:10713000139615003306C40003570600B376F70014
:10714000634AA8021308B0006346B802930706001A
:107150009305840103D727006304070093E6160014
:107160002391070093872700E396F5FE0357060057
:1071700083D7440193C7F7FFB3F7E7002310F60066
:1071800083D7640133F7D700630007046384D71AF9
:1071900013862403930684019384C401130700001B
:1071A0008357060083D506009386E6FF1306E6FFA5
:1071B000B387B700B387E70013D707012391F60021
:1071C00013771700E31E96FC635820198357440079
:1071D000639E0712B7870000231C04009387E7FF14
:1071E00063C82709231124018320C10103248101DD
:1071F00083244101032901018329C100032A81005D
:10720000832A410013010102678000006354090EC4
:10721000930700F7635CF908930724001304A401A3
:1072200093872700239F07FEE39C87FE6FF0DFFB19
:10723000930780016308F51693075003631AF51E40
:1072400037170000B7070004930660009387F77FA5
:107250001307078023AAF40023A4D400239CE4008E
:1072600023A6D400930760006FF05FEA231C04009C
:10727000B787FFFF93C7F7FF2311F400930744007C
:10728000130484012390070093872700E31CF4FE76
:107290006FF09FF5930724001304A4019387270040
:1072A000239F07FEE39C87FE6FF01FF49305090000
:1072B00013050400EFF05FA06304050093091000BC
:1072C000638C0A0C03A5440083A70400E314F5DED5
:1072D000930700096304F50A83578401130504002A
:1072E00093F71700B3E9F900EFF00FD803A54400B6
:1072F0006FF05FE3E3800AEE03A5440083A7040078
:10730000E31AF5DAE34020E36FF09FFC1305040075
:10731000EFF08FD5B787000013091900231C040074
:107320009387E7FFE3C627F5E35E09EA231104002C
:107330006FF09FEB6394090C83A7C40003D784010B
:1073400093971700B307F40083D70700B3F7E7005C
:10735000E39007E4E34C20E7930700096306F50098
:1073600013050400EFF0CFD683574400E39007FAEB
:10737000231C0400E34C09FA6FF0DFE603A6840047
:1073800083D74401131616003306C40003570600C2
:10739000B3F6E7006FF01FDE231C04002311040086
:1073A0006FF09FE4B70780009387F70F1307400043
:1073B00023AAF4009307001023A4E400239CF40004
:1073C00023A6E40093074000130700106FF01FD4BA
:1073D0009307700023A4F400B70701809387F7FF99
:1073E00023AAF40093071000239CF4009307600085
:1073F00023A6F400130710006FF05FD1E30A0AD848
:107400006FF09FDCB70780009387F70F13076000CA
:1074100023AAF4009307001023A4E400239CF400A3
:1074200023A6E40093076000130700106FF01FCE3F
:107430009307C00023A4F400B70701809387F7FFE8
:1074400023AAF40093071000239CF4009307B000D4
:1074500023A6F400130710006FF05FCB130101FDAA
:1074600023229102232E31019384050083592500A4
:10747000232611022324810223202103232C4101EE
:1074800013090600232A51012328610123267101D3
:1074900023248101232291012320A101130A050045
:1074A000EFF05FA303D424009307050013850400C5
:1074B000B389F940930A4903EFF0DFA13304A440F4
:1074C0001307E90493870A0093872700239F07FE89
:1074D000E39CE7FE634A3409930B4A00138B440094
:1074E0009389F9FF930CAA01138C240013070B0056
:1074F00093870B0003D60700835607009387270066
:1075000013072700631AD60AE39697FF13068A012A
:1075100013878401930600008357070083550600F4
:107520001307E7FFB387D740B387B74093D6070168
:107530002311F70093F616001306E6FFE31EECFC9A
:10754000130D100013850A00EFF08FB88357C9049C
:107550001304F4FF13850400336DFD002316A90501
:10756000EFF00FB7E31434F993060400032481020B
:107570008320C1028329C101032A8101832A410199
:10758000032B0101832BC100032C8100832C4100BC
:10759000032D01009307090013850400032901024C
:1075A0008324410213070000130600009305000026
:1075B000130101036FF0DFA9130D0000E3E4C6F827
:1075C0006FF0DFF4035705008357250063060700BB
:1075D00037870000B3E7E7002399F500035725003C
:1075E000B78700009387F7FF6304F70293076500EE
:1075F000938505011305850103D7070093872700AD
:107600009385E5FF2391E500E398A7FE67800000DE
:10761000930765001305A50103D70700938727008B
:10762000631A0702E39AA7FE1387250193870500D3
:1076300093872700239F07FEE31CF7FE83D72501CE
:10764000378700001307F7FFB3E7E7002399F5003A
:107650006780000013870501938705009387270043
:10766000239F07FEE31CF7FEB7C7FF7F23A8F500A3
:1076700067800000130101F723286107035B2501E0
:10768000B78700009387F7FF232C410733FA670180
:10769000131A0A0123248108232291082320210997
:1076A000232E310723261108232A51072326710789
:1076B0002324810723229107135A0A01930405000A
:1076C0001389050013040600938906006312FA105B
:1076D000EFF08FB0631A0528835A2901B3775A0156
:1076E0006382472B13850400EFF04FDB630E052EFA
:1076F000B75501809385054E13050900EFF04FC87B
:1077000063060536835A2901B78700009387F7FF80
:10771000B3FA5701939A0A0193DA0A016394FA2C97
:1077200013050900EFF08FD76310053283D72401CA
:10773000B3F7FA006398570B13850400EFF00FD6E8
:107740006318050013050900EFF04FD5630C050819
:1077500013850400EFF04FAF9304050013050900F3
:10776000EFF08FAEB384A440B33490009394F40050
:10777000231994001307240193070400938727001B
:10778000239F07FEE31CF7FE835724013787000081
:107790001307F7FFB3E7E7002319F4008320C108BC
:1077A0000324810883244108032901088329C10790
:1077B000032A8107832A4107032B0107832BC10674
:1077C000032C8106832C4106130101096780000008
:1077D00083DA250133F75701131707011357070100
:1077E000630AF704138504009305C100EFF0CFA9E5
:1077F0001305090093058102EFF00FA98354E100FE
:107800000359A102639C04049307010193064102FA
:107810006388D72003D7070093872700E30A07FE72
:107820001305C100EFF00FEB0357A102B304A04012
:107830006F00000313850500EFF00F9AE30605ECD7
:107840001307490183570900130929001304240071
:10785000231FF4FEE318E9FE6FF05FF4130709003D
:10786000930A09009307C1029306010463120702F9
:107870006382F61C03D7070093872700E30A07FEFD
:1078800013058102EFF00FE50357A102B30AA940E7
:1078900083578102138C8903239BE902239AF902FF
:1078A0001387E90493070C002390070093872700B0
:1078B000E31CF7FE138AC904930B0000130941026D
:1078C000930C0101130B6104035509001309E9FF2F
:1078D0006318050C03D7C90493070A00B3EBEB0048
:1078E00003D7E7FF9387E7FF2391E700E39A87FF3A
:1078F000239C0902E31A99FD138749039307810228
:1079000093052104035607009387270013072700D8
:10791000239FC7FEE398F5FEB7C6FFFFB38454016B
:107920009386260093850B00130581029387090037
:1079300013070004B386D40013060000EFF04FF1E4
:10794000035781028357C100930504001305810288
:10795000B387E740B337F000B307F0402314F102D8
:10796000EFF05FC66FF09FE31387440183D70400F5
:107970009384240013042400231FF4FEE398E4FE00
:107980006FF0DFE113050900EFF00F85E31A05EA58
:1079900013850400EFF08FB0E30805D66FF05FD5D4
:1079A0001306410493058102EFE09FF993050A0055
:1079B000130600001307C10503D80500835707000D
:1079C0009385E5FF1307E7FFB3870701B387C70078
:1079D00013D607012391F50013761600E31E67FD09
:1079E0006FF05FEF03DB2401B78700009387F7FF99
:1079F00033FB6701131B0B01135B0B01E314FBDE6D
:107A000013850400EFF08FA9E31405D483572901EF
:107A100093C7F7FF13971701E31607DC6FF09FD2A8
:107A20009307440113042400231F04FEE39C87FEF4
:107A30006FF0DFD69307440113042400231F04FED4
:107A4000E31CF4FE6FF09FD5B75501809385054E7A
:107A500013850400EFF0CF92630A050083D7240159
:107A6000B3F7FA00E38E57F96FF05FFA13070401DA
:107A70009307040093872700239F07FEE39CE7FEFC
:107A8000B7C7FF7F2328F4006FF05FD1835725012C
:107A9000130101F52324810A93C7F7FF2322910ADA
:107AA0002320210B232E31092326110A232C4109DF
:107AB000232A5109232861092326710923248109D6
:107AC000232291092320A109232EB107139717011F
:107AD000130905009389050013040600938406002A
:107AE00063160700EFE05FEF6318053883D72901BD
:107AF00093C7F7FF13971701630E0708375A0180E2
:107B000093050A4E13050900EFF08F8763040510F3
:107B1000035A290103D72901B78700009387F7FF8C
:107B200033FA4701B3FAE700631AFA0813050900AC
:107B3000EFF0CF966308051063984A01138509009A
:107B4000EFF0CF956310050E930744011304240052
:107B5000231F04FEE31CF4FE8320C10A0324810AD0
:107B60008324410A0329010A8329C109032A8109BF
:107B7000832A4109032B0109832BC108032C8108A7
:107B8000832C4108032D0108832DC1071301010B2C
:107B90006780000013850900EFE01FE4E30005F6AD
:107BA0001387490183D7090093892900130424000E
:107BB000231FF4FEE398E9FE6FF01FFA6386FA08CC
:107BC000130509009305C101EFE01FEC9305810344
:107BD00013850900EFE05FEB835BA1030359E1012B
:107BE00063920B0C9307C103930D0105638EFD3463
:107BF00003D7070093872700E30A07FE13058103D5
:107C0000EFF04FADB307A0400356E1012326F1008A
:107C10006F00C00993050A4E13850900EFE05FF677
:107C2000E31805EE13070401930704009387270068
:107C3000239F07FEE39CE7FEB7C7FF7F2328F400DE
:107C40006FF09FF1E39E4AF713850900EFF00F856F
:107C5000E30805F613050900EFE01FDF93040500B4
:107C600013850900EFE05FDEB387A440B337F0006F
:107C70009397F7002319F4001307240193070400D6
:107C800093872700239F07FEE39CE7FE8357240189
:107C9000378700001307F7FFB3E7E7002319F40065
:107CA0006FF09FEB232671011306090023242101A5
:107CB0009307010293064103631206026380F62ACA
:107CC00003D7070093872700E30A07FE1305C101C6
:107CD000EFF04FA0B307A9402324F100032781034D
:107CE000138D840393070D0023AAE4021389E4048F
:107CF00093872700239F07FEE31CF9FE13058103EA
:107D0000EFE09FB6035C2102370A0100930D0105E5
:107D1000931A0C01B38A8A41130BA103130AFAFFC9
:107D2000930CE106930961058357C1030357E103EF
:107D3000930B0A0093970701B387E70063E8FA0003
:107D4000B3D78703939B070193DB0B011306410510
:107D50009305C10113850B00EFE09FBE1307C1031C
:107D60009307810583D507000356070093872700F3
:107D7000130727006390C512E39697FF930700004F
:107D80009305C10613860D000357060003D80500AE
:107D90001306E6FF3307F740330707419357070100
:107DA0002311E60093F717009385E5FFE31E66FDB8
:107DB00023107D019307C10303D727009387270072
:107DC000239FE7FEE39AB7FF23180104130D2D004C
:107DD000E31CA9F5930500009307C1039306210551
:107DE00003D7070093872700B3E5E500E39AD7FEA2
:107DF0009397050193D7074163840700930510000B
:107E00009395050193D505011387440393078103D7
:107E1000035607009387270013072700239FC7FEF9
:107E2000E398F6FE8327C10003278100B7460000D0
:107E30009386F6FFB38BE740130581039387040015
:107E400013070004B386DB0013060000EFF04FA019
:107E5000035781038357C101930504001305810370
:107E6000B387E740B337F000B307F040231CF102BB
:107E7000EFF04FF56FF05FCE13074901835709000C
:107E80001309290013042400231FF4FEE318E9FE5C
:107E90006FF09FCCE374B6EE9387FBFF93980701D6
:107EA00093D8080193070000930541031306C10608
:107EB0000357060003D805001306E6FF3307F74013
:107EC00033070741935707012311E60093F7170083
:107ED0009385E5FFE31E36FD1307C1039307810574
:107EE00083D5070003560700938727001307270051
:107EF0006398C500E39697FF938B08006FF01FE827
:107F0000E37CB6FE9387EBFF939B070193DB0B01AA
:107F100013060000930541031307C10683570700AA
:107F200003D805001307E7FFB387C740B3870741AE
:107F300013D607012311F700137616009385E5FF8A
:107F4000E31E37FD6FF09FE3930744011304240001
:107F5000231F04FEE39C87FE6FF01FC00357C1017F
:107F6000835781036304F700378600002319C40098
:107F7000130724019307040093872700239F07FE1C
:107F8000E31CF7FE83572401378700001307F7FF30
:107F9000B3E7E7002319F4006FF01FBC130101FDE4
:107FA0002324810223261102138405009307410034
:107FB0001307E10193872700239F07FEE39CE7FE59
:107FC0000356E5009317060193D7074163CA0706D6
:107FD000B78700009387F7FF231201003376F6007E
:107FE000630CF6069307E5002313C1001307A100F5
:107FF00083D6E7FF9387E7FF13072700231FD7FEEA
:10800000E318F5FE63120602231401009305040031
:1080100013054100EFF00FDB8320C102032481022E
:108020001301010367800000930710009305F0FF20
:10803000130541002314F100EFE01FC86FF01FFD8E
:108040009307F0FF2312F100B78700009387F7FF33
:108050003376F600E318F6F8930705009306E5007B
:1080600003D7070093872700631C0704E39AD7FE12
:10807000130744019307040093872700239F07FEFB
:10808000E31CF7FE130724019307040093872700DE
:10809000239F07FEE31CF7FE835724013787000068
:1080A0001307F7FFB3E7E7002319F4008317E50090
:1080B000E3D407F613050400EFE05F946FF0DFF5FB
:1080C000130704019307040093872700239F07FEEB
:1080D000E31CF7FEB7C7FF7F2328F4006FF0DFF340
:1080E00083A8C500130101E183AE050003AE45007E
:1080F00003A38500232E1103832505049308F0FFB5
:1081000023201117930800092324811E232C411DCD
:108110002326111E2322911E2320211F232E311DD1
:10812000232A511D2328611D2326711D2324811D0F
:108130002322911D2320A11D232EB11B2328D1030F
:10814000232AC103232C6102232211172320C100FB
:108150002324D1002326E100232C0101130A05006A
:10816000138407006380050203274504930710006A
:10817000B397E70023A2E50023A4F500EF104056D3
:1081800023200A04930901069385090013050103BE
:10819000EFF0DFE013850900EFE01F8B03270100FC
:1081A0003335A0002320A40093073000E302F71426
:1081B000930740012322F100E318075E835721074C
:1081C0000327411693C7F7FF232AE10013971701EE
:1081D0006318070013850900EFE01F80E3140540D2
:1081E000930700092322F1161307C107938709009B
:1081F0001306410783D6070093872700130727003C
:10820000231FD7FEE398C7FE0356E1082328010089
:108210009317060193D7074163DE07001316160173
:10822000B7070100135616019387F7FF2317C108FC
:108230002328F100375B0180930D0B4E138C4D0109
:10824000930600009307810913070C00130DC10A60
:108250006F0080008356070093872700239FD7FE77
:1082600013072700E398A7FF63080614B7870000E9
:108270009387F7FFE306F6568317C108E3D8075A3A
:108280009305C10713050C00EFE09F8F63020514EF
:10829000E34C050C8357E108E39C07628317C10890
:1082A000930400001309011663C4070213848D119F
:1082B0001306C10793060900930506001305040081
:1082C000EFF04FBB8317C1089384F4FFE3D207FE9E
:1082D0001304010D930B810E130704009307C107CC
:1082E0001306010983D60700938727001307270089
:1082F000231FD7FEE398C7FE93060000930781096A
:1083000013070C006F008000835607009387270037
:10831000239FD7FE13072700E398A7FF938C8D02B6
:10832000138DCD12B7FAFFFF938D8D116F00C00032
:10833000130D4D01938C4C019305040013050C00A3
:10834000EFE01F84930705009305040013050D005B
:108350006356F004EFE0DF829307050093060900FF
:10836000130604009305040013850C0063C0070284
:10837000EFF04FB01306810993060900930506003C
:1083800013850C00EFF00FAFB384540193D7FA01BB
:10839000B387570193DA1740E39CBCF913068109B0
:1083A0009306090093050C0013050600EFF00FEE8D
:1083B000930A41126F0000039307C1079306E10877
:1083C00003D7070093872700E31C07EAE39AD7FE49
:1083D00093040000930A4112130901161304010DBE
:1083E000930B810E9305040013058109EFE0CFE99B
:1083F000130781099307040083D60700938727009A
:1084000013072700231FD7FEE39877FF9305040087
:108410001305C1072318010AEFE00FE79307C1070F
:10842000035704001304240093872700239FE7FECB
:10843000E31874FF13058109130609009305C107AA
:10844000231A0108EFF08F810355C11A6314051C2C
:10845000930C41091304E107130C610B93050B4EB8
:108460001305C107EFE0CFF16306051A13070000FB
:1084700093860C006F00C001131717002390F600BD
:10848000131707019386E6FF1357070163848604D9
:1084900083D70600139607011356064193971700DA
:1084A00063540600136717009397070193D70701DA
:1084B0001376270093E51700E30006FC1317170057
:1084C0002390B600131707019386E6FF13570701A1
:1084D000E39086FC1307410B9307C10783D607007F
:1084E0009387270013072700231FD7FEE39897FFE2
:1084F0002316010C130700009306C10C6F00C00186
:10850000131717002390F600131707019386E6FF51
:10851000135707016384860583D706001396070166
:10852000135606419397170063540600136717000C
:108530009397070193D707011376270093E5170058
:10854000E30006FC131717002390B600131707016A
:108550009386E6FF13570701E39086FD130700009B
:108560009306C10C6F00C001131717002390F6008B
:10857000131707019386E6FF1357070163848605E7
:1085800083D70600139607011356064193971700E9
:1085900063540600136717009397070193D70701E9
:1085A0001376270093E51700E30006FC1317170066
:1085B0002390B600131707019386E6FF13570701B0
:1085C000E39086FD1306000093860C001307C10C90
:1085D00083D50600835707009386E6FF1307E7FF5E
:1085E000B387B700B387C70013D607012391F600FE
:1085F00013761600E31E87FD130581091306090093
:108600009305C107EFE09FE50355C11A9384F4FF7A
:10861000E30605E4832701018326010013073000E8
:10862000B337F000B307F04093F7D7009387070202
:108630002302F112832741006394E600B387970079
:108640001307A002138407006354F7001304A00269
:108650001307A0006302E54E130505031307E002AC
:10866000A302A1122303E112E3C2071E93077112B2
:108670002328F100130C0000232E910093040C001A
:10868000130C090003290101930C410B930D4109BF
:10869000930BE107130D610B1307000013860D0008
:1086A0006F00C001131717002310F60013170701FE
:1086B0001306E6FF13570701630476058357060088
:1086C0009395070193D505419397170063D405004F
:1086D000136717009397070193D707019375270036
:1086E00013E51700E38005FC131717002310A600FD
:1086F000131707011306E6FF13570701E31076FD72
:1087000013870C009307C10703D607009387270040
:1087100013072700231FC7FEE398B7FF2316010C9A
:10872000130700001306C10C6F00C00113171700D8
:108730002310F600131707011306E6FF135707016E
:108740006304A605835706009395070193D5054159
:108750009397170063D405001367170093970701D9
:1087600093D707019375270013E51700E38005FCF5
:10877000131717002310A600131707011306E6FFAF
:1087800013570701E310A6FD130700001306C10CE1
:108790006F00C001131717002310F600131707010D
:1087A0001306E6FF135707016304A6058357060067
:1087B0009395070193D505419397170063D405005E
:1087C000136717009397070193D707019375270045
:1087D00013E51700E38005FC131717002310A6000C
:1087E000131707011306E6FF13570701E310A6FD51
:1087F0009305000013860D001307C10C03550600F6
:10880000835707001306E6FF1307E7FFB387A700A8
:10881000B387B70093D507012311F60093F5150030
:10882000E31EA7FD13060C009305C107130581097C
:10883000EFE0DFC28357C11A330799009384140015
:10884000138607032300C700E35894E41345F4FF9D
:10885000032701011355F5413375A4008324C10199
:108860001309150033092701330CA7001307400033
:10887000635EF70413075000E380E7008347E9FFD6
:108880001307E9FF93F7F707634404789306E002C0
:108890001306800393050003638ED7006352F678B6
:1088A0008347F7FF2300B7001307F7FF93F7F70796
:1088B0006FF09FFE8347F7FF93068003E3F4F60013
:1088C0009307100393841400A30FF7FEB75501809C
:1088D000138604009385C54D13050C00EF10D0746A
:1088E00083572107032741012328911693C7F7FFD8
:1088F0002322E11613971701631E07001385090051
:10890000EFE0CFB96310052213850900EFE0CF8CAB
:10891000631A05208326C100034741129387140080
:1089200023A0F60093870A00630A07029306E00279
:10893000630CD71C03C7170093871700E31A07FEC1
:108940009306500463E6FA006F0040016388570104
:1089500003C7F7FF9387F7FFE31AD7FE23800700CB
:1089600093870A00930600021306D00203C707008C
:108970006304D7006316C700938717006FF01FFFCB
:1089800013840A006F00C00003C7070013840600A9
:108990002300E4009306140093871700E31607FEF4
:1089A00083260100930720000347F4FF6386F61235
:1089B000832741009386070063D4970093860400C1
:1089C000930700036316F702B307544163D2F6021C
:1089D000130600036F00800063DCE6008347E4FFBA
:1089E000A30F04FE1304F4FF33075441E386C7FECC
:1089F00003270100930730006302F70A83278100F1
:108A000023220A04938697009307700163F2D70C20
:108A10001307100093074000939717001386470130
:108A20009305070013071700E3F8C6FE2322BA04D4
:108A300013050A00EF0050402320AA0493850A0082
:108A400093040500EF10D065832781016388070038
:108A5000330454413384840023A087008320C11E43
:108A60000324811E0329011E8329C11D032A811DA0
:108A7000832A411D032B011D832BC11C032C811C48
:108A8000832C411C032D011C832DC11B1385040065
:108A90008324411E1301011F6780000083274100CA
:108AA000B384970063C804508327C1000327810063
:108AB00083A70700B307F7002324F1008327810071
:108AC00023220A049386370093077001E3E2D7F468
:108AD000930500006FF0DFF593070003E310F7F252
:108AE000B307544193061000E3C4F6EE6FF01FF194
:108AF00083248100232291009307A00263D097EC86
:108B00002322F1006FF08FEB03C70700E30A07E2AF
:108B100003C7170093871700A38FE7FEE31A07FE2A
:108B20006FF01FE20327C100B72700009387F7709B
:108B30002320F7006FF0DFE213071003A302E11216
:108B40001307E0022303E11293841400635CF02A0C
:108B500093070003A303F112930781121304F4FF98
:108B60002328F1006FF01FB1930C410B13870C0009
:108B70009307C1071306010983D6070093872700CF
:108B800013072700231FD7FEE398C7FEB74700004F
:108B90009387E7082313F10CB78700009387F7FF4B
:108BA000232EF100B7C7FFFF930A41121304010DF2
:108BB000130E000113838D0C938727002324410398
:108BC0002322510393040000938A0C001309011619
:108BD000930C0400930BA10A2320F102130A0E0048
:108BE00013040300930609001306810993850A0004
:108BF00013050400EFE09FE91307C10493078109FF
:108C000083D607009387270013072700231FD7FE6B
:108C1000E398A7FF8327C1018355E10533F6F500EB
:108C2000832701023305F6006350A03A13060009BA
:108C30003306A64013870C009307C10483D60700B0
:108C40009387270013072700231FD7FEE39837FFDA
:108C50006354C0069307F00013870C0063DCC7025F
:108C6000130606FF935646001387160013171700C6
:108C70003387EC0093870C0093872700239F07FE20
:108C8000E39CE7FE130600083306A64093964600D1
:108C90003306D640131616003386CD0083570700DF
:108CA00083560623B3F7D7002310F70093950501E9
:108CB00093D5054163C005169307810913870C00FE
:108CC00003D6070083560700938727001307270062
:108CD0006314D602E396FBFE13870A00930781090B
:108CE00083D607009387270013072700231FD7FE8B
:108CF000E398A7FFB3844401130444019387CD1282
:108D0000135A1A00E310F4EE8357610C0357E1087D
:108D100013840C00032A8102B387E70037C7FFFFE3
:108D2000938C0A00130727F7832A4102B387E700D1
:108D30002313F10C1307C10793870C001306810C52
:108D400083D607009387270013072700231FD7FE2A
:108D5000E398C7FE13070000930781096F008000A6
:108D600003570C0093872700239FE7FE130C2C006A
:108D7000E398A7FF138D8D02371C0000938D8D1192
:108D80006F000001135C1C006300BD29130D4D0131
:108D900093850C0013850D00EFD09FDE930705002F
:108DA00093850C0013050D006340F026EFD05FDDC6
:108DB000E34AA0FC9306090013860C0093850C007F
:108DC00013050D00EFE09FCC1306810993060900FF
:108DD0009305060013050D00EFE0DF89B3848401DD
:108DE0006FF05FFA930A4112B75501809385854B66
:108DF00013850A00B7240000EF1010239384F47049
:108E00006FF01FAE130C7112E39207AC232881019F
:108E10006FF05F869307C10413870C006F00C000DA
:108E20009306E105E38AF6E803D6070083560700B8
:108E30009387270013072700E304D6FE8357210EEC
:108E40000327C101B377F700639EE70013850C0089
:108E5000EFD09FB8E31205E613850C00EFD01FE4B6
:108E6000E31C05E49305C10E13050C00EFD0DFC130
:108E70009305811013850C00EFD01FC10356C10E5E
:108E80000355A1108358E10E1346F6FF1316060191
:108E9000135606012316C10EB385A840930605009C
:108EA000635EB00683264102130781109307011207
:108EB000835507001307270093862600239FB6FEDD
:108EC000E318F7FE231E0112130781109306C10E4B
:108ED0006F00800003D6060013072700231FC7FE7C
:108EE00093862600E318F7FE832741022310011220
:108EF0001307C10E1306C11383D6070093872700FB
:108F000013072700231FD7FEE398C7FE8356A1103F
:108F1000B305154123120110138506006386052C45
:108F20002326D1029307F0F663C8F5061305C10E98
:108F3000EFD09FD88326C102930505009307011245
:108F4000130541100356C10E03578110630AE62E24
:108F5000130700001306070003D707000358050096
:108F60009387E7FF3307C7403307074113560701CD
:108F70002391E7001307A110137616001305E5FFF0
:108F8000E39CE7FC13061000930709001307000495
:108F900013058110EFE0CF8B93850C001305811032
:108FA000EFE04FE26FF05FD1832781009384F7FFFA
:108FB0006FF05FB48327C1002302011213840A00FB
:108FC00023A007006FF09FAF93870C001307410E9B
:108FD00093872700239F07FEE39CE7FE6FF01FCDDA
:108FE00083270101930A4112638A0706B75501805E
:108FF0009385054C13850A00B7240000EF10D002BA
:109000009384F4706FF0DF8D930B810E6FF08FBD42
:1090100093071003230FF9FE938414006FF01F8B46
:10902000938717002300F7006FF05F8A930A4112BD
:10903000B75501809385854D13850A00B72400003C
:10904000EF10807E9384F4706FF09F898357C11A6C
:10905000130C6112130971126FF05F81B755018013
:109060009385C54C13850A00B7240000EF10C07B20
:109070009384F4706FF0DF86930581091305C107AF
:10908000EFE04FD493050B4E13058109EFD05FAF8E
:10909000631605FEE34C04828347E9FF138727FD2F
:1090A000133717001347F7FF3307EC000347070098
:1090B00013771700E30C07801307E9FF93F7F7070F
:1090C0006FF0CFFC93871700A30FF7FE6FF01F80A0
:1090D0001304010D930504001305C107B74C0000EC
:1090E000EFD09F9A93040000930B810E1309C10CDB
:1090F000930A210D938CECFF8357810E93F7770031
:10910000639A070C1307410B9307040083D60700EB
:109110009387270013072700231FD7FEE39877FFC5
:109120001305410B2316010CEFD00FF41305410B6F
:10913000EFD08FF3130600009306090013870B008E
:1091400083D50600835707009386E6FF1307E7FFE2
:10915000B387B700B387C70013D607012391F60082
:1091600013761600E31E57FD8357610B0357810BDF
:1091700093873700231BF10A630007021305410B95
:10918000EFD08FEE8357610B0357810B9387170046
:10919000231BF10AE31407FE8357C10C639C0702EB
:1091A0008357610B63E8FC02130704009307410B2C
:1091B00083D607009387270013072700231FD7FEB6
:1091C000E39827FF2314010E9384F4FF930750FDC7
:1091D000E394F4F29305C10713050400EFE08FBE9A
:1091E000130901166FF04F8F1307C1109307010F7A
:1091F00083D807000356070093872700130727002B
:109200006398C80213066110E394C7FE0357C10EAA
:10921000835781106302F70693870C001307410EF2
:1092200093872700239F07FEE39CE7FE6FF0DFA8EC
:109230006366160D93070112130541106FF09FD05E
:10924000130700001303E10E03D8070003560500BF
:109250009387E7FF1305E5FF330606013307E600B2
:10926000135607012391E70013771600E31E65FCF0
:10927000130600006FF05FD11387060063920606A5
:109280008317E11063CE0704930601126F000002FA
:109290002390F60013171700131707019386E6FFB4
:1092A0009307A11013570701E388F6CE83D7060072
:1092B000139607011356064193971700635406004F
:1092C000136717009397070193D7070113762700B9
:1092D00093E51700E30E06FA2390B6006FF09FFBAC
:1092E0001306C11093070112631207086382C708AF
:1092F00003570600130626006FF01FFF03264102E6
:109300001307811093070112035507001307270065
:1093100013062600231FA6FEE318F7FE231E0112E4
:10932000130681101307C10E1305411003580700DF
:109330001307270013062600231F06FFE318A7FEC6
:1093400003274102231001129308C10E1306C11313
:10935000035807001307270093882800239F08FF5E
:10936000E318C7FE231201106FF0DFBD138516004E
:109370002315A1106FF05FC2032785008327C50066
:109380000326050083264500130101FC1305010097
:10939000930541012324E1002326F100232E11022D
:1093A0002320C1002322D100EFE05FBF8357610279
:1093B0001305000093C7F7FF13971701631A0700FF
:1093C00013054101EFD04FE11335150013051500CA
:1093D0008320C10313010104678000001305050FFA
:1093E0006780000013850112678000001385011259
:1093F00067800000130101FF232611002324810050
:1094000023229100630C0602B75501809385857372
:109410001305060013040600EFA0CFA8B75401807F
:1094200063120502138544738320C1000324810065
:10943000832441001301010167800000B7540180BB
:109440006FF05FFE9385447313050400EFA08FA5B2
:10945000E30A05FCB75501809385C5311305040067
:10946000EFA04FA4E30005FC130500006FF0DFFB45
:1094700003C58115678000009307050003A5C11C83
:1094800013860500938507006FF0DFF6130101FFD7
:1094900013870500232481002322910093050600F1
:1094A0001304050013860600130507002326110088
:1094B00023AA0122EF605FE99307F0FF630CF50038
:1094C0008320C10003248100832441001301010192
:1094D0006780000083A74123E38407FE8320C10047
:1094E0002320F4000324810083244100130101019F
:1094F0006780000003A34111670003006380050239
:1095000063020604638806048347060023A0F5006F
:10951000034506003335A00067800000130101FFFA
:109520009305C10063040602638A060283470600AE
:1095300023A0F500034506003335A0001301010107
:10954000678000001305000067800000130500001D
:109550006FF0DFFE1305E0FF678000001305E0FFFA
:109560006FF0DFFD9377350093F6F50F638A0702FE
:109570009307F6FF630E06021306F0FF6F008001EB
:109580001305150013773500630E07009387F7FF67
:109590006380C70203470500E314D7FE678000001D
:1095A00093070600130730006366F702639607000F
:1095B0001305000067800000B307F5006F00C000CE
:1095C00013051500E386A7FE03470500E31AD7FE3F
:1095D0006780000037070100939885001307F7FFA5
:1095E000B3F8E80093F5F50FB3E5B80093980501DB
:1095F000B3E8B8003708FFFEB78580801308F8EF9E
:1096000093850508130330000327050033C7E800DE
:10961000330607011347F7FF3377E6003377B700C8
:10962000E31C07F89387C7FF13054500E36EF3FCBF
:10963000E39407F86FF0DFF78327C504130101FFF8
:1096400023248100232291002326110023202101BD
:109650001304050093840500638E0702139524000C
:10966000B387A70003A507006306050403270500C9
:1096700023A0E70023280500232605008320C1003E
:109680000324810083244100032901001301010107
:10969000678000001306100293054000EF508025FC
:1096A0002326A40493070500E31A05FA1305000016
:1096B0006FF0DFFC130910003319990013065900ED
:1096C000131626009305100013050400EF508022A6
:1096D000E30E05FC23229500232425016FF09FF95A
:1096E0006380050203A745008327C50413172700DD
:1096F000B387E70003A7070023A0E50023A0B70076
:1097000067800000130101FE232A910083A4050154
:1097100037030100232C8100232821012326310156
:10972000232E11002324410113890500930905000C
:109730001384060013884501930800001303F3FF08
:10974000832708001308480093881800B3F66700C1
:10975000B386C60293D70701B387C702B3868600D4
:1097600013DE060133F76600B386C701939706013F
:109770003387E700232EE8FE13D40601E3C298FCEA
:10978000630204028327890063D0F40493874400B2
:1097900093972700B307F90023A28700938414004E
:1097A000232899008320C1010324810183244101DE
:1097B0008329C100032A810013050900032901013F
:1097C0001301010267800000832549001385090009
:1097D00093851500EFF05FE603260901130A0500E3
:1097E0009305C90013062600131626001305C500AD
:1097F000EF904FFE0327490083A7C90413172700E2
:10980000B387E70003A707002320E90023A027016F
:1098100013090A006FF09FF7130101FE232C81004A
:10982000232A9100232821012326310123244101E9
:109830001388860093079000232E110023225101E4
:109840003348F802938906001309050013840500C4
:10985000130A06009304070063D6D70C9307100081
:10986000930500009397170093851500E3CC07FF3D
:1098700013050900EFF05FDC930710002328F500C3
:10988000232A9500930790009305050063D64709A6
:10989000930A940093840A003304440183C60400AD
:1098A0001306A00013050900938606FDEFF09FE55F
:1098B0009384140093050500E39284FE13048AFF49
:1098C00033848A0063563A03B3894941B3093401AA
:1098D000834604001306A00013050900938606FDC5
:1098E000EFF05FE21304140093050500E39289FE94
:1098F0008320C10103248101832441010329010143
:109900008329C100032A8100832A410013850500B1
:1099100013010102678000001304A400130A9000E1
:109920006FF05FFA930500006FF09FF43707FFFFB9
:109930003377E50093070500130500006316070061
:109940009397070113050001370700FF33F7E7007E
:10995000631607001305850093978700370700F00B
:1099600033F7E70063160700130545009397470098
:10997000370700C033F7E70063160700130525001B
:109980009397270063C80700139717001305150066
:109990006354070067800000130500026780000021
:1099A000832705001307050093F6770063840602FA
:1099B00093F6170013050000639E060693F6270032
:1099C0006380060893D717002320F70013051000C3
:1099D000678000009396070193D6060113050000E7
:1099E0006396060093D707011305000193F6F70F5E
:1099F000639606001305850093D7870093F6F7005A
:109A0000639606001305450093D7470093F6370089
:109A1000639606001305250093D7270093F61700D9
:109A2000639C060093D71700130515006396070083
:109A300013050002678000002320F7006780000004
:109A400093D727002320F70013052000678000002C
:109A5000130101FF232481001384050093051000E6
:109A600023261100EFF05FBD8320C100232A85006B
:109A700003248100130710002328E50013010101CE
:109A800067800000130101FE2328210123263101F4
:109A900003A9050183290601232A910023244101FA
:109AA000232E1100232C8100138A05009304060045
:109AB000634C390113870900938405009309090059
:109AC000130A06001309070083A7840083A5440036
:109AD00033842901B3A78700B385F500EFF0DFB524
:109AE0001303450193182400B308130193070300DF
:109AF0006378130123A0070093874700E3EC17FF67
:109B000013084A01131E2900938E440193952900DE
:109B1000330EC801B385BE006376C8139387540122
:109B2000130F400063F0F516370601001306F6FF29
:109B30006F00800193DF0F0163980F08130848003E
:109B4000130343006370C811832F0800B3F4CF00E0
:109B5000E38204FE9303030093820E0013090000C6
:109B600003A7020083AF030093834300B376C700CB
:109B7000B38696029357070133F7CF0093DF0F01A7
:109B800093824200B3879702B386E600B38626012C
:109B900013D70601B3F6C600B387F701B387E70012
:109BA00013970701B366D70023AED3FE13D907017D
:109BB000E3E8B2FAB307E30123A02701832F0800EB
:109BC00093DF0F01E38C0FF60327030093020300DA
:109BD00093860E00930407009303000083A70600FA
:109BE00093D904013377C700B3F7C700B387F703EE
:109BF00083A44200938242009386460033F9C40056
:109C0000B3873701B38777009393070133E7E30006
:109C100023AEE2FE03D7E6FF93D707013307F7032E
:109C2000330727013307F70093530701E3E8B6FA38
:109C3000B307E30123A0E700130848001303430020
:109C4000E364C8F1634880006F0080011304F4FFEF
:109C50006308040083A7C8FF9388C8FFE38807FE52
:109C60008320C1012328850003248101832441012D
:109C7000032901018329C100032A81001301010284
:109C800067800000338F9540130FBFFE137FCFFF17
:109C9000130F4F006FF05FE9130101FE232C8100C9
:109CA0002326310123244101232E1100232A910070
:109CB0002328210193773600130406009309050039
:109CC000138A05006394070C1354244013090A00F7
:109CD0006308040683A48904638E040C937714003C
:109CE00013090A006390070213541440630A040422
:109CF00003A5040063080506930405009377140088
:109D0000E38407FE13860400930509001385090008
:109D1000EFF05FD7630809060327490083A7C9044A
:109D20001354144013172700B387E70003A7070055
:109D30002320E90023A0270113090500E31A04FAF0
:109D40008320C10103248101832441018329C100AF
:109D5000032A8100130509000329010113010102EF
:109D600067800000138604009385040013850900B2
:109D7000EFF05FD123A0A400232005009304050089
:109D80006FF0DFF7130905006FF01FF69387F7FFF9
:109D9000375701801307877493972700B307F7009D
:109DA00003A6070093060000EFF0DF95130A0500F5
:109DB0006FF09FF19305100013850900EFF0DF8726
:109DC00093071027232AF500930710002328F50096
:109DD00023A4A90493040500232005006FF01FF0BD
:109DE000130101FE2324410103AA050183A7850075
:109DF0002326310193595640338A4901232C81008F
:109E0000232A91002328210123225101232E11000E
:109E100013091A00938405001304060083A5450066
:109E2000930A050063D827019397170093851500BF
:109E3000E3CC27FF13850A00EFF01F8013084501CC
:109E400063543003938959009399290033073501EE
:109E5000930708009387470023AE07FEE39CE7FEC5
:109E60009389C9FE3308380103A70401938744018D
:109E70001373F401131627003386C700630C03081D
:109E800093050002B385654093080800930600001F
:109E900003A707009388480093874700331767009C
:109EA0003367D70023AEE8FE03A7C7FFB356B7005A
:109EB000E3E0C7FE13875401930740006372E6088E
:109EC0003308F8002320D80063840600130A090031
:109ED00003A7440083A7CA048320C10113172700E6
:109EE000B387E70003A70700232845010324810166
:109EF00023A0E40023A0970003290101832441014A
:109F00008329C100032A8100832A41001301010231
:109F10006780000003A707009387470013084800E5
:109F2000232EE8FEE3F6C7FA03A70700938747004E
:109F300013084800232EE8FEE3EEC7FC6FF05FF93C
:109F4000B30796409387B7FE93F7C7FF9387470001
:109F50003308F8002320D800E38C06F66FF01FF7D3
:109F60000327050183A70501130805003305F74002
:109F70006314F7049397270013084801938545015C
:109F80003307F800B387F5006F0080006376E802BE
:109F90008326C7FF03A6C7FF1307C7FF9387C7FF23
:109FA000E386C6FEB3B6C6003305D0401375E5FFA1
:109FB00013051500678000006780000083A7050176
:109FC00003270601130101FE232C8100232A91009F
:109FD000232821012326310123244101232E1100AE
:109FE0001389050093090600338AE740138445016D
:109FF000930446016398E70413172700B307E400AE
:10A000003387E4006F0080006370F41A03A8C7FF71
:10A010008326C7FF9387C7FF1307C7FFE306D8FE52
:10A020006376D80213070400930709001384040021
:10A03000138909009304070093890700130A10008D
:10A040006F00C000E3400AFE130A000083254900A8
:10A05000EFF08FDE032E090183AF09019302450162
:10A06000931E2E00939F2F00B70801002326450161
:10A07000B30ED401B38FF401138F020013880400D0
:10A0800013030400930700009388F8FF03270300DD
:10A0900083250800130F4F00B3761701B386F6002F
:10A0A000B3F71501B386F64093D505019357070121
:10A0B000B387B74013D70641B387E700139707016B
:10A0C000B3F61601B366D70013084800232EDFFE4F
:10A0D0001303430093D70741E36AF8FB13C6F4FF69
:10A0E0003386CF0093841400135626001307000014
:10A0F00063E49F00131726003387E20093054000B6
:10A1000063E69F0013061600931526003304B4007F
:10A11000B382B200637ED405B70801001388020041
:10A12000930504009388F8FF03A70500130848006F
:10A1300093854500337617013306F60093560641A2
:10A1400093570701B387D70093960701337616011B
:10A15000B3E6C600232ED8FE93D70741E3E6D5FD2C
:10A160001387FEFF330787401377C7FF3387E2006B
:10A17000639A06008327C7FF130EFEFF1307C7FF6E
:10A18000E38A07FE8320C101032481012328C5013E
:10A1900083244101032901018329C100032A81008D
:10A1A000130101026780000093050000EFF0CFC8A3
:10A1B0008320C10103248101930710002328F500A7
:10A1C000232A050083244101032901018329C100B9
:10A1D000032A81001301010267800000B707F07FA6
:10A1E000B3F5B700B707C0FCB385F5006358B000FE
:10A1F000930700001385070067800000B305B04097
:10A2000093D545419307300163C8B700B7070800ED
:10A21000B3D5B7406FF0DFFD1387C5FE9306E001AD
:10A220009305000093071000E3C6E6FCB707008023
:10A23000B3D7E7001385070067800000130101FE14
:10A24000232A910083240501232C81001304450156
:10A2500093942400B30494002328210103A9C4FF8C
:10A2600023263101232441011305090093890500A8
:10A27000232E1100EFF08FEB13070002B307A74066
:10A2800023A0F9009307A000138AC4FF63D0A70896
:10A29000130555FF6370440583A784FF630005041D
:10A2A000B306A74033D7D7003319A9003369E900B3
:10A2B000138684FF3707F03F3367E900B397A700A1
:10A2C0006372C40203A644FFB356D600B3E7D700B7
:10A2D0006F00400193070000631405063707F03F45
:10A2E0003367E9008320C1010324810183244101F4
:10A2F000032901018329C100032A81001385070076
:10A300009305070013010102678000009306B00067
:10A31000B386A640B707F03F3357D9003367F7003D
:10A32000930700006376440183A784FFB3D7D70067
:10A33000130555013315A900B367F5006FF09FFAB7
:10A340003315A9003707F03F3367E5009307000096
:10A350006FF05FF9130101FD232A5101938A050073
:10A36000930510002324810223229102232021033C
:10A3700093040600232E3101232C4101938906000A
:10A380001309070023261102EFF00FAB13D7440186
:10A39000370610009307F6FF9316570113040500C4
:10A3A000B3F79700137AF77F63840600B3E7C7001B
:10A3B0002326F100638C0A06130581002324510132
:10A3C000EFF00FDE0327C100930705006316050AAF
:10A3D00083268100232AD400B334E0009384140040
:10A3E000232CE4002328940063040A06130ADABC31
:10A3F000330AFA001305500323A04901B307F540BF
:10A400002320F9008320C1021305040003248102E4
:10A4100083244102032901028329C101032A810106
:10A42000832A410113010103678000001305C10065
:10A43000EFF00FD7930710002328F4008327C10003
:10A4400093041000232AF40093070502E3100AFA8C
:10A45000139724003307E400032507019387E7BC23
:10A4600023A0F900EFF08FCC93945400B384A44060
:10A47000232099006FF01FF9032681009306000244
:10A48000B386A640B316D700B3E6C6003357A7007D
:10A49000232AD4002326E1006FF01FF4130101FDED
:10A4A000232021031389050093058100232611022F
:10A4B0002324810223229102232E310193090500D6
:10A4C000EFF0DFD79304050013840500130509009E
:10A4D0009305C100EFF09FD68327090103A7090167
:10A4E0008326C1003307F7408327810013175700E5
:10A4F000B387D740B307F70093060500635EF00209
:10A500009397470133848700138606001385040060
:10A510009386050093050400EF60106F8320C1024D
:10A520000324810283244102032901028329C101FA
:10A53000130101036780000013974701B385E540CD
:10A540006FF09FFC130101FF23202101232611003E
:10A550002324810023229100930770011309050031
:10A5600063D6A70483A7011A83A5411A03A4811AFD
:10A5700083A4C11A13850700130604009386040000
:10A58000EF7080561309F9FF93070500E31409FEE5
:10A590008320C1000324810083244100032901009A
:10A5A000138507001301010167800000B757018080
:10A5B000131935009387877433892701832709018D
:10A5C0008320C100032481008325490183244100A5
:10A5D00003290100138507001301010167800000B2
:10A5E000832606019385F5FF93D555409385150085
:10A5F000930746019396260093952500B386D700CE
:10A60000B305B50063F8D7021307050003A80700D8
:10A610009387470013074700232E07FFE3E8D7FE81
:10A62000B387C6409387B7FE93F7C7FF938747006A
:10A630003305F5006378B50013054500232E05FEAC
:10A64000E36CB5FE678000000327050113D6554073
:10A65000930645016352C70293172700B387F6009C
:10A6600063F2F60403A7C7FF9387C7FFE30A07FE59
:10A67000130510006780000093172600B387F600CB
:10A68000E350E6FE93F5F501E38C05FC03A6070015
:10A69000130510003357B600B315B700E302B6FC3C
:10A6A000678000001305000067800000130101FFB0
:10A6B00013870500232481002322910093050600BF
:10A6C0001304050013860600130507002326110056
:10A6D00023AA0122EF50DFD39307F0FF630CF500AC
:10A6E0008320C10003248100832441001301010160
:10A6F0006780000083A74123E38407FE8320C10015
:10A700002320F4000324810083244100130101016C
:10A7100067800000130101FF23229100B70400802D
:10A72000232481002326110093C4F4FF13040600A0
:10A7300023200600B3F6B4003706F07F93870500A8
:10A740001307050063DEC604B3E8A600638A0804A5
:10A7500033F6C50013880500930800006310060255
:10A7600083A6411B03A6011BEF70003813070500E9
:10A7700013880500B3F6B4009308A0FC93D64641B5
:10A78000B70710809387F7FF938626C03378F800C9
:10A79000B3861601B707E03FB367F8002320D40063
:10A7A0008320C10003248100832441001305070096
:10A7B000938507001301010167800000130101F672
:10A7C000930EC108232AF10837030080B707FFFF63
:10A7D000138E05001343F3FF2326D10893878720A8
:10A7E0009305810093860E00232E1106232AF10083
:10A7F0002328E108232C0109232E11092324C10158
:10A80000232CC101232E6100232861002322D101C2
:10A81000EF00402783278100238007008320C107A2
:10A820001301010A67800000130E0500130101F6F1
:10A8300003A5C11C930E8108232AF1083703008069
:10A84000B707FFFF1343F3FF2324C1082326D108D2
:10A85000938787201386050093860E009305810059
:10A86000232E1106232AF1002328E108232C0109B5
:10A87000232E11092324C101232CC101232E6100A1
:10A88000232861002322D101EF00C01F832781000C
:10A89000238007008320C1071301010A678000009D
:10A8A000B367B50093F737006392070803A7050065
:10A8B000B7867F7F9386F6F7B377D700B387D70045
:10A8C000B3E7E700B3E7D7001306F0FF639EC706C0
:10A8D000130605001308F0FF2320E60003A7450038
:10A8E0009385450013064600B377D700B387D7009A
:10A8F000B3E7E700B3E7D700E38007FF83C70500AE
:10A9000003C7150083C625002300F600638A0700ED
:10A91000A300E600630607002301D6006394060047
:10A9200067800000A3010600678000009307050010
:10A9300003C705009387170093851500A38FE7FED3
:10A94000E31807FE67800000130605006FF01FFB89
:10A950009377350013070500639C0704B7867F7F54
:10A960009386F6F79305F0FF0326070013074700C9
:10A97000B377D600B387D700B3E7C700B3E7D700F4
:10A98000E384B7FE8346C7FF0346D7FF8347E7FF4D
:10A990003307A74063800604630A06023335F000DC
:10A9A0003305E5001305E5FF67800000E38806FA3C
:10A9B000834707001307170093763700E39807FED5
:10A9C0003307A7401305F7FF678000001305D7FF83
:10A9D000678000001305C7FF67800000B3E7A5008C
:10A9E00093F73700130705006398070693073000B5
:10A9F00063F4C7063703FFFEB78880801303F3EFC5
:10AA000093880808130E300083A60500B3876600FC
:10AA100013C8F6FFB3F70701B3F71701639E0702E8
:10AA20002320D7001306C6FF130747009385450070
:10AA3000E36CCEFC938515009307170063040602B0
:10AA400083C6F5FF1308F6FFA38FD7FE638E0600BB
:10AA50001387070013060800938515009307170056
:10AA6000E31006FE678000003306C700630A080093
:10AA700093871700A38F07FEE39CC7FE6780000043
:10AA800067800000130101E12326111E2320211FEE
:10AA90002324811D2320A11D138C0500130906000A
:10AAA000232AD1002324811E2322911E232E311D0F
:10AAB000232C411D232A511D2328611D2326711D8E
:10AAC0002322911D232EB11B130D0500EFE09F9152
:10AAD00083270500138507002328F102EFF05FE7C5
:10AAE0000357CC002328010E232A010E232C010E2C
:10AAF000232E010E137707082326A10263080700FF
:10AB000003270C01631407006F10C0569307C11090
:10AB1000376701802322F10E938807009307078788
:10AB200037670180232CF100130B09009307C79EA0
:10AB30002324F10083470B002326010E2324010E5A
:10AB400023200102232A0102232C0102232E0102C9
:10AB50002324010423260104232601006384072201
:10AB600013040B00930650026384D72C8347140010
:10AB700013041400E39A07FEB304644163046421E0
:10AB80008326C10E8327810E23A06801B386960019
:10AB90009387170023A298002326D10E2324F10EB9
:10ABA000930670009388880063CCF6280327C100C1
:10ABB00083470400330797002326E1006384071CC2
:10ABC00083441400A303010C13041400930DF0FF3D
:10ABD00093090000130A00001309A005930A9000CE
:10ABE000930BA002938C080013041400938704FEB7
:10ABF0006364F9040327810193972700B387E70073
:10AC000083A707006780070093090000938604FD6F
:10AC10008344040093972900B38737019397170063
:10AC2000B389F600938604FD13041400E3F2DAFE00
:10AC3000938704FEE370F9FC93880C00638404148A
:10AC400023069114A303010C930A1000930C100027
:10AC5000130BC11423280100930D000023240102CB
:10AC600023220102232E0100937B2A0063840B0020
:10AC7000938A2A0013794A088327C10E63160900B4
:10AC800033885941E34C00638346710C638A0602A2
:10AC90008326810E1306710C23A0C800938717002A
:10ACA000130610009386160023A2C8002326F10E77
:10ACB0002324D10E1306700093888800634CD64C71
:10ACC000638A0B028326810E1306810C23A0C80021
:10ACD00093872700130620009386160023A2C8003E
:10ACE0002326F10E2324D10E1306700093888800CA
:10ACF000E34CD66A93060008E300D942B38D9D4128
:10AD0000E34EB04D93760A10E39A062C0327810E8A
:10AD1000B387970123A068011307170023A29801A6
:10AD20002326F10E2324E10E9306700063C0E65A39
:10AD300093888800137A4A0063060A00B384594155
:10AD40006346905A63D4590193890A000327C100CE
:10AD5000330737012326E100E39C075283270101D3
:10AD60002324010E638807008325010113050D00CC
:10AD7000EF609FD99308C110130B040083470B00A9
:10AD8000E39007DE8327C10E638407006F10503401
:10AD90000357CC0013770704630407006F20803F3C
:10ADA0008320C11E0324811E0325C1008324411E6C
:10ADB0000329011E8329C11D032A811D832A411DE8
:10ADC000032B011D832BC11C032C811C832C411CD4
:10ADD000032D011C832DC11B1301011F678000007F
:10ADE00013050D00EFE00FE08327450013850700F2
:10ADF0002326F104EFF0DFB59307050013050D00DE
:10AE0000938407002324F104EFE0CFDD832785003E
:10AE1000232EF102638404006F1040168344040063
:10AE20006FF09FDC83440400136A0A026FF0DFDBDB
:10AE3000B3046441E31664D5834704006FF01FD860
:10AE40001306410E93050C0013050D00EF4090060C
:10AE5000E31005F49308C1106FF05FD593778A0073
:10AE600093880C00638407006F10800A83274101D8
:10AE70001305010B232891019387770093F787FF30
:10AE800083A5070003A6470093878700232AF100C4
:10AE9000EF90904F8327010B832801012328F10EA7
:10AEA0008327410B232AF10E8327810B232CF10EDC
:10AEB0008327C10B232EF10E1305010F2328110147
:10AEC000EFE08FCB2326A10C9307200083280101FC
:10AED0006314F5006F108065930710006314F5008C
:10AEE0006F105007930710066394F4006F20C01989
:10AEF000930710046394F4006F10D05293FBF4FD99
:10AF00009307F0FF232A71056394FD006F10502111
:10AF1000930770046394FB006F20801E0323C10F0E
:10AF200023244103032E010F832E410F032F810F92
:10AF300093670A10635403006F20C039232C010467
:10AF4000138A070023280100930760046394FB0021
:10AF50006F10902B93075004232211056384FB008C
:10AF60006F10D03313891D00930A010B930609005B
:10AF70001308C10D9307010D1307C10C1306200020
:10AF800093850A0013050D002328C10B2320C1055A
:10AF9000232AD10B2322D103232CE10B2320E1030D
:10AFA000232E610A232E6100EFD08F930323C1016A
:10AFB000032F0102832E4102032E01048328410442
:10AFC000130B050033092501930C010A93850C002E
:10AFD00013850A00232E11012328C10B232AD10B2C
:10AFE000232CE10B232E610A2320010A2322010ACC
:10AFF0002324010A2326010AEF70400B8328C10194
:10B0000013070900630205020327C10D637E2701B0
:10B010009306000393071700232EF10C2300D7009B
:10B020000327C10DE36827FFB30767412320F1021F
:10B030000327C10C93077004232EE1000327410569
:10B040006314F7006F105011032741059307600444
:10B050006314F7006F10D0348327C1010327410523
:10B06000930510049387F7FF2326F10C93F6F40F52
:10B07000130600006318B7009386F60093F6F60FE8
:10B0800013061000230AD10C9306B00263DA0700FE
:10B090000327C101930710009306D002B387E7404E
:10B0A000A30AD10C9306900063C4F6006F20400FF2
:10B0B0001308310E130508001306A000130E300606
:10B0C00033E7C70293050500938607001305F5FFD4
:10B0D00013070703A38FE5FEB3C7C702E342DEFEF3
:10B0E0009387070313F6F70FA30FC5FE9387E5FFBA
:10B0F00063E407016F2080399306610D6F008000C3
:10B1000003C607002380C6009387170093861600A6
:10B11000E39807FF9307510EB387B7401307610DFC
:10B12000B307F7009306410DB387D740232CF102F4
:10B13000032701028326810393071000B30CD70075
:10B1400063C4E7006F2000238327C102B38CFC0097
:10B150008327810293CAFCFF93DAFA4113FAF7BFFF
:10B16000136A0A10B3FA5C012324010223220102AC
:10B17000232E010083278105639407006F101005BB
:10B180009307D002A303F10C930D0000938A1A00D9
:10B190006FF09FAD1306410E93050C0013050D00D3
:10B1A000EF404051E31005108327C10E9308C110F2
:10B1B0006FF01FB18326810E938C17008327010245
:10B1C0001306100023A068019384160013898800D9
:10B1D000E358F6369307100023A2F8002326910FB8
:10B1E0002324910E93077000E3C0974A8327C1027E
:10B1F0000327010393841400B38CFC002322F9007D
:10B200002320E9002326910F2324910E9307700039
:10B2100013098900E3CC97488327010F1386140094
:10B220009305010A2328F10A8327410F1305010B17
:10B23000232EC100232AF10A8327810F2320010A2C
:10B240002322010A232CF10A8327C10F2324010A98
:10B250002326010A232EF10AEF6050650326C1015F
:10B26000832701029308890093060600938DF7FF58
:10B27000E30C052E13071B00B38CBC012320E9004F
:10B280002322B9012326910F2324C10E93077000B6
:10B2900063D4C7006F1080019307090193862400CF
:10B2A0001389080093880700032681031307410DC3
:10B2B0002320E900B30796012322C9002326F10EBB
:10B2C0002324D10E13077000E356D7A61306410EB0
:10B2D00093050C0013050D00EF40C03D6314057C81
:10B2E0008327C10E9308C1106FF0DFA493060001FD
:10B2F0000327810E63C496006F101012B766018099
:10B30000938EC69D13090001130A7000138B0E0063
:10B310006F00C000938404FF63569904938707016C
:10B320001307170023A0680123A228012326F10E8A
:10B330002324E10E93888800E35EEAFC1306410EA5
:10B3400093050C0013050D00EF40C036631C057417
:10B35000938404FF8327C10E0327810E9308C11035
:10B36000E34E99FA930E0B00B3879700130717006B
:10B3700023A0D80123A298002326F10E2324E10E56
:10B3800093067000E3D0E69C1306410E93050C0073
:10B3900013050D00EF400032631605708327C10EC0
:10B3A0006FF05F9A83274101A303010C93880C007F
:10B3B00003AB070013894700E3020B4E9307F0FF2E
:10B3C0006394FD006F10C01F13860D0093050000ED
:10B3D00013050B00232A9101EFE0CF982328A10049
:10B3E00083284101631405006F10C0758327010194
:10B3F000232A210123280100B38C67418347710C64
:10B4000093CAFCFF93DAFA412324010223220102AA
:10B41000232E0100B3FA5C01930D0000E38607843C
:10B42000938A1A006FF05F840327410193880C0010
:10B43000A303010C8327070013074700232AE10019
:10B440002306F114930A1000930C1000130BC1147F
:10B450006FF05F8083440400136A4A006FF0CFF8F6
:10B460008326410193770A0293880C0003A7060004
:10B4700093864600232AD100E390072893770A0198
:10B48000638407006F10C01293770A046384070077
:10B490006F10803D137A0A2063140A006F10401168
:10B4A0008327C100130B04002300F7006FF01F8DEA
:10B4B000834404009307C006E38EF438136A0A013C
:10B4C0006FF08FF203274101B787FFFF93C7078310
:10B4D0002314F10C93074700232AF10003290700E6
:10B4E000B75701809387872F93880C00232AF10296
:10B4F000930C0000936B2A009307200093048007AD
:10B50000A303010C1307F0FF6386ED203367990155
:10B5100013FAFBF7631E071E63940D266390071C46
:10B5200093FC1B00130B011BE3900C1C938A0C0073
:10B5300063D4BC01938A0D008347710C232801005A
:10B540002324010223220102232E0100E39A07ECA7
:10B550006FF08FF193880C00136A0A0193770A0247
:10B56000E38C070683274101138B7700137B8BFF46
:10B5700003290B00832C4B0093078B00232AF10037
:10B58000937BFABF930700006FF09FF7834404009A
:10B5900093078006E388F42C136A0A046FF0CFE463
:10B5A00093880C00936B0A0193F70B02E38C07045A
:10B5B00083274101138B7700137B8BFF93078B004D
:10B5C000232AF10003290B00832C4B009307100062
:10B5D0006FF01FF383440400136A8A006FF0CFE01A
:10B5E000832741018344040083A907009387470010
:10B5F000232AF10063DA09DEB3093041136A4A00F5
:10B600006FF08FDE83440400136A1A006FF0CFDD01
:10B610008347710C83440400639807DC930700029E
:10B62000A303F10C6FF04FDC83440400136A0A0893
:10B630006FF08FDB834404001307140063947401DC
:10B640006F10505F938604FD13040700930D0000F4
:10B6500063EEDAD88344040093972D00B387B701D3
:10B6600093971700B38DD700938604FD130414003D
:10B67000E3F2DAFE6FF08FD79307B0028344040041
:10B68000A303F10C6FF04FD693880C00136A0A01E4
:10B6900093770A026380077A83274101138B77002F
:10B6A000137B8BFF83274B0003290B0013078B00B1
:10B6B000232AE100938C070063C6077A9307F0FF03
:10B6C000930B0A006384FD02B3679901937BFAF739
:10B6D000639E070063920D02138A0B00930D000016
:10B6E000930C0000130B011B6FF05FE4E3960C401A
:10B6F00093079000E3E2274113090903A307211BE5
:10B70000138A0B00930C1000130BF11A6FF01FE259
:10B71000930B0A0013071000E38AE7FC13072000CD
:10B72000638CE706130B011B1397DC0193777900F9
:10B7300013593900938707033369270193DC3C00D1
:10B74000A30FFBFE3367990113060B00130BFBFFDE
:10B75000E31C07FC93F61B00638A060693060003AE
:10B760006386D7061306E6FF9307011BA30FDBFED4
:10B77000B38CC740138A0B00130B06006FF01FDB5E
:10B78000130710006394E7006F10101713072000D1
:10B79000930B0A00E398E7F883264103130B011B80
:10B7A0009377F900B387F60003C7070013594900E0
:10B7B0009397CC0133E9270193DC4C00A30FEBFEF8
:10B7C000B3679901130BFBFFE39C07FC9307011B75
:10B7D000B38C6741138A0B006FF05FD59306500658
:10B7E000E3DA969C8326010F9305010A1305010BEA
:10B7F0002328D10A8326410F232211052320F10497
:10B80000232AD10A8326810F2320010A2322010A39
:10B81000232CD10A8326C10F2324010A2326010ADF
:10B82000232ED10AEF609008832701048328410466
:10B83000631C05380327810EB75601809386863234
:10B8400023A0D80093871700930610001307170052
:10B8500023A2D8002326F10E2324E10E93067000C4
:10B8600093888800E3CCE6440327C10C83260102B9
:10B870006350D766032701038326C102938888009B
:10B8800023ACE8FE0327810EB387D70023AED8FE92
:10B89000130717002326F10E2324E10E93067000F0
:10B8A00063CCE676032701029304F7FF635490C844
:10B8B000930600010327810EE3D29642130900018B
:10B8C000930C70006F00C000938404FFE35899400C
:10B8D00083268100938707011307170023A0D80050
:10B8E00023A228012326F10E2324E10E9388880049
:10B8F000E3DCECFC1306410E93050C0013050D0070
:10B90000EF30505B6310051A8327C10E0327810EA9
:10B910009308C1106FF05FFB33895941635020BF1A
:10B92000130600018326810E63542607130E0001BF
:10B93000930B70006F00C000130909FF635A2E05B6
:10B9400003278100938707019386160023A0E80050
:10B9500023A2C8012326F10E2324D10E9388880048
:10B96000E3DCDBFC1306410E93050C0013050D0010
:10B97000EF30505463180512130E0001130909FF2C
:10B980008327C10E8326810E9308C110E34A2EFB44
:10B9900003278100B38727019386160023A0E800C0
:10B9A00023A228012326F10E2324D10E13067000B2
:10B9B000938888006354D6B41306410E93050C0097
:10B9C00013050D00EF30104F631E050CB38D9D4124
:10B9D0008327C10E9308C1106356B0B3130600014C
:10B9E0008326810E6352B607930B00011309700082
:10B9F0006F00C000938D0DFF63D8BB050327810046
:10BA0000938707019386160023A0E80023A27801FC
:10BA10002326F10E2324D10E93888800E35CD9FC01
:10BA20001306410E93050C0013050D00EF309048EE
:10BA3000631A0506938D0DFF8327C10E8326810EA1
:10BA40009308C110E3CCBBFB03278100B387B70188
:10BA50009386160023A0E80023A2B8012326F10E46
:10BA60002324D10E1306700093888800635CD6A847
:10BA70001306410E93050C0013050D00EF309043A3
:10BA8000631205028327C10E9308C1106FF08FA7C0
:10BA90001306410E93050C0013050D00EF30904185
:10BAA000630E05AA832B010163840BAE93850B0003
:10BAB00013050D00EF604F856FF08FAD3767018084
:10BAC000130600018326810E930EC79D635C060951
:10BAD000232081042322910413040D0093040C00FD
:10BAE000130E000193027000130C0800138D0E005A
:10BAF0006F00C000130C0CFF635A8E05938707017B
:10BB00009386160023A0A80123A2C8012326F10EC4
:10BB10002324D10E93888800E3DED2FC1306410E65
:10BB20009385040013050400EF30D038E3120516A6
:10BB3000130E0001130C0CFF8327C10E8326810E08
:10BB40009308C11093027000E34A8EFB13080C00A7
:10BB5000930E0D00138C0400130D04008324410484
:10BB600003240104B38707019386160023A0D8019C
:10BB700023A208012326F10E2324D10E1306700000
:10BB8000938888006352D6901306410E93050C00EB
:10BB900013050D00EF301032E31605F08327C10EB8
:10BBA0009308C1106FF04F8E1306410E93050C00E1
:10BBB00013050D00EF301030E31605EE8327C10E9C
:10BBC0009308C1106FF00F938325C10C635CB07EA6
:10BBD0000327C101832601029304070063C2E63CE8
:10BBE000635690028326810EB387970023A06801D5
:10BBF0009386160023A298002326F10E2324D10E4B
:10BC00001306700093888800E34CD64093C6F4FF77
:10BC10000327C10193D6F641B3F4D400B30497408F
:10BC2000634E90480327C10193760A40B30DEB00A1
:10BC3000639A064E8324C10C0327010263C6E40005
:10BC400093761A00E3820640832601030327C1028C
:10BC50001306700023A0D8008326810EB387E70067
:10BC600023A2E800938616002326F10E2324D10E8A
:10BC700093888800E344D66A832601023307DB00F9
:10BC8000B38496403307B741138904006354970087
:10BC900013090700635620030327810EB38727018A
:10BCA00023A0B8011307170023A228012326F10EB1
:10BCB0002324E10E9306700093888800E3CAE66AA5
:10BCC0001347F9FF1357F7413377E900B384E44092
:10BCD000634490006FF00F86930600010327810EE6
:10BCE00063DE967E13090001930C70006F00C000A4
:10BCF000938404FF6354997E832681009387070110
:10BD00001307170023A0D80023A228012326F10E31
:10BD10002324E10E93888800E3DCECFC1306410E3B
:10BD200093050C0013050D00EF30D018E31C05D669
:10BD30008327C10E0327810E9308C1106FF05FFBAC
:10BD400093771A00639807C823A2C8002326910F8F
:10BD50002324910E9307700063CA9754938626009C
:10BD6000938808016FF04FD46350B0D513070001DA
:10BD70006344B7016F10806B130B700093040600CF
:10BD80006F000001938D0DFFE35EB71193841400E3
:10BD900083278100938C0C012322E9002320F900E2
:10BDA0002326910F2324910E13098900E35C9BFC49
:10BDB0001306410E93050C0013050D00EF30900F94
:10BDC000E31205CE832CC10E8324810E1309C1100A
:10BDD000130700016FF01FFB8326410193770A01CF
:10BDE000138746006394071893770A04E3860714C1
:10BDF00083274101930C0000232AE10003D90700A7
:10BE00006FF00FF88326410193F70B01138746006B
:10BE10006394071493F70B04E38007108327410111
:10BE2000930C0000232AE10003D9070093071000B8
:10BE30006FF00FED8326410193770A0113874600C7
:10BE40006392071093770A04E388070A8327410166
:10BE5000232AE10003990700935CF94193870C00C2
:10BE6000E3DE0784B3372001B30C9041B38CFC4070
:10BE70009307D002A303F10C33092041930B0A006E
:10BE8000930710006FF00FE81306410E93050C00A6
:10BE900013050D00EF301002E31605C0832CC10E10
:10BEA0008324810E1309C1106FF04FB41306410EA5
:10BEB00093050C0013050D00EF30C07FE31405BEA1
:10BEC000832CC10E8324810E1309C1106FF0CFB4EF
:10BED00013771A00631407006FE0DFE56FF09F9996
:10BEE00093880C006FF0CFFA93070003A307F11AB1
:10BEF000130BF11A6FF08FE38326C100130B0400BC
:10BF000093D7F6412320D7002322F7006FE01FE7E5
:10BF1000032741018327070013074700232AE10075
:10BF200083A5070003A6470083A6870083A7C70051
:10BF30002328B10E232AC10E232CD10E232EF10E5D
:10BF40006FE09FF703A90600232AE100935CF94103
:10BF500093870C006FF04FF603A90600930C0000C6
:10BF6000232AE100930710006FF08FD903A9060080
:10BF7000930C0000232AE1006FF08FE08327C103B8
:10BF800083440400639407006FE01FC683C7070063
:10BF9000639407006FE05FC5136A0A406FE0DFC477
:10BFA00093840600E34090C46FF05FC693880C0052
:10BFB000930B0A006FF04FDFB75701809387872FED
:10BFC00093880C00232AF10293770A026380072CDE
:10BFD00083274101138B7700137B8BFF03290B0011
:10BFE000832C4B0093078B00232AF10093771A00D0
:10BFF000638E0700B3679901638A07009307000304
:10C000002304F10CA304910C136A2A00937BFABF5A
:10C01000930720006FF0CFCE1306410E93050C005E
:10C0200013050D00EF300069E31E05A68327C10E3E
:10C030009308C1106FF01F87B75701809387C730EF
:10C0400093880C00232AF1026FF01FF893880C00EC
:10C050006FF0CFD083441400136A0A021304140053
:10C060006FE09FB883441400136A0A20130414007D
:10C070006FE09FB79305000413050D00EF600FFC00
:10C080002320AC002328AC00631405006F10C03CD3
:10C0900013070004232AEC006FE05FA793076000FA
:10C0A000938C0D0063EEB77937570180938A0C00AB
:10C0B000232A2101130B07326FE0DFB913060001B9
:10C0C0008326810E6358966A930C0001930D7000CD
:10C0D0006F00C000938404FF63DE9C680327810027
:10C0E000938707019386160023A0E80023A29801F6
:10C0F0002326F10E2324D10E93888800E3DCDDFC97
:10C100001306410E93050C0013050D00EF30805A05
:10C11000E31A05988327C10E8326810E9308C11068
:10C120006FF05FFB03270102832C4102232E4101A4
:10C1300023208104232231052322510383298102F4
:10C1400023246103B30BEB000324C103032A8104FE
:10C15000832AC1049304700013090001130B0C001F
:10C1600063880C08639809081304F4FF938CFCFFA0
:10C170000327810EB387470123A058011307170037
:10C1800023A248012326F10E2324E10E9388880080
:10C1900063C4E414834604003386BB41138C060059
:10C1A0006354D600130C0600635680038326810E69
:10C1B000B387870123A0B8019386160023A28801C4
:10C1C0002326F10E2324D10E63C0D4348346040009
:10C1D000938888001346FCFF1356F6413377CC0052
:10C1E000338CE640634C8001B38DDD00E39C0CF69C
:10C1F000638C09729389F9FF6FF09FF78326810E94
:10C20000634889016F008005130C0CFF6358890592
:10C2100003278100938707019386160023A0E80077
:10C2200023A228012326F10E2324D10E938888000F
:10C23000E3DCD4FC1306410E93050B0013050D003F
:10C24000EF304047631C055A130C0CFF8327C10EC7
:10C250008326810E9308C110E34C89FB03278100DC
:10C26000B38787019386160023A0E80023A28801E4
:10C270002326F10E2324D10E63C4D4768346040012
:10C2800093888800B38DDD006FF05FF6832641014F
:10C2900093770A01138746006384072003A90600E9
:10C2A000930C0000232AE1006FF05FD41306410EC7
:10C2B00093050C0013050D00EF30C03F631405FE1D
:10C2C0008326810E832CC10E93084111938616009C
:10C2D0001309C1106FE05FFD1306410E93050B00BB
:10C2E00013050D00EF30003D631A05508327C10E82
:10C2F0009308C1106FF01FEA130B011B9307000096
:10C3000023288100232E910013040B0023223103E4
:10C31000130B0C009304090093890C0013FA0B40D3
:10C32000832CC103930AF00F138C080013890700B4
:10C330006F0040021306A00093060000138504005E
:10C3400093850900EF4010086380094C93040500B1
:10C35000938905001306A0009306000013850400CE
:10C3600093850900EF40504913050503A30FA4FE70
:10C37000130919001304F4FFE30E0AFA83C60C0034
:10C38000E31AD9FAE30859FB639A0942930790002C
:10C3900063E6974293080C009307011B130C0B00F4
:10C3A000130B0400232E91038324C101832941022E
:10C3B0000324010123202103B38C6741138A0B005E
:10C3C0006FF0CF968326810E375601801306863292
:10C3D00023A0C80093871700130610009386160049
:10C3E00023A2C8002326F10E2324D10E13067000C9
:10C3F00093888800634CD6066398052003270102C2
:10C4000093761A00B3E6E600639406006FE09F920D
:10C41000832601030327C1021306700023A0D8005E
:10C420008326810EB387E70023A2E80093861600D7
:10C430002326F10E2324D10E634ED64A938888001A
:10C44000032701029386160023A06801B387E70043
:10C4500023A2E8002326F10E2324D10E1307700037
:10C460006344D7006FE0DF8C6FE05FE61306410E98
:10C4700093050C0013050D00EF30C023631405E293
:10C480008325C10C8327C10E9308C1106FF0DFF61E
:10C49000832B0101130D0400138C04006FF0CFE017
:10C4A00093770A04638C072283274101930C0000D1
:10C4B000232AE10003D907006FF05FB31306410E92
:10C4C00093050C0013050D00EF30C01E631C05DC46
:10C4D0008327C10E9308C1106FF00FB98326810026
:10C4E000B387970023A2980023A0D8001307170052
:10C4F0002326F10E2324E10E9306700063C4E600A8
:10C500006FE01F836FE09FDC1306410E93050B0065
:10C5100013050D00EF30001A6312052E8346040048
:10C520008327C10E9308C1106FF0DFCA8327010F64
:10C530009305010A1305010B2328F10A8327410FF4
:10C540002320010A2322010A232AF10A8327810FCB
:10C550002324010A2326010A232CF10A8327C10F71
:10C56000232EF10AEF5090558328010163420552B2
:10C570008347710C13077004635E97283757018057
:10C58000130BC72E232801002324010223220102BA
:10C59000232E0100137AFAF7930A3000930C30002F
:10C5A000930D0000638407006FE09FE76FE0CFEB1F
:10C5B0008327C100130B04002320F7006FE00FFC5A
:10C5C00013050B0023209105EFE08FB88347710C12
:10C5D000934AF5FF93DAFA41232A21012328010027
:10C5E0002324010223220102232E010083280104B7
:10C5F000930C0500B37A5501930D00006384070086
:10C600006FE01FE26FE04FE6832601030327C102BC
:10C610001306700023A0D8008326810EB387E7009D
:10C6200023A2E800938616002326F10E2324D10EC0
:10C63000938888006340D62CE3D405E0130600FFFE
:10C64000B304B040E3D4C52613090001930C700075
:10C650006F00C000938404FFE35A992403278100EC
:10C66000938707019386160023A0E80023A22801E0
:10C670002326F10E2324D10E93888800E3DCDCFC12
:10C680001306410E93050C0013050D00EF308002D8
:10C69000631A05C08327C10E8326810E9308C1103B
:10C6A0006FF05FFB938614001307890083278100D6
:10C6B000B38CBC012322B9012320F9002326910F5A
:10C6C0002324D10E93077000E3C2D7BE93861600D1
:10C6D00093088700130907006FE01FBD93770A20B6
:10C6E000638E071C83274101930C0000232AE1007D
:10C6F00003C907006FF09F8F93770A206384071A9E
:10C7000083274101232AE10003890700935CF94153
:10C7100093870C006FE05FFA93F70B20638807168E
:10C7200083274101930C0000232AE10003C907007D
:10C73000930710006FE0DFDC93770A20638E071207
:10C7400083274101930C0000232AE10003C907005D
:10C750006FE01FE38327C10F63C807188347710C7D
:10C7600013077004635C974637570180130B472FFC
:10C770006FF05FE103278100B3879700938616006F
:10C7800023A0E80023A298002326F10E2324D10E33
:10C7900013067000938888006356D6C81306410EAE
:10C7A00093050C0013050D00EF20D070631C05AE3F
:10C7B0008327C10E9308C1106FF0CFC68327810471
:10C7C0008325C104130900003304F44013860700D5
:10C7D00013050400EFE08FA083C51C001306A00022
:10C7E000930600003338B0001385040093850900D8
:10C7F000B38C0C01EF40003D6FF05FB5832B01015E
:10C80000130C0B006FF04FAA93079000E3E097B46E
:10C810006FF05FB837570180130B872E6FF09FD6EC
:10C820001306410E93050C0013050D00EF209068D0
:10C83000631A05A68327C10E9308C1106FF00FBDC0
:10C84000930C60006FF05F86832601023307DB00E4
:10C85000B38496403308B74113890400635298C6E5
:10C86000130908006FF0CFC58327C100130B040024
:10C870002310F7006FE08FD083274101930C000055
:10C88000232AE10003A907006FE09FCF832741011E
:10C89000930C0000232AE10003A90700930710006E
:10C8A0006FE01FC683274101232AE10003A9070087
:10C8B000935CF94193870C006FE01FE083274101EF
:10C8C000930C0000232AE10003A907006FF00FF288
:10C8D0001306410E93050C0013050D00EF20905D2B
:10C8E0000357CC006FE00FCB9307D002A303F10CEA
:10C8F0006FF01FE71306410E93050C0013050D00A2
:10C90000EF20505B6310059A8325C10C8327C10E6D
:10C910008326810E9308C110E3D405B26FF01FD2B5
:10C92000930D60006FE08FDF03270102130C0B00F3
:10C93000032B8102232E8102032AC101B306EB00DF
:10C940000324010483294104832A410263F4B6AF1E
:10C95000938D06006FF00FAE0327C1019307D0FF40
:10C960006344F70063DAED009384E4FF93F7F4FD8A
:10C97000232AF1046FE04FEE832701020327C10150
:10C980006344F72683278102930C070093F717006F
:10C99000638607008327C102B30CF7008327810257
:10C9A00093F70740638607008327C101E34AF0122B
:10C9B00093CAFCFF93DAFA41B3FA5C019304700660
:10C9C00023240102232201026FE0CFFA8347710C76
:10C9D000930D0000638407006FE09FA46FE0CFA871
:10C9E0001306410E93050B0013050D00EF20904C2C
:10C9F000E31605E0834604008327C10E9308C110A7
:10CA0000B38DDD006FF08FFE930A010B1308C10D8B
:10CA10009307010D1307C10C93860D001306300018
:10CA200093850A0013050D00232211052328C10B4D
:10CA30002320C105232AD10B2322D103232CE10B70
:10CA40002320E103232E610A232E6100EFB04FE97A
:10CA50000323C101032F0102832E4102032E01048F
:10CA600083284104130B0500930760043309BB01BD
:10CA7000639AFB6283460B0093070003E386F6107C
:10CA8000930C010A8327C10C3309F9006FE00FD41E
:10CA90009307D002A303F10C6FF0DFAD930A010BF3
:10CAA0009307010D1308C10D1307C10C93860D00E8
:10CAB0001306200093850A0013050D002328C10BDF
:10CAC0002320C105232AD10B2322D103232CE10BE0
:10CAD0002320E103232E610A232E6100EFB04FE0F3
:10CAE000930770040323C101032F0102832E410227
:10CAF000032E010483284104130B0500E396FBF683
:10CB00008327810293F717006398075893077004EF
:10CB10000327C10D232AF1046FE00FD11306410E44
:10CB200093050C0013050D00EF20D03863040500B9
:10CB30006FE05FF78324C10C8327C10E9308C110F7
:10CB40006FF08F938347710C232A21012324010264
:10CB500023220102232E0100938A0D00938C0D00E5
:10CB6000930D0000638407006FE09F8B6FE0CF8F11
:10CB70001306410E93050C0013050D00EF209033B2
:10CB8000630405006FE01FF28324C10C0327010238
:10CB90008327C10E9308C110B30497406FF04F92E2
:10CBA000832781020327C10193F71700B3E7B70179
:10CBB000E354E0046396077A832CC1019304600672
:10CBC0008327810293F70740639E077093CAFCFF97
:10CBD00093DAFA41B3FA5C016FF09FDE37570180B8
:10CBE000130B072F6FF01F9A832701020327C1023F
:10CBF00093047006B38CE7008327C101E342F0FC85
:10CC0000B38CFC40938C1C0093CAFCFF93DAFA416E
:10CC1000B3FA5C016FF0DFDAB7660180938EC69DD0
:10CC20006FE08FF4930700032304F10C9307800552
:10CC300013672A00A304F10C2324E10293073006B2
:10CC400023280100130BC11463CEB7410323C10F86
:10CC500093FBF4FD232A7105232C0104032E010FFD
:10CC6000832E410F032F810F136A2A10634203386A
:10CC700093071006638EF454930710046384F40042
:10CC80006FE08FAC930A010B13850A00232811056E
:10CC90002328C10B232AD10B232CE10B232E610A5D
:10CCA000EF80C00D1306C10CEFD0DFA61386050080
:10CCB0009305050013850A00EF70106D8327010BA3
:10CCC000930C010A130901092328F1088327410B5A
:10CCD0001306010893050900232AF1088327810B15
:10CCE00013850C002320C104232CF1088327C10BDA
:10CCF0002320010823220108232EF108B707FC3F57
:10CD00002326F10823240108EF50806F0328010A2D
:10CD1000032E410A832E810A032FC10A93850C003A
:10CD200013850A002328010B23220105232AC10BA6
:10CD30002322C103232CD10B2320D103232EE10B6B
:10CD4000232EE1012320010A2322010A2324010AC0
:10CD50002326010AEF508035032FC101832E0102E3
:10CD6000032E4102032841048328010563160500B0
:10CD7000930710002326F10CB75701809387C73023
:10CD80002322F1029386FDFF232E410523229106E3
:10CD90002326B107232AA107232C8107930B0B001D
:10CDA000232081062324310723281107138C060032
:10CDB000232E6107130D0800930D0E0093840E00BF
:10CDC000130A0F006F00800493850C0013850A007E
:10CDD0002320C102232EF101232CF10B232EC10AA3
:10CDE0002328610B232A310B2320010A2322010A65
:10CDF0002324010A2326010AEF50402B832FC1016F
:10CE000003260102130CFCFF6302050EB707034063
:10CE10001306090093850C0013850A00232EF108E0
:10CE20002320A10B2322B10B2324910A2326410B9B
:10CE300023280108232A0108232C0108EF50405C15
:10CE400013850A00EF70102E9305050013040500EA
:10CE500013850A008329010B8324410B032B810BCB
:10CE6000032AC10BEF70503D0327010B0326010479
:10CE7000930509002320E1080327410B13850C00CB
:10CE8000232831092322E1080327810B232A910853
:10CE9000232C61092324E1080327C10B232E410918
:10CEA0002326E108EF60005683274102032B010A85
:10CEB0008329410A3387870003470700832F810AAC
:10CEC0000326C10A232871052380EB002322810554
:10CED0009307F0FF938B1B00130D0B00938D09003C
:10CEE00093840F00130A0600E310FCEE8328010769
:10CEF00093030B00938209003709FE3F93850C00D2
:10CF000013850A0023201103232E8100032AC10563
:10CF100083244106032401062328710A2322710673
:10CF2000232A510A23205106232CF10B232EF1052D
:10CF3000232EC10A2320C1042320010A2322010A2F
:10CF40002324010A2326210BEF500023832DC10641
:10CF5000032D4107032C8107032BC1078329810679
:10CF6000832801026340A00A83234106832201062D
:10CF7000832FC1050326010493850C0013850A0045
:10CF80002328710A232A510A232CF10B232EC10ACC
:10CF90002320010A2322010A2324010A2326210B2C
:10CFA000EF50C01083280102631805008327C101D8
:10CFB00093FC170063980C048327410413060003B5
:10CFC00093861700B386DB0063C80700938B1B00B2
:10CFD000A38FCBFEE39CDBFEB3876B412320F102E2
:10CFE0006FE00F852324410323280100130A090061
:10CFF000B707008033C367009307D002232CF104E6
:10D000006FF01FC78327010593860B00232EF10CB9
:10D010008327410203C6FBFF83C5F7006310B602F6
:10D0200013050003A38FA6FE8326C10D9387F6FF89
:10D03000232EF10C03C6F6FFE386C5FE930516000A
:10D040001305900393F5F50F6306A600A38FB6FEB4
:10D050006FF09FF88327410283C5A700A38FB6FE18
:10D060006FF09FF793851D0013050D002328110114
:10D07000EF50CFFC83280101130B05006308053E28
:10D080002328A1006FF09FBC930700032304F10C39
:10D09000930780076FF0DFB9930770043309BB0172
:10D0A000232AF104930C010A6FD05FF20327810059
:10D0B000B38797009386160023A0E80023A2980068
:10D0C0002326F10E2324D10E130670006358D6B622
:10D0D0001306410E93050C0013050D00EF20805D33
:10D0E000630405006FE01F9C8327C10E8326810E19
:10D0F0009308C1106FF0CFB4930B0A006FE0CFDF3D
:10D1000063940D00930D10000323C10F032E010F34
:10D11000832E410F032F810F13690A10E34403ECA0
:10D12000930A010B1308C10D9307010D1307C10CDE
:10D1300093860D001306200093850A0013050D0049
:10D14000232211052328C10B2320C105232AD10B3B
:10D150002322D103232CE10B2320E103232E610A98
:10D16000232E6100EFA0DFF70323C1012324410335
:10D17000032F0102832E4102032E01048328410460
:10D18000130B0500130A090023280100232C0104B6
:10D190006FF01F979307F0FF2326F1006FD05FC059
:10D1A0009306610D6318060093060003230BD10C50
:10D1B0009306710D1307011B938707033386E6401F
:10D1C0002380F6009307D60D232CF1026FD05FF673
:10D1D000930A010B13850A00232811052328C10B8C
:10D1E000232AD10B232CE10B232E610AEF70103977
:10D1F0001306C10CEFD00FD213860500930505006E
:10D2000013850A00EF7050188327010B930C010A55
:10D21000130901092328F1088327410B130601088C
:10D2200093050900232AF1088327810B13850C003D
:10D230002320C104232CF1088327C10B23200108DC
:10D2400023220108232EF108B707FC3F2326F1080B
:10D2500023240108EF50C01A0328010A032E410AB3
:10D26000832E810A032FC10A93850C0013850A00BF
:10D270002328010B23220105232AC10B2322C103EA
:10D28000232CD10B2320D103232EE10B232EE101EC
:10D290002320010A2322010A2324010A2326010A4A
:10D2A000EF40D060032FC101832E0102032E410203
:10D2B0000328410483280105631605009307100025
:10D2C0002326F10CB75701809387872F2322F10281
:10D2D0006FF05FAB23280100138A07006FF05FD166
:10D2E000930470060326C1039306F00F83470600DC
:10D2F0006388D7180327C1011305000093050000B8
:10D3000063DEE7003307F7408347160063840704B2
:10D310009385150013061600E394D7FE232EC10251
:10D32000232EE1002322B1022324A102032781023C
:10D3300083274102B387E70003278104B387E7020D
:10D34000B38C970193CAFCFF93DAFA41B3FA5C01FC
:10D350006FD05FE283470600130515006FF0DFFB17
:10D360008327C10293046006B30CF700B38CBC01A1
:10D370006FF01F858327810293F7170063940700DE
:10D380006FD01FDD6FD05FDC930C010A93850C001A
:10D3900013850A00232211052328C10B2320C10570
:10D3A000232AD10B2322D103232CE10B2320E103D9
:10D3B000232E610A232E61002320010A2322010A61
:10D3C0002324010A2326010AEF40504E0323C10102
:10D3D000032F0102832E4102032E010483284104FE
:10D3E000630205EA93071000B387B7412326F10CC7
:10D3F0003309F9006FD09FBD639A0700930A1000AC
:10D4000093046006930C10006FF08FDB8327C1023A
:10D4100093046006938C1700B38CBC0193CAFCFF85
:10D4200093DAFA41B3FA5C016FF08FD913870800E1
:10D430006FF0CFA78327410183AD07009387470093
:10D4400063D40D00930DF0FF83441400232AF100F0
:10D45000130407006FD04FF99307C0002320FD008D
:10D460009307F0FF2326F1006FD09F930357CC0062
:10D4700093670704138707002316FC006FD09F9162
:10D4800023240102232201026FF05FEA93072000A8
:10D49000232CF1026FD0DFC983A74506130101FDDC
:10D4A00023286101232611022324810223229102D1
:10D4B00023202103232E3101232C4101232A510152
:10D4C000232671012324810113972701130B0600E2
:10D4D0006358070A83278600832B060013890500FB
:10D4E00093090500930AF0FF6388070803AC4B001B
:10D4F00003A40B00135A2C0063060A0693040000D1
:10D500006F00C00013044400630C9A0483250400D8
:10D510001306090013850900EF10805B9384140043
:10D52000E31255FF1305F0FF8320C102032481029B
:10D5300023240B0023220B00832441020329010230
:10D540008329C101032A8101832A4101032B01019F
:10D55000832BC100032C81001301010367800000AD
:10D5600083278B00137CCCFFB38787412324FB00E8
:10D57000938B8B00E39C07F6130500006FF0DFFA36
:10D58000EF10805F6FF05FFA0327860063040700E7
:10D590006FF09FF023220600130500006780000053
:10D5A000130101ED232E3111232C4111232671117A
:10D5B00023261112232481122322911223202113C6
:10D5C000232A51112328611123248111232291112F
:10D5D0002320A111232EB10F2328D100130A050007
:10D5E00093890500930B06006306050083278503D6
:10D5F000638E075E0397C9009317070193162701EF
:10D6000093D7070163CA0602B727000083A649061D
:10D61000B367F7009397070137E7FFFF93D70741F9
:10D620001307F7FF33F7E6002396F90093970701F6
:10D6300023A2E90693D7070113F787006300074089
:10D6400003A70901630C073E93F7A7011307A00086
:10D650006386E740B76701809387C79F376B018078
:10D660009304C104232AF1003769018093078BB624
:10D67000138C0B0023209104232401042322010492
:10D68000232C0100232E010023220102232001026A
:10D69000232601002324F100130989B7938B04008A
:10D6A00083470C006388072613040C0013075002FD
:10D6B000638EE7428347140013041400E39A07FEC5
:10D6C000B30C844163088425032781048327410424
:10D6D00023A08B013387EC009387170023A29B01C3
:10D6E0002324E1042322F10493067000938B8B0022
:10D6F00063D0F602E30A073A130601049385090092
:10D7000013050A00EFF05FD9631A0520938B04001C
:10D710000327C10083470400330797012326E10054
:10D72000638A071E03471400130C1400A30D0102A3
:10D73000930AF0FF23220100130B0000930CA005B5
:10D74000130D90001306A002130C1C00930707FE94
:10D7500063E8FC048326410193972700B387D70031
:10D7600083A707006780070023220100930707FDB6
:10D770008325410003470C00130C1C0093962500E1
:10D78000B386B60093961600B387D7002322F10024
:10D79000930707FDE37EFDFC930707FEE3FCFCFA1D
:10D7A000630A07162306E108A30D0102930C10007B
:10D7B000130D10001304C108930A0000937F2B007F
:10D7C00063840F00938C2C0003274104137F4B08C4
:10D7D00083278104930617001386060063180F0041
:10D7E00083254100B38D9541E342B0098345B103E0
:10D7F00093868B00638C05021307B1039387170090
:10D8000023A0EB001307100023A2EB002324F10454
:10D810002322C104130770006340C77E130706006C
:10D82000938B06001306160093868600638E0F0402
:10D830001307C1039387270023A0EB0013072000E1
:10D8400023A2EB002324F1042322C1041307700058
:10D85000E350C700E384072A1306010493850900F7
:10D8600013050A002324E103EFF01FC36318050A20
:10D870000327410483278104032F81029306410576
:10D8800013061700938B0400930500086306BF5A24
:10D89000B38AAA4163425069B307FD0023A08B00FD
:10D8A00023A2AB012324F1042322C1041307700037
:10D8B0006352C702E38E070A130601049385090029
:10D8C00013050A00EFF05FBD631A05048327810486
:10D8D0009386040013734B00630803000327410081
:10D8E000B30B9741E344700B03244100635494014C
:10D8F00013840C000327C100330787002326E100AF
:10D900006398076C83470C0023220104938B040067
:10D91000E39C07D883278104E39A076483D7C9006F
:10D9200093F70704E39207688320C112032481124E
:10D930000325C10083244112032901128329C11147
:10D94000032A8111832A4111032B0111832BC1105A
:10D95000032C8110832C4110032D0110832DC10F46
:10D96000130101136780000013050A00EFB09FA7A1
:10D9700083274500138507002320F102EFC05FFDD8
:10D980009307050013050A00138407002322F10200
:10D99000EFB05FA5832785001306A002232EF100B8
:10D9A000E318042A03470C006FF01FDA03470C004A
:10D9B000136B0B026FF05FD9136B0B0193770B02A4
:10D9C00063840716832701019387770093F787FF06
:10D9D00003A7470003AD0700938787002328F100C2
:10D9E000930C0700634A07161307F0FF930D0B0013
:10D9F0006388EA0033679D01937DFBF7E30C070A18
:10DA0000E3960C1613079000E362A71793070D0324
:10DA1000A307F10E138B0D00130D10001304F10E6C
:10DA2000938C0A0063D4AA01930C0D008347B103C1
:10DA3000B337F000B38CFC006FF05FD8938509001A
:10DA400013050A00EF80DF9AE310055683D7C9005B
:10DA50001307A00093F7A701E39EE7BE8397E900B1
:10DA6000E3CA07BE8326010113860B0093850900D4
:10DA700013050A00EF0090582326A1006FF0DFEA9B
:10DA8000136B0B0193770B02638A0706832701014F
:10DA90009387770093F787FF03AD070083AC4700B8
:10DAA000938787002328F100937DFBBF13070000B5
:10DAB000A30D01029306F0FF6384DA0CB3669D01A7
:10DAC00013FBFDF76390065A639C0A306318077EC8
:10DAD00013FD1D001304010FE3040DF4930700036D
:10DAE000A307F10E1304F10E6FF09FF3B30C844102
:10DAF000E31C84BD834704006FF09FC283260101AD
:10DB000093770B0113874600E39C071693770B046A
:10DB1000E388073883270101930C00002328E100E4
:10DB200003DD07006FF05FF88326010193770B0197
:10DB300013874600E394071093770B04E3820732C0
:10DB4000832701012328E100039D0700935CFD4129
:10DB500013870C00E35A07E83337A001B30E904156
:10DB6000B38CEE401307D002A30DE1029306F0FF41
:10DB7000330DA041930D0B0013071000E390DAF46E
:10DB800093061000E30ED7E6930620006304D72621
:10DB90001304010F9397DC0113777D00135D3D00A3
:10DBA0001307070333EDA70193DC3C00A30FE4FE4A
:10DBB000B3679D01130604001304F4FFE39C07FC04
:10DBC00093F71D006382072693070003630EF72473
:10DBD0001306E6FFA30FF4FE9307010F338DC74032
:10DBE000138B0D00130406006FF09FE3EF309F9935
:10DBF0006FF05FA083270101A30D010203A40700BA
:10DC0000938D4700E30004229307F0FFE388FA12A4
:10DC100013860A009305000013050400EFB09F94DB
:10DC2000E3000536330D85402328B101930A000037
:10DC30006FF01FDF03270101A30D0102930C1000F9
:10DC400083270700130747002328E1002306F10874
:10DC5000130D10001304C1086FF01FB683270101D4
:10DC60003787FFFF1347078303AD070093874700FC
:10DC70002328F100B75701809387872F231EE102E5
:10DC8000930C0000936D2B00232CF1001307200050
:10DC90006FF01FE203470C009307C006E306F71678
:10DCA000136B0B016FF05FAA03470C00930780060C
:10DCB000E304F714136B0B046FF01FA9936D0B01B2
:10DCC00093F70D0263840760832701011307100097
:10DCD0009387770093F787FF03AD070083AC470076
:10DCE000938787002328F1006FF09FDC03470C0027
:10DCF000136B0B086FF05FA58326010103470C002F
:10DD000083A70600938646002328D1002322F10032
:10DD1000E3DC07A2B307F0402322F100136B4B00B2
:10DD20006FF09FA203470C00136B1B006FF0DFA185
:10DD30008347B10303470C00E39807A09307000251
:10DD4000A30DF1026FF05FA003470C00136B4B00B3
:10DD50006FF09F9F9307B00203470C00A30DF102E1
:10DD60006FF09F9E03470C0093061C00E30AC72434
:10DD7000930707FD138C0600930A0000E368FD9CDF
:10DD800003470C0093962A00B38A5601939A1A000F
:10DD9000B38AFA00930707FD130C1C00E372FDFE23
:10DDA0006FF0DF9A8326010193770B0203A7060029
:10DDB000938646002328D100639A076A93770B0164
:10DDC000E39C070493770B04E390071413730B2071
:10DDD000E30403048327C1002300F7006FF05F8C86
:10DDE00093061000E30ED71A93062000930D0B0044
:10DDF000E310D7DA832681011304010F9377FD0026
:10DE0000B387F60003C70700135D4D009397CC015D
:10DE100033EDA70193DC4C00A30FE4FEB3679D0133
:10DE20001304F4FFE39C07FC9307010F338D874035
:10DE3000138B0D006FF0DFBE83254100B38D95413C
:10DE4000E358B0A593050001E3D6B517930E000182
:10DE5000130F70006F00800113062700938B8B0057
:10DE600013870600938D0DFF63DCBE0593870701C2
:10DE70009306170023A02B0123A2DB012324F10426
:10DE80002322D104E35ADFFC638007161306010442
:10DE90009385090013050A00EFF00FE0E31005A8D1
:10DEA00003274104930E0001938D0DFF8327810406
:10DEB000938B040013061700130F7000E3C8BEFB1A
:10DEC0009305060013858B00B387B70123A02B01B0
:10DED00023A2BB012324F1042322B1041307700001
:10DEE000635AB7526386077E1306010493850900BF
:10DEF00013050A00EFF04FDAE31205A203274104ED
:10DF0000B38AAA41832781049306410513061700AB
:10DF1000938B0400E35250999305000163D0557B25
:10DF200093080001930D70006F0080011306270015
:10DF3000938B8B0013870600938A0AFF63DA5805D8
:10DF4000938707019306170023A02B0123A21B012F
:10DF50002324F1042322D104E3DADDFC63820706E3
:10DF6000130601049385090013050A00EFF0CFD2D0
:10DF7000E316059A0327410493080001938A0AFFD8
:10DF800083278104938B040013061700E3CA58FB10
:10DF900093858B00B387570123A02B0123A25B013C
:10DFA0002324F1042322C104130770006346C72C05
:10DFB0001306160093868500938B05006FF0DF8DA6
:10DFC0001306100013070000938B04006FF0DFF6B8
:10DFD000130601049385090013050A00EFF0CFCB67
:10DFE000E30205926FF09F931306100013070000E1
:10DFF000938B04006FF01FE7638C07301306010456
:10E000009385090013050A002326E1032324F10365
:10E01000EFF08FC8E31405900327410483278104A0
:10E02000032FC102832F81029306410513061700B7
:10E03000938B04006FF08FFF9307C1032326F10435
:10E04000930720002328F1041306100093064105CE
:10E0500013070600938B06001306170093868B00A8
:10E060006FF09F82930D0B006FF09FB113060001BC
:10E070006350B67313860B00930E0001930B0400DC
:10E0800093027000138409002324F10393890D0087
:10E09000930D0C00138C0A00930A0F006F00C0014F
:10E0A000130527001306860013870600938909FFCE
:10E0B00063DE3E05930617008325810093870701E1
:10E0C0002322D6012320B6002324F1042322D104E5
:10E0D000E3D8D2FC63860708130601049305040005
:10E0E00013050A00EFF04FBB6316054C03274104EC
:10E0F000930E0001938909FF83278104138604008E
:10E100001305170093027000E3C63EFB832F8102C4
:10E11000138F0A0093050500930A0C00138C0D0061
:10E12000938D09009309040013840B00930B0600E0
:10E1300003278100B387B70123A2BB0123A0EB0013
:10E140002324F1042322B104130770006342B71E95
:10E15000938B8B0013861500138705006FF00FE972
:10E160001307000013051000138604006FF01FF45E
:10E170002322010413734B006302030E03274100A3
:10E18000B30B9741635C700D938604001307000185
:10E190000326410463527761130D0001930D700053
:10E1A0006F00800113052600938686001306070082
:10E1B000938B0BFF635A7D058325810093870701AD
:10E1C0001307160023A0B60023A2A6012324F104FE
:10E1D0002322E104E3D8EDFC638A07061306010459
:10E1E0009385090013050A00EFF00FAB631805F2E1
:10E1F00003264104938B0BFF83278104938604003D
:10E2000013051600E34A7DFB9305050003278100F3
:10E21000B387770123A2760123A0E6002324F1042B
:10E220002322B104130770006350B7EC6388070220
:10E23000130601049385090013050A00EFF0CFA52A
:10E24000631E05EC832781046FF00FEA13051000AD
:10E2500013060000938604006FF09FF5032441002D
:10E260006354940113840C008327C100B387870093
:10E270002326F1006FF00FE96382073413060104CF
:10E280009385090013050A00EFF00FA1631805E854
:10E2900003264104832781049306410513061600D3
:10E2A000938B04006FF04FDF23220104938B040053
:10E2B0006FF00FC6639C0AF4138B0D00930A0000E5
:10E2C000130D00001304010F6FF08FF58326010179
:10E2D00093F70D01138746006398071493F70D0415
:10E2E0006380073A83270101930C00002328E10093
:10E2F00003DD0700130710006FF08FFB9306410545
:10E300001306100013070000938B04006FF0CFD7A3
:10E3100063800F189307C1032326F104930720009D
:10E320002328F10413071000930B41056FF0DFD28F
:10E3300063820722130601049385090013050A006E
:10E340002326E1032324F103EFF00F95631805DC86
:10E350000327410483278104032FC102832F8102F5
:10E36000938B0400130617006FF04FC893F70D400E
:10E370002324410323263103138A0C0093090D0043
:10E38000130B0000032DC1011304010F938C070030
:10E390006F0040021306A0009306000013850900D9
:10E3A00093050A00EF201002630E0A30930905005E
:10E3B000138A05001306A0009306000013850900C8
:10E3C00093050A00EF20504313050503A30FA4FE95
:10E3D000130B1B001304F4FFE38E0CFA83460D00AD
:10E3E000E39A66FB9307F00FE306FBFA63140A183F
:10E3F0009307900063E037199307010F232EA101C3
:10E40000032A81028329C102338D8740138B0D00BB
:10E410006FF00FE113861500930685001387050042
:10E42000930B05006FF0CFC62328E10003AD060073
:10E43000930C0000130710006FF08FE703AD060088
:10E440002328E100935CFD4113870C006FF08FD906
:10E450008327C10103470C00638807AE83C7070009
:10E46000638407AE136B0B406FF00FAE8326C100C1
:10E4700093D7F6412320D7002322F7006FF04FA255
:10E4800003AD0600930C00002328E1006FF0CFE1FC
:10E49000130700009306410513061000938B040038
:10E4A0006FF08FBE930D0B006FF09F81B757018007
:10E4B0009387C730232CF10093770B026380070604
:10E4C000832701019387770093F787FF03AD070048
:10E4D00083AC4700938787002328F10093761B00C5
:10E4E000638E0600B3669D01638A060093060003EF
:10E4F000230ED102A30EE102136B2B00937DFBBF11
:10E50000130720006FF0CFDAB75701809387872F6A
:10E51000232CF10093770B02E39407FA0326010101
:10E5200093770B0193064600638A070A032D0600C2
:10E53000930C00002328D1006FF05FFA130504004C
:10E54000EFC00FC1130D05002328B101930A00008D
:10E550006FF00FCD0347B103631A0718E39E0FACAA
:10E56000130700001306100093064105938B040067
:10E570006FF08FB18327410283250102130B000046
:10E580003304F4401386070013050400EFC00FC5E1
:10E5900083451D001306A000930600003337B0002A
:10E5A0001385090093050A00330DED00EF2080610B
:10E5B0006FF0DFDF930904006FF04FB61307100010
:10E5C00093070D00232681042328A1052324A105F8
:10E5D0002322E104930641056FF0CFAF93770B043C
:10E5E0006382070683270101930C00002328D100D2
:10E5F00003DD07006FF09FEE03471C00136B0B2039
:10E60000130C1C006FF04F9403471C00136B0B029C
:10E61000130C1C006FF04F938327C1002320F700D9
:10E620006FF00F8893076000138D0A0063EC570B9F
:10E63000375E0180930C0D002328B10113040E32C4
:10E640006FF08F9793770B20638807108327010162
:10E65000930C00002328D10003CD07006FF01FE8C2
:10E6600093770B20638E070C832701012328E10099
:10E67000038D0700935CFD4113870C006FF08FB68C
:10E6800093F70D206382070A83270101930C000092
:10E690002328E10003CD0700130710006FF04FC1DE
:10E6A00093770B206388070683270101930C0000F2
:10E6B0002328E10003CD07006FF00FBF938506000C
:10E6C0006FF05F8D93079000E3E237CF6FF0DFD2FA
:10E6D000930641051306100013070000938B0400F6
:10E6E0006FF00F9B130D60006FF09FF49307B10361
:10E6F0002326F104930710002328F10413061000C9
:10E70000930641056FF08F918327C1002310F70016
:10E710006FE01FF983270101930C00002328E1001B
:10E7200003AD07006FF04FB883270101930C000081
:10E730002328E10003AD0700130710006FF04FB767
:10E74000832701012328E10003AD0700935CFD410D
:10E7500013870C006FF00FA983270101930C0000B1
:10E760002328D10003AD07006FF05FD71306010423
:10E770009385090013050A00EFE01FD26FF00F9A8E
:10E78000138D0A002328B101930A00006FF04FA9EE
:10E79000938506006FF0DF99930516006FF01FA7B1
:10E7A000930D0B006FF08FA69307F0FF2326F10067
:10E7B0006FF08F9713850600930506006FF0CFF07A
:10E7C0008327010183AA07009387470063D40A00C7
:10E7D000930AF0FF03471C002328F100138C060066
:10E7E0006FE09FF69307050003A5C11C9306060082
:10E7F00013860500938507006FE09FDA83D7C50075
:10E8000003AE450603D3E50083A8C50103A845026E
:10E81000130101B893F7D7FF13070040232C81465B
:10E82000231AF10013840500930701079305810063
:10E83000232A914623282147232E11461309050038
:10E840002326C107231B6100232211032326010372
:10E850002324F100232CF1002328E100232EE100E2
:10E8600023200102EFE0DFD393040500635C05027F
:10E870008357410193F70704638807008357C40057
:10E8800093E707042316F4008320C147032481473C
:10E8900003290147138504008324414713010148DC
:10E8A000678000009305810013050900EF20DF93C6
:10E8B000E30005FC9304F0FF6FF09FFB03A301113D
:10E8C00067000300638405029307F00F63E8C70045
:10E8D0002380C50013051000678000009307A0087F
:10E8E0002320F5001305F0FF6780000013050000EA
:10E8F00067800000B385C502130101FF2324810056
:10E9000023261100EF309FF313040500630805026E
:10E910000326C5FF130740021376C6FF1306C6FF82
:10E920006360C706930630019307050063E2C602E1
:10E9300023A0070023A2070023A407008320C1000F
:10E940001305040003248100130101016780000006
:10E9500023200500232205009307B00163F0C704BC
:10E96000232405002326050093070501E312E6FC96
:10E970002328050093078501232A05006FF05FFB1C
:10E9800093050000EF40CFF68320C100130504007B
:10E9900003248100130101016780000093078500B3
:10E9A0006FF01FF9130101FD23248102232E310191
:10E9B000232861012326110223229102232021030F
:10E9C000232C4101232A5101130B050093890500D3
:10E9D00013040600EFA0DFA9930710006310F502EF
:10E9E0009387F9FF1307E00F636AF70013F7F90F36
:10E9F0002306E100130910006F00C0029306C4054E
:10EA0000138609009305C10013050B00EF20800B4E
:10EA10009307F0FF130905006304F50A630E050868
:10EA20000347C10093040000130AF0FF930AA000FB
:10EA30006F00800283270400938617002320D400F0
:10EA40002380E700938414009307C100B3879700E5
:10EA500063F4240703C70700832784009387F7FF25
:10EA60002324F400E3D807FC8326840193050700E0
:10EA70001306040013050B0063C4D700E31C57FB07
:10EA8000EF10D06AE31045FD1309F0FF8320C102A7
:10EA900003248102832441028329C101032A8101C5
:10EAA000832A4101032B01011305090003290102F7
:10EAB0001301010367800000138909006FF01FFD37
:10EAC0008357C40093E707042316F4006FF01FFC7C
:10EAD0008317C600139727016340070203274606E2
:10EAE000B7260000B3E7D700B72600003367D7008A
:10EAF0002316F6002322E6066FF0DFEA130101FE7B
:10EB0000232C810003A4C11C232E110013860500B1
:10EB100093050500630604008327840363800704CC
:10EB20008317C60013972701634007020327460691
:10EB3000B7260000B3E7D700B72600003367D70039
:10EB40002316F6002322E6061305040003248101A0
:10EB50008320C101130101026FF0DFE42324A1002F
:10EB6000130504002326C100EF20DFA10326C10006
:10EB7000832581006FF0DFFA83278600638E0732DA
:10EB800083D7C500130101FD23248102232C4101F9
:10EB9000232A51012326110223229102232021033B
:10EBA000232E3101232861012326710123248101B1
:10EBB000232291012320A10113F78700130A0600E5
:10EBC000930A0500138405006306070803A70501DF
:10EBD0006302070813F7270083240A00630C070861
:10EBE000832744028325C401370B0080930900006A
:10EBF00013090000134B0BC01386090013850A008C
:10EC0000630209049306090063742B0193060B0049
:10EC1000E78007006358A02883278A00B389A900EA
:10EC20003309A9403385A7402324AA00630A05209D
:10EC3000832744028325C4011386090013850A0033
:10EC4000E31209FC83A9040003A94400938484000F
:10EC50006FF09FFA9305040013850A00EF704FF9D7
:10EC6000631C053A8357C40083240A0013F7270066
:10EC7000E31807F613F7170063140724832C8400A6
:10EC800003250400370B0080934BEBFF130C0000AF
:10EC900013090000134BFBFF630E090E13F7072047
:10ECA000630C0724138D0C006362992F13F7074838
:10ECB000630A070883294401832504011307190007
:10ECC00093961900B386360193D9F601330DB540FA
:10ECD000B389D90093D919403307A70113860900D6
:10ECE00063F6E900930907001306070093F707404E
:10ECF0006384072E9305060013850A00EF301FB4C6
:10ED0000930C0500630205308325040113060D00F2
:10ED1000EF404FAC8357C40093F7F7B793E707086A
:10ED20002316F4003385AC01B387A941232894014D
:10ED30002320A400232A3401930C09002324F40087
:10ED4000130D090013060D0093050C00EF00402D74
:10ED5000032784008327040093090900B30C97411B
:10ED6000B387A701232494012320F4001309000092
:10ED700003268A00330C3C01B309364123243A01AF
:10ED80006380090C832C8400032504008357C4008E
:10ED9000E31609F003AC040003A944009384840043
:10EDA0006FF09FEF83A9440003AC040093848400B8
:10EDB000E38A09FE138609009305A00013050C00E1
:10EDC000EFA04FFA6304051213051500330B8541BC
:10EDD00093070B00938B090063F43701938B0700B3
:10EDE00003250400832704018326440163F8A70058
:10EDF00003298400338926016342790963C8DB1A39
:10EE0000832744028325C40113060C0013850A00DE
:10EE1000E7800700130905006356A008330B2B4158
:10EE200013051000630A0B1603268A00330C2C010D
:10EE3000B38929413309264123242A01631A090889
:10EE4000130500008320C1020324810283244102B0
:10EE5000032901028329C101032A8101832A410177
:10EE6000032B0101832BC100032C8100832C410063
:10EE7000032D0100130101036780000093050C00BE
:10EE800013060900EF00C01983270400930504004E
:10EE900013850A00B38727012320F400EF20CFB4A5
:10EEA000E30E05F68317C40093E707042316F40066
:10EEB0001305F0FF6FF01FF91305000067800000D5
:10EEC000130B000013050000130C00009309000051
:10EED000E38A09ECE31E05EE138609009305A00002
:10EEE00013050C00EFA00FE8E31005EE938719005F
:10EEF000138B07006FF01FEE8327040163E2A70462
:10EF000083274401636EF9029306090063F42B0121
:10EF100093060B00B3C6F602032744028325C401FF
:10EF200013060C0013850A00B386F602E7000700FB
:10EF300093090500E358A0F6330939416FF05FE308
:10EF400093890C00637499019309090013860900E1
:10EF500093050C00EF00C00C8327840003270400F6
:10EF6000B3873741330737012324F4002320E4001B
:10EF7000E39407FC9305040013850A00EF20CFA655
:10EF8000E31205F2330939416FF09FDE930C09005B
:10EF9000130D09006FF01FDB9305040013850A00B1
:10EFA000EF208FA4E30205E86FF0DFEF13860B007C
:10EFB00093050C00EF00C00683278400032604009D
:10EFC00013890B00B3877741330676012324F400BD
:10EFD0002320C4006FF09FE413850A00EF00401661
:10EFE000930C0500E31005D48325040113850A0062
:10EFF000EF209FB18317C4001307C00023A0EA00CD
:10F0000093F7F7F76FF05FEA1307C0008317C400A8
:10F0100023A0EA006FF05FE91305F0FF6FF09FE2B5
:10F0200063F6A502B387C5006372F5023307C50016
:10F03000630A060E83C6F7FF9387F7FF1307F7FFF0
:10F040002300D700E398F5FE678000009307F000E7
:10F0500063E8C702930705009306F6FF630C060CEE
:10F0600093861600B386D70003C705009387170061
:10F0700093851500A38FE7FEE398D7FE6780000015
:10F08000B3E7A50093F737006390070A930806FFDC
:10F0900093F808FF938808013308150113870500CA
:10F0A00093070500832607001307070193870701CD
:10F0B00023A8D7FE832647FF23AAD7FE832687FFF0
:10F0C00023ACD7FE8326C7FF23AED7FEE31CF8FC94
:10F0D0001377C600B38515011378F600630E070495
:10F0E0001387050093880700130E300003230700E1
:10F0F00013074700B306E84023A06800B386D50095
:10F1000093884800E364DEFE1307C8FF1377C7FF48
:10F110001307470013763600B387E700B385E50091
:10F120006FF09FF3678000009306F6FF93070500DA
:10F130006FF01FF367800000130608006FF0DFF127
:10F14000130101FD23202103232611022324810220
:10F1500023229102232E3101232C4101232A510124
:10F16000232861012326710123248101130906004C
:10F17000638205221384050093090500EF400F8583
:10F180009304B9009307600163FC970E93F484FF26
:10F190001387040063CC040E63EA240F8327C4FFA3
:10F1A000930A84FF13FAC7FF338B4A01635AEA18A4
:10F1B000938B81C203A68B0083264B00630E6623CC
:10F1C00013F6E6FF3306CB0003264600137616003F
:10F1D0006314061A93F6C6FF3306DA00635EE6325E
:10F1E00093F7170063940702032C84FF338C8A4142
:10F1F00083274C0093F7C7FFB386D700B38B460134
:10F2000063DAEB34B30BFA0063D2EB0C930509001D
:10F2100013850900EF308FE213090500630C050424
:10F220008327C4FF130785FF93F7E7FFB387FA002F
:10F230006382E7301306CAFF9307400263E6C730D4
:10F240001307300183260400636CC726930705006B
:10F250001307040023A0D7008326470023A2D7006A
:10F260000327870023A4E700930504001385090002
:10F27000EF209F8913850900EF309FF56F00C001D3
:10F280009304000113070001E3FA24F19307C0007F
:10F2900023A0F900130900008320C1020324810286
:10F2A000832441028329C101032A8101832A410168
:10F2B000032B0101832BC100032C810013050900DE
:10F2C0000329010213010103678000008327CC009A
:10F2D00003278C001306CAFF930640022326F7007B
:10F2E00023A4E70013098C00330B7C0163E4C62ED2
:10F2F00093053001032704009307090063F2C50258
:10F300002324EC00032744009307B0012326EC00DC
:10F3100063E2C7300327840093070C0113048400C1
:10F3200023A0E70003274400138A0B00930A0C0074
:10F3300023A2E700032784001304090023A4E700A5
:10F3400083A74A0033079A409306F00093F717000B
:10F3500063ECE606B367FA0023A2FA0083274B00AA
:10F3600093E717002322FB0013850900EF305FE6C7
:10F37000130904006FF05FF293F71700E39807E8B2
:10F38000032C84FF338C8A4183274C0093F7C7FFFB
:10F390006FF05FE7032481028320C10283244102CE
:10F3A000032901028329C101032A8101832A410122
:10F3B000032B0101832BC100032C81009305060060
:10F3C000130101036F308FC7B3E7970023A2FA0040
:10F3D000B3859A001367170023A2E50083274B002B
:10F3E000938585001385090093E717002322FB000E
:10F3F000EF208FF16FF05FF793F6C6FF3306DA0068
:10F40000938504016350B60E93F71700E39007E06D
:10F41000032C84FF338C8A4183274C0093F7C7FF6A
:10F42000B386D700338B4601E34EBBDC8327CC0089
:10F4300003278C001306CAFF930640022326F70019
:10F4400023A4E70013098C0063EEC6209305300166
:10F45000032704009307090063F2C5022324EC008C
:10F46000032744009307B0012326EC0063E4C72080
:10F470000327840093070C011304840023A0E700F2
:10F480000327440023A2E7000327840023A4E70006
:10F4900033079C00B3079B4023A4EB0093E71700BE
:10F4A0002322F70083274C001385090093F71700E8
:10F4B000B3E4970023229C00EF309FD16FF0DFDD93
:10F4C0002320D500832644001307B0012322D50052
:10F4D0006360C712832684001307840093078500A6
:10F4E0006FF05FD7B38A9A00B307964023A45B01FD
:10F4F00093E7170023A2FA008327C4FF13850900AE
:10F500001309040093F71700B3E49700232E94FE29
:10F51000EF301FCC6FF05FD88327CB0003278B0021
:10F52000130A0600338BCA002326F70023A4E70042
:10F530006FF01FE18327C5FF93F7C7FF330AFA0077
:10F54000338B4A016FF0DFDF93050400EFF05FAD0E
:10F550006FF09FD18327CB0003278B001306CAFFD0
:10F56000930640022326F70023A4E70003278C001C
:10F570008327CC0013098C00330B7C012326F70072
:10F5800023A4E70063E8C6049306300103270400C0
:10F5900093070900E3F6C6D82324EC0003274400B0
:10F5A0009307B0012326EC0003278400E3F6C7D6B7
:10F5B0002328EC000327C40093074002232AEC0011
:10F5C000032704016304F60693078C011304040166
:10F5D0006FF01FD59305040013050900EFF05FA439
:10F5E00013040900138A0B00930A0C006FF05FD517
:10F5F000032784002324E5000327C4002326E50015
:10F60000832604016302F60413070401930705012E
:10F610006FF05FC4832784002328FC008327C40085
:10F62000232AFC0003270401E310D6FA232CEC0064
:10F630000327440193070C0213048401232EEC00DA
:10F64000032704006FF0DFCD2328D5008326440173
:10F650001307840193078501232AD500832684019B
:10F660006FF05FBF9305040013050900EFF05F9B87
:10F670006FF01FE2832784002328FC008327C40047
:10F68000232AFC00032704016308D60093078C019A
:10F69000130404016FF09FDE232CEC0003274401C8
:10F6A00093070C0213048401232EEC0003270400AB
:10F6B0006FF0DFDC83278600130101FD232A51014F
:10F6C00023261102232481022322910223202103D5
:10F6D000232E3101232C41012328610123267101AE
:10F6E00023248101930A060063880714130B050085
:10F6F0008329060003A5050083A485001384050063
:10F700006F00400D8357C40013F70748630A0708CA
:10F7100083264401832504011307190093941600DE
:10F72000B386D40093D4F601330AB540B384D40031
:10F7300093D41440330747011386040063F6E400B2
:10F74000930407001306070093F707406386070A30
:10F750009305060013050B00EF304F8E130C0500C8
:10F76000630A050A8325040113060A00EF309F8609
:10F770008357C40093F7F7B793E707082316F400FD
:10F7800033054C01338A4441232A94002324440145
:10F79000232884012320A40093040900130A0900EC
:10F7A00013060A0093850B00EFF09F870327840060
:10F7B0000325040083A78A00B3049740330545015D
:10F7C000232494002320A4003389274123A42A0161
:10F7D0006304090603A9490083AB0900138A0400E6
:10F7E00093898900E30809FEE37E99F093040900F8
:10F7F000130A09006FF0DFFA13050B00EFF05F94B6
:10F80000130C0500E31E05F68325040113050B0008
:10F81000EF208FAF9307C0002320FB008357C40065
:10F820001305F0FF93E707042316F40023A40A004E
:10F8300023A20A006F00C00023A20A0013050000E3
:10F840008320C1020324810283244102032901028F
:10F850008329C101032A8101832A4101032B01016C
:10F86000832BC100032C810013010103678000007A
:10F8700083D7C500130101ED232C41112328611109
:10F880002320A11123261112232481122322911255
:10F8900023202113232E3111232A511123267111E4
:10F8A0002324811123229111232EB10F93F70708EE
:10F8B0002326D100138A0500130B0500130D060043
:10F8C0006386070083A70501E384075EB7670180AD
:10F8D000930AC1049387C7C8B76B0180B7640180DE
:10F8E00093090D0023205105232401042322010440
:10F8F000232A0100232C010023200102232E0100D2
:10F90000232401002328F100938B8BDF938484E070
:10F91000138D0A0083C70900638C07201384090034
:10F92000930650026388D72A8347140013041400F7
:10F93000E39A07FE330C3441630C341F83268104A1
:10F940008327410423203D01B38686019387170056
:10F9500023228D012324D1042322F1049306700075
:10F96000130D8D0063C0F628032781008347040030
:10F97000330787012324E100638C071A9308F0FF03
:10F980008346140093091400A30D010223220100F1
:10F9900013090000130CA005930C90009305A0021E
:10F9A0001384080093891900938706FE6368FC049A
:10F9B0000327010193972700B387E70083A7070078
:10F9C0006780070023220100938706FD032641007C
:10F9D00083C6090093891900131726003307C7004F
:10F9E00013171700B387E7002322F100938706FD62
:10F9F000E3FEFCFC938706FEE37CFCFA638A0612B6
:10FA00002306D108A30D0102130C1000930C100063
:10FA10001304C10893080000137F290063040F003A
:10FA2000130C2C00937E490883278104032641048C
:10FA300063980E0003274100B30D8741634AB07BF2
:10FA40000345B1039305160093068D00630005047A
:10FA50001305B103938717002320AD001305100091
:10FA60002322AD002324F1042322B10413057000E6
:10FA7000E340B50A930F260013050D011386050018
:10FA8000138D060093850F0093060500630C0F028B
:10FA90001306C103938727002320CD0013062000FF
:10FAA0002322CD002324F1042322B1041307700084
:10FAB000E342B70A13860500138D060093851500EF
:10FAC0009386860013050008638CAE54B38D98416D
:10FAD0006344B063B387FC0023208D0023229D0183
:10FAE0002324F1042322B104130770006342B76C8E
:10FAF000137349006308030003274100B30C8741D7
:10FB0000E3489009032441006354840113040C006A
:10FB100003278100330787002324E100639A076AE3
:10FB200083C7090023220104138D0A00E39807DE2E
:10FB300083278104E39E07568357CA0093F707047F
:10FB4000E394075A8320C112032481120325810004
:10FB500083244112032901128329C111032A81112F
:10FB6000832A4111032B0111832BC110032C811017
:10FB7000832C4110032D0110832DC10F130101139C
:10FB80006780000013050B00EF90DF858327450099
:10FB900013850700232EF100EFA09FDB93070500DC
:10FBA00013050B00938D07002320F102EF909F8334
:10FBB000832785009305A002232CF100E3980D1EF6
:10FBC00083C609006FF01FDE83C6090013690902AE
:10FBD0006FF05FDD330C3441E31234D78347040008
:10FBE0006FF09FD91306010493050A0013050B005B
:10FBF000EFF05FACE31205F4138D0A006FF0DFD66F
:10FC00008327C10093080400A30D010203A4070089
:10FC1000938D4700E30404389307F0FFE38EF82642
:10FC20001386080093050000130504002326110124
:10FC3000EF905F938328C100E3060548B30C85402D
:10FC40002326B101930800006F0040090327C1007B
:10FC5000A30D0102130C10008327070013074700B0
:10FC60002326E1002306F108930C10001304C108B9
:10FC70006FF05FDA9377090293080400638E070E32
:10FC80008327C1009387770093F787FF83A64700F8
:10FC900083AC0700938787002326F100138C0600AE
:10FCA00063C406109306F0FF930D09006388D80023
:10FCB000B3E68C01937DF9F7638E0676E31C0C00A6
:10FCC00093069000E3E8960193870C03A307F10ED7
:10FCD00013890D00930C10001304F10E138C08000F
:10FCE00063D49801138C0C008347B103B337F00041
:10FCF000330CFC006FF05FD2930804001369090114
:10FD000093770902638407748327C1009387770080
:10FD100093F787FF83AC070003AC47009387870006
:10FD20002326F100937DF9BF93060000A30D010285
:10FD30001306F0FF638EC80833E68C0113F9FDF754
:10FD40006314064A63920828639A066E93FC1D00AA
:10FD50001304010FE3840CF893070003A307F10ECB
:10FD60001304F10E6FF09FF71369090193770902ED
:10FD700093080400E39607F00327C1009377090175
:10FD800093064700E392070493770904E386072666
:10FD90008327C1002326D100839C070013DCFC418C
:10FDA00093060C00E3D006F0B3369001B30E804109
:10FDB000338CDE409306D002A30DD1021306F0FF70
:10FDC000B30C9041930D090093061000E396C8F61A
:10FDD00013061000E384C6EE130620006380C620DD
:10FDE0001304010F9317DC0193F67C0093DC3C00B5
:10FDF00093860603B3EC9701135C3C00A30FD4FE7B
:10FE0000B3E78C01930504001304F4FFE39C07FCA3
:10FE100093F71D00638E071E93070003638AF61E87
:10FE20009385E5FFA30FF4FE9307010FB38CB74052
:10FE300013890D00138405006FF05FEA9308040036
:10FE4000936D090193F70D02638807628327C10050
:10FE50009306100013897700137989FF93078900AF
:10FE6000832C0900032C49002326F1006FF01FECBE
:10FE70008327C100B786FFFF93C6068383AC0700C4
:10FE8000938747002326F100B75701809387872F78
:10FE9000231ED10293080400130C0000936D290067
:10FEA000232AF100930620006FF05FE883C6090063
:10FEB000136909086FF01FAF83C609001387190083
:10FEC000E38AB622938706FD930907001304000016
:10FED000E3ECFCAC83C6090013172400B3088700C9
:10FEE000939818003384F800938706FD93891900CE
:10FEF000E3F2FCFE6FF05FAB83C6090013694900B3
:10FF00006FF05FAA9307B00283C60900A30DF10248
:10FF10006FF05FA90327C10083C60900832707008C
:10FF2000130747002326E1002322F100E3DC07A6A4
:10FF3000B307F0402322F100136949006FF09FA638
:10FF400083C60900136919006FF0DFA58347B10369
:10FF500083C60900E39807A493070002A30DF102EA
:10FF60006FF05FA483C6090093078006638EF67E58
:10FF7000136909046FF01FA30327C10093770902D7
:10FF800083260700130747002326E100639C075ED2
:10FF900093770901639E077E93770904E394071022
:10FFA000137309206306037E832781002380F600F4
:10FFB0006FF05F9683C609009307C006638EF67ADA
:10FFC000136909016FF01F9E13061000E384C61029
:10FFD00013062000930D0900E394C6E08326410137
:10FFE0001304010F93F7FC00B387F60003C7070063
:10FFF00093DC4C009317CC01B3EC9701135C4C00DD
:02000004800179
:10000000A30FE4FEB3E78C011304F4FFE39C07FCA9
:100010009307010FB38C874013890D006FF01FCC3D
:1000200003274100B30D8741E352B0AB1305000134
:10003000E356B50B232281029306000113040A0044
:10004000930E7000138A0D00938D090093890800A8
:100050006F00C000130A0AFF63DA460593870701A1
:100060001306160023209D002322DD002324F10423
:100070002322C104130D8D00E3DECEFC1306010420
:100080009305040013050B00EFF0CFE2631E056E2D
:1000900093060001130A0AFF832781040326410403
:1000A000138D0A00930E7000E3CA46FB9388090083
:1000B00093890D00930D0A00130A040003244102E2
:1000C0001306160013058D00B387B70123209D008A
:1000D0002322BD012324F1042322C104130770004D
:1000E000634AC764B38D9841930516009306850053
:1000F000130D0500E350B09F13050001635EB57357
:1001000093060001930870006F00C000938D0DFFEF
:1001100063DAB605938707011306160023209D00B6
:100120002322DD002324F1042322C104130D8D00BA
:10013000E3DEC8FC1306010493050A0013050B0057
:10014000EFF04FD7E31A059E93060001938D0DFF44
:100150008327810403264104138D0A00930870004D
:10016000E3CAB6FB9305160013068D00B387B701EB
:1001700023209D002322BD012324F1042322B10466
:10018000130770006342B732130D06009385150004
:10019000B387FC0023208D0023229D012324F1043A
:1001A0002322B1041307700093068600E352B7942C
:1001B0001306010493050A0013050B00EFF08FCF1F
:1001C000E31C05968327810493860A006FF05F92F3
:1001D0001306010493050A0013050B00EFF08FCD01
:1001E000E30005946FF05F95930D09006FF05FBE1B
:1001F0009306000163DEB60B13070D00930F70002A
:10020000130D0C002322E103130C09002324D10356
:1002100013090A00138A09009309040013840D00CE
:10022000938D0C00938C08006F00C000130404FF32
:1002300063DA8604938707011306160023207701EB
:100240002322D7002324F1042322C10413078700AB
:10025000E3DECFFC130601049305090013050B0030
:10026000EFF04FC56316054A93060001130404FF1F
:10027000832781040326410413870A00930F70002B
:10028000E3CA86FA032F4102832E810293880C0071
:10029000938C0D00930D04001384090093090A0048
:1002A000130A090013090C00130C0D00130D0700AD
:1002B000B387B7011306160023207D012322BD0159
:1002C0002324F1042322C10493067000130D8D0032
:1002D00063D8C6F61306010493050A0013050B0044
:1002E000232611032324D1032322E103EFF08FBC43
:1002F000E314058483278104032641048328C10273
:10030000832E8102032F4102138D0A006FF04FF3F9
:100310001306010493050A0013050B00232611039D
:100320002324D1032322E103EFF0CFB8E3160580A5
:1003300003264104832781048328C102832E81027E
:10034000032F41029306410593051600138D0A0001
:100350006FF0CFF31306010493050A0013050B0099
:10036000232411032322D103EFF0CFB4631605FC3D
:10037000032641048327810483288102832E4102BE
:100380009306410593051600138D0A006FF08FF355
:10039000130600010327410463509607930D0001E3
:1003A000130470006F00C000938C0CFF63D69D0592
:1003B000938707011307170023A0760123A2B60134
:1003C0002324F1042322E10493868600E35EE4FC07
:1003D0001306010493050A0013050B00EFF08FAD1F
:1003E000631C05F4938C0CFF8327810403274104CD
:1003F00093860A00E3CE9DFBB3879701130717008E
:1004000023A0760123A296012324F1042322E104F0
:100410009306700063D8E6EE1306010493050A0004
:1004200013050B00EFF00FA9631805F08327810473
:100430006FF04FEDE39A088813890D0093080000D0
:10044000930C00001304010F6FF05F890327C100B4
:10045000937709019306470063920718937709047D
:10046000638E07368327C100130C00002326D100BA
:1004700083DC07006FF01F8B0327C10093F70D018A
:1004800093064700639A071093F70D0463860738B5
:100490008327C100130C00002326D10083DC070052
:1004A000930610006FF09F881306010493050A005D
:1004B00013050B00EFF00FA0631005E8832541043E
:1004C000832781049306410593851500138D0A0047
:1004D0006FF04FE093F70D402324410323263103AF
:1004E000130A0C0093890C0013090000832C81016E
:1004F0001304010F23221103138C07006F00400225
:100500001306A000930600001385090093050A0056
:10051000EF00406B63060A3293090500138A050059
:100520001306A000930600001385090093050A0036
:10053000EF00902C13050503A30FA4FE1309190067
:100540001304F4FFE30E0CFA83C60C00E39A26FBB7
:100550009307F00FE306F9FA631C0A16930790005D
:1005600063E837179307010F232C91018328410279
:10057000032A81028329C102B38C874013890D00AD
:100580006FF0CFF5032781009357F74123A0E600D2
:1005900023A2F6006FF00FB82326D100832C0700AA
:1005A000130C0000930610006FF04FF883278101B1
:1005B00083C60900638807BE83C70700638407BE3C
:1005C000136909406FF00FBE832C07002326D1006A
:1005D00013DCFC4193060C006FF08FEC832C0700BA
:1005E000130C00002326D1006FF0CFF3B757018022
:1005F0009387C730232AF1009377090293080400F8
:10060000638C07068327C1009387770093F787FFE2
:1006100083AC070003AC4700938787002326F100D3
:1006200013761900630E060033E68C01630A060098
:1006300013060003230EC102A30ED1021369290081
:10064000937DF9BF930620006FF04FEE93080400EE
:10065000930D09006FF00FFF930804006FF04FEA4D
:10066000B75701809387872F232AF10093770902D8
:1006700093080400E39807F80327C1009377090162
:1006800013064700638A0708832C0700130C000039
:100690002326C1006FF0DFF813050400EFA04FAB75
:1006A000930C05002326B101930800006FF00FE3BF
:1006B00093050004EF208F982320AA002328AA0086
:1006C000630C052493070004232AFA006FF00FA09F
:1006D000832701028325C101130900003304F4407C
:1006E0001386070013050400EFA04FAF83C51C005D
:1006F0001306A000930600003338B00013850900EC
:1007000093050A00B38C0C01EF00C04B6FF0DFE0E3
:10071000130A09006FF04FC2937709046382070A36
:100720008327C100130C00002326C10083DC0700CF
:100730006FF01FEF1306010493050A0013050B0069
:1007400023221103EFE01FF7631805BE03264104BF
:1007500083278104832841029306410593051600EF
:10076000138D0A006FF08FB683C619001369092034
:10077000938919006FF00FA383C61900136909024A
:10078000938919006FF00FA2130A04006FF0CFBA1B
:100790008327810023A0F6006FF0CF9793076000B6
:1007A000938C080063F41701930C6000375E01809E
:1007B000138C0C002326B10113040E326FF08FA5A9
:1007C000937709206386070C8327C100130C000070
:1007D0002326C10083CC07006FF09FE493770920A4
:1007E000638E07088327C100130C00002326D10065
:1007F00083CC07006FF00FD393770920638407063B
:100800008327C1002326D100838C070013DCFC4121
:1008100093060C006FF0CFC893F70D206388070292
:100820008327C100130C00002326D10083CC0700CE
:10083000930610006FF08FCF138606006FF01F93A2
:1008400093079000E3EA37CD6FF0DFD18327C10033
:10085000130C00002326D10083AC07009306100080
:100860006FF0CFCC8327C1002326D10083AC0700D3
:1008700013DCFC4193060C006FF08FC28327C1008C
:10088000130C00002326D10083AC07006FF08FC942
:100890008327C100130C00002326C10083AC07008E
:1008A0006FF01FD8832781002390F6006FF08F86AA
:1008B0001306010493050A0013050B00EFE09FDF08
:1008C0006FF08FA7938C08002326B10193080000D6
:1008D0006FF0CFC0930D09006FF00FBF13850600B6
:1008E000138605006FF04FFE9307F0FF2324F100FD
:1008F0006FF04FA58327C10003A40700938747002B
:10090000635404001304F0FF83C619002326F1008A
:10091000930907006FF00F899307C0002320FB00A5
:100920009307F0FF2324F1006FF0CFA1130101FE24
:10093000232C8100232A910023282101232E11003A
:1009400023263101130905009384050013040600D2
:100950006306050083278503638807140317C40013
:1009600083268401937787002324D40093160701FC
:1009700093D606016382070883270401638E070666
:100980001396260193F9F40F93F4F40F635E0608AF
:100990000327040083264401B307F74063DED70A28
:1009A00083268400130617002320C4009386F6FFD5
:1009B0002324D40023003701032744019387170021
:1009C0006308F70C8357C40093F71700638607008A
:1009D0009307A000638EF40A8320C10103248101E0
:1009E000032901018329C1001385040083244101E7
:1009F000130101026780000093050400130509003C
:100A0000EF501F9F631E05080317C40093F9F40FEE
:100A1000832704019316070193D606011396260136
:100A200093F4F40FE34606F68326440637260000C7
:100A30003367C70037E6FFFF1306F6FFB3F6C600BD
:100A40002316E400032704002322D406832644014E
:100A5000B307F740E3C6D7F4930504001305090074
:100A6000EF008FF8631E050203270400832684002D
:100A700093071000130617009386F6FF2320C40087
:100A80002324D4002300370103274401E31CF7F299
:100A90009305040013050900EF000FF5E30E05F2BE
:100AA0009304F0FF6FF05FF3EF00DFAD6FF01FEB2B
:100AB0009307050003A5C11C138605009385070055
:100AC0006FF0DFE6130101FE232C8100232A910041
:100AD000232E110083A7011113040500938406003F
:100AE00063820502E78007009307F0FF6306F502C3
:100AF0008320C101032481018324410113010102E8
:100B0000678000001306000093054100E78007009E
:100B10009307F0FFE31EF5FC23A004009307A00851
:100B20008320C1012320F400032481018324410197
:100B30001301010267800000130101FE232C8100D4
:100B4000232A9100232E110083A4C11C83A7011125
:100B500013040600630A05021386050093060400C9
:100B60009305050013850400E78007009307F0FF55
:100B7000630AF5028320C10103248101832441011A
:100B800013010102678000009306060093054100EF
:100B90001306000013850400E78007009307F0FFA9
:100BA000E31AF5FC232004008320C1010324810102
:100BB0009307A00823A0F40083244101130101023C
:100BC000678000009308050093870500130806005E
:100BD000138506001383080063940628B766018016
:100BE0009386C6EC63F6C50E370701006378E60C02
:100BF0001307F00F3337C700131737003355E600DC
:100C0000B386A60083C60600130500023387E600FC
:100C1000B306E540630CE500B397D70033D7E8008F
:100C20003318D600B365F7003393D8009358080102
:100C3000B3D7150313160801135606011357030102
:100C4000B3F6150313850700B305F6029396060164
:100C500033E7E600637EB700330707011385F7FF2C
:100C6000636807016376B7001385E7FF3307070161
:100C70003307B740B377170313130301135303016B
:100C8000335717039397070133E36700B306E60270
:100C900013060700637CD300330368001306F7FFD5
:100CA000636603016374D3001306E7FF13150501A0
:100CB0003365C500930500006F00400E3705000145
:100CC00013070001E36CA6F2130780016FF01FF316
:100CD00063160600130710003358C70237070100D8
:100CE0006370E80C1307F00F6374070113058000AD
:100CF0003357A800B386E60003C7060013060002B8
:100D00003307A700B306E6406316E60AB387074138
:100D10009305100093580801131608011356060195
:100D200013570301B3F61703B3D7170393960601BE
:100D300033E7E600330EF60213850700637EC70132
:100D4000330707011385F7FF636807016376C7015F
:100D50001385E7FF330707013307C741B37717034D
:100D60001313030113530301335717039397070119
:100D700033E36700B306E60213060700637CD30083
:100D8000330368001306F7FF636603016374D3003F
:100D90001306E7FF131505013365C50067800000E2
:100DA0003707000113050001E364E8F4130580012F
:100DB0006FF01FF43318D800B3D5E7003393D80091
:100DC000B397D70033D7E800935808013366F7008C
:100DD00033F715039317080193D70701135506013D
:100DE000B3D51503131707013367A700B386B702FE
:100DF00013850500637ED700330707011385F5FFD0
:100E0000636807016376D7001385E5FF33070701A1
:100E1000B306D74033F7160313160601135606011F
:100E2000B3D6160313170701B388D702B367C700F9
:100E30001387060063FE1701B38707011387F6FFC8
:100E400063E8070163F617011387E6FFB38707011D
:100E500093150501B3871741B3E5E5006FF09FEBEC
:100E600063E6D5183707010063F4E6041307F00FB3
:100E7000B335D700939535003767018033D5B60079
:100E80001307C7EC3307A700034707001305000249
:100E90003307B700B305E5406316E50213051000FC
:100EA000E3EEF6EE33B5C800134515006FF01FEF03
:100EB0003707000193050001E3E0E6FC930580019C
:100EC0006FF09FFB3353E600B396B6003363D30055
:100ED00013550301B31EB60033D6E700B376A6025E
:100EE000B397B70033D7E8003368F70093170301CF
:100EF00093D70701135708013356A60293960601AC
:100F000033E7E600338FC702130E0600637EE70166
:100F100033076700130EF6FF636867006376E70127
:100F2000130EE6FF330767003307E741B376A702E6
:100F30003357A702939606013386E70293170801F9
:100F400093D70701B3E7F6009306070063FEC700D7
:100F5000B38767009306F7FF63E8670063F6C7008F
:100F60009306E7FFB387670013150E01370E0100E4
:100F70003365D5009306FEFF3378D500B387C740AD
:100F8000B3F6DE001356050193DE0E013303D802DB
:100F9000B306D602135703013308D8033308D80029
:100FA000330707013306D6036374D7003306C6013F
:100FB000935607013386C60063E6C702E39CC7CE9B
:100FC000B70701009387F7FF3377F700131707017F
:100FD0003373F300B398B80033076700930500003C
:100FE000E3FEE8DA1305F5FF6FF0DFCC93050000B0
:100FF000130500006FF09FDA9308060013870600C0
:101000009307050013880500639C0622B7660180DC
:101010009386C6EC63FCC50C37030100637E660A49
:101020001303F00F6374C300130780003353E6000B
:10103000B386660003CE0600330EEE0013070002EF
:101040003303C741630CC701B3956500335EC50127
:10105000B31866003368BE00B317650013D60801E5
:101060003377C802139508011355050193D607017C
:101070003358C80213170701B366D70033080503B6
:1010800063FA0601B386160163E6160163F40601EE
:10109000B3861601B386064133F7C602939707015C
:1010A00093D70701B3D6C602B306D50213150701BD
:1010B000B367F50063FAD700B387170163E617013A
:1010C00063F4D700B3871701B387D74033D56700E0
:1010D000930500006780000037030001130700013B
:1010E000E36666F4130780016FF05FF46316060091
:1010F00013061000B35816033706010063F2C80A3E
:101100001306F00F637416011307800033D6E8004E
:10111000B386C60003CE0600330EEE0013070002AE
:101120003303C7416318C709B385154113D70801B5
:10113000139508011355050113D60701B3F6E5020F
:10114000B3D5E50293960601B3E6C600B305B50232
:1011500063FAB600B386160163E6160163F4B600BF
:10116000B3861601B385B640B3F6E502939707013F
:1011700093D70701B3D5E502B305B5021395060170
:10118000B367F50063FAB700B387170163E6170189
:1011900063F4B700B3871701B387B7406FF01FF34D
:1011A0003706000113070001E3E2C8F613078001C8
:1011B0006FF0DFF5B398680033D7C501B31765004A
:1011C000335EC50113D50801B376A702B395650058
:1011D000336EBE009395080193D5050113560E0199
:1011E0003357A70293960601B3E6C6003387E5029C
:1011F00063FAE600B386160163E6160163F4E600BF
:10120000B38616013386E640B376A602131E0E019E
:10121000135E0E013356A602939606013386C5026D
:10122000B3E5C60163FAC500B385150163E6150190
:1012300063F4C500B3851501B385C5406FF01FEF9A
:10124000E3EAD5E83707010063FCE604130EF00F6C
:101250003337DE0013173700B768018033D3E60059
:101260009388C8ECB388680003CE0800330EEE0004
:10127000130700023303C741631EC70363E4B600CC
:10128000636AC500B307C540B385D5403335F50063
:101290003388A54013850700930508006FF09FE38E
:1012A000B708000113070001E3E816FB13078001EC
:1012B0006FF09FFA3357C601B3966600336FD700BD
:1012C000B3D7C50113570F01B3F8E702B395650013
:1012D0003358C5013368B80093150F0193D5050144
:1012E000935608013316660033156500B3D7E7023D
:1012F00093980801B3E6D800B38EF50293880700EF
:1013000063FED601B386E6019388F7FF63E8E60142
:1013100063F6D6019388E7FFB386E601B386D6412C
:10132000B3FEE6021318080113580801B3D6E6020B
:10133000939E0E01B3EE0E01B385D502938706008E
:1013400063FEBE00B38EEE019387F6FF63E8EE0105
:1013500063F6BE009387E6FFB38EEE01B385BE4011
:1013600093980801B70E0100B3E8F8009387FEFFD9
:1013700033F8F8009356060193D80801B377F600C6
:101380003307F802B387F8023308D802B388D802CB
:101390003308F80093560701B386060163F4F6009C
:1013A000B388D801B70701009387F7FF13D8060168
:1013B000B3F6F600939606013377F700B3081801E9
:1013C0003387E60063E61501639E1501637CE50043
:1013D0003306C7403337C7003307E701B388E84017
:1013E000130706003307E5403335E500B3851541A3
:1013F000B385A540B397C5013357670033E5E700D0
:10140000B3D565006FF01FCD130101FD93D74501E2
:101410002322910223202103232C4101232861014F
:10142000232481019394C5002326110223248102E1
:10143000232E3101232A51012326710113975701CD
:1014400013090500130B0600138C060093D4C40087
:1014500013DAF5016304070A93FAF77F9307F07F25
:101460006380FA109359D50193943400B3E4990042
:10147000B7098000B3E9340113143500938A1AC008
:10148000930B000093574C011315CC001397570191
:101490009354C50093F5F77F135CFC0163000710BC
:1014A0009307F07F6382F516139534009357DB01A1
:1014B00033E5A700B7048000B3649500931F3B0099
:1014C000138515C01306000093972B00B3E7C700E0
:1014D0009387F7FF1307E000B3468A01B385AA405C
:1014E0006360F7163767018093972700130787E13A
:1014F000B387E70083A7070067800700B3E9A4006C
:10150000638E09066380040413850400EF30103EE7
:10151000930755FF1307C001634CF7029309D001ED
:10152000130485FFB389F940B3948400B35939019A
:10153000B3E99900331489009305D0C0B38AA5405C
:101540006FF01FF4EF30903A130505026FF05FFC67
:10155000930485FDB3199900130400006FF0DFFDBB
:10156000B3E9A4006384090213040500938904000D
:10157000930AF07F930B30006FF0DFF0130400004C
:10158000930A0000930B10006FF0DFEF13040000CC
:10159000930AF07F930B20006FF0DFEEB3EF64014E
:1015A00063800F086382040413850400EF30103455
:1015B00093050500938755FF1307C001634EF7029B
:1015C0009306D001938F85FFB386F6403395F401DF
:1015D000B356DB00B3E4A600B31FFB011307D0C072
:1015E0003305B7406FF01FEE13050B00EF301030DE
:1015F000930505026FF01FFC138585FDB314AB0046
:10160000930F00006FF09FFDB3EF640163820F0240
:10161000930F0B001305F07F130630006FF0DFEA25
:101620009304000013050000130610006FF0DFE9BB
:10163000930400001305F07F130620006FF0DFE82D
:1016400063E63401639C9934636AF4351396F901B7
:10165000135714009317F40193D919003364E6006B
:101660001395840093D88F01B3E8A80013550501A2
:1016700033D8A902939E080193DE0E01135704018B
:1016800013938F00B3F4A902930F080033860E035F
:101690009399040133673701637EC700330717014D
:1016A000930FF8FF636817016376C700930FE8FF95
:1016B000330717013307C740335EA7021314040131
:1016C000135404013377A70213060E003388CE03A8
:1016D000131707013367E400637E0701330717011F
:1016E0001306FEFF63681701637607011306EEFF1A
:1016F0003307170133040741939F0F013708010097
:10170000B3EFCF00130EF8FF13D60F0133F7CF015D
:10171000135F0301337EC301B303EE02B304C603B8
:101720003307EF02B302E6033306970013D7030132
:101730003307C70063749700B38202011356070191
:1017400033065600B70201009382F2FF3378570048
:1017500013180801B3F35300330878006368C4001A
:1017600093840F006314C40463F20705B387670012
:1017700033B76700330717013304E4009384FFFF96
:1017800063E688006394880263E267026366C400CC
:10179000631E860063FC0701B387670033B76700E9
:1017A000330717019384EFFF3304E40033880741C4
:1017B0003304C440B3B707013304F440930FF0FF80
:1017C00063848812B35FA402135708013374A40220
:1017D00013860F00B387FE031314040133648700DC
:1017E000637EF400330414011386FFFF6368140161
:1017F0006376F4001386EFFF330414013304F440DE
:101800003357A40213180801135808013374A402B3
:1018100093070700B38EEE021314040133648800AB
:10182000637ED401330414019307F7FF6368140146
:101830006376D4019307E7FF3304140113160601FE
:101840003366F6009317060193D707011357060175
:101850003308EF023304D441330FFF02B38EC703C2
:10186000330EC70393D70E01330FCF01B387E701C0
:1018700063F6C701370701003308E80013D70701F3
:1018800033070701370801001308F8FF33F5070194
:1018900013150501B3FE0E013305D5016368E4009D
:1018A0006310E424930F060063000504338488006A
:1018B000930FF6FF636414036366E4006310E4228D
:1018C0006370A3029317130033B36700B3081301C7
:1018D000930FE6FF33041401138307006314E4003D
:1018E0006304650093EF1F009387F53F6358F01082
:1018F00013F77F006300070213F7FF001306400091
:10190000630AC70013864F00B33FF601B384F401A6
:10191000930F060013977400635A0700B70700FF80
:101920009387F7FFB3F4F400938705401307E07F34
:101930006340F70A93DF3F001397D4013367F70141
:1019400013D53400939747013706F07F1315C50070
:101950008320C10203248102B3F7C7001355C500D9
:1019600033E5A7009396F601B367D50083244102BF
:10197000032901028329C101032A8101832A41012C
:10198000032B0101832BC100032C810013050700E9
:101990009385070013010103678000009385F5FF1D
:1019A000930700006FF0DFCB93060A0093840900D1
:1019B000930F040013860B00930730006308F60EA4
:1019C00093071000630EF60E93072000E31EF6F057
:1019D00013050000130700009307F07F6FF09FF6D8
:1019E00093060C006FF05FFDB7040800930F000032
:1019F00093060000130630006FF01FFC1305100063
:101A00003305F54013078003634CA70A1307F00161
:101A10006344A7069385E541B397B40033D7AF007D
:101A2000B395BF00B3E7E700B335B000B3E7B70045
:101A300033D5A40013F777006300070213F7F7000C
:101A400013064000630AC70013874700B337F70047
:101A50003305F50093070700131785006348070651
:101A60001317D50193D737003367F70013553500A7
:101A7000930700006FF01FED130710FEB307F74048
:101A800013060002B3D7F400130700006306C50075
:101A90009385E5433397B400B36FF701B33FF0018B
:101AA000B3E7F701130500006FF0DFF83705080012
:101AB000130700009307F07F930600006FF09FE884
:101AC00013050000130700006FF09FFA13050000D4
:101AD00013070000930710006FF0DFE613860F0076
:101AE000930F06006FF01FE0130101FD93D745012E
:101AF0002324810223229102232E3101232C410130
:101B0000232A51019394C500232611022320210387
:101B1000232861012326710113975701130405003F
:101B200093090600938A060093D4C40013DAF501E2
:101B30006306070A13FBF77F9307F07F6302FB102E
:101B40009357D50193943400B3E49700B70780000E
:101B5000B3E4F40013193500130B1BC0930B000002
:101B600093D74A011394CA00139757011354C40022
:101B700013F5F77F93DAFA01630007109307F07FFC
:101B80006300F51693D7D9011314340033E48700AA
:101B9000B70780003364F400130515C0939739002C
:101BA0001307000093962B00B3E6E6003305AB0065
:101BB0009386F6FF1308E00033465A01930515009B
:101BC000636CD8143765018093962600130545E5AC
:101BD000B386A60083A606006780060033E9A4004A
:101BE000630C09066380040413850400EF30005081
:101BF000130755FF9307C00163CCE7029307D00199
